:020000040800F2
:1000000000500020ADC3000859C40008BDAE000870
:1000100059C4000859C4000859C400080000000071
:1000200000000000000000000000000059C40008AB
:1000300059C400080000000059C40008ADAE000813
:1000400059C4000859C4000859C4000859C400081C
:1000500059C4000859C4000859C4000859C400080C
:1000600059C4000859C4000859C4000859C40008FC
:1000700059C4000859C40008FDAC000859C4000860
:1000800035AD000859C4000859C4000859C4000817
:1000900059C4000859C4000859C4000859C40008CC
:1000A00059C4000859C4000859C4000849AC0008E4
:1000B00041AC000835AC000829AC000859C4000860
:1000C00059C4000859C4000859C4000859C400089C
:1000D00059C40008C1AC000859C4000855AC000858
:1000E00059C4000859C4000859C4000800000000A1
:1000F0000000000000000000000000000000000000
:0C01000000000000000000005FF808F1A3
:100110002DE9F04F674B684C9FB02360002363606C
:1001200009F095FB18B906F05DFB09F0B3FB0AF086
:1001300035FA00230993614D0A930B934FF4E013B2
:100140000C932B685E4943F480338A7B2B60AB6948
:100150008B4643F01003AB612B6803F400330A9322
:10016000099B013309930A9B1BB9099BB3F5A06F47
:10017000F2D12968514B11F4003101D0022315E06E
:10018000186840F00100186009912B6803F0020321
:100190000A93099B013309930A9B1BB9099BB3F589
:1001A000A06FF2D12B68990739D501230B93454BEA
:1001B000454F196841F010011960196821F00301D9
:1001C0001960196841F0020119606B686B606B6817
:1001D0006B606B6843F480636B603C4B1968043B55
:1001E00021F0704159603A493960696821F47C1105
:1001F0006960596841F000415960D96821F40041B3
:10020000D9609B681B0449BF324B4FF4E0133B603D
:100210004FF480130C930B9B012B01D117E0FEE7E9
:10022000022B18D16AB10C9BB3F5801F02D14FF499
:10023000A01305E00C9BB3F5E01F02D14FF40013AF
:100240000C936A680C9B134343F4803302E06B68A1
:1002500043F460136B602B6843F080732B602A6853
:10026000164B9601FBD55A6822F003025A605A6871
:1002700042F002025A606B68104A03F00C03082B2C
:100280000593F8D15168144B01F00C01042903D0F7
:10029000082904D00E4A00E03A681A6028E0516844
:1002A0005068C1F38341C00301F1020118D40B4A25
:1002B0001CE000BFFD1E0008800600200010024068
:1002C000D819002000200240140000200410014032
:1002D00000127A00001BB7008400002000093D00D6
:1002E000526812F4003F3A6818BF5208514319602F
:1002F0006A681EAEC2F303123A4492F804A01A6868
:100300004FF0000922FA0AFABA4AC3F800A0BA4B21
:10031000BA489A60BA4ADFF82483DA60AA6942F0E0
:100320000102AA616A6A42F080726A62AA6942F0B6
:100330001C02AA614FF6FF7226F82C2D314602935B
:100340008DF84E9002F09CFAAE4A31461046039268
:1003500002F096FAAC48314602F092FAAB4948688E
:1003600040F000704860304605F042F91399A84803
:10037000029BB1FBF0F14FF47A70A160BAFBF0FA86
:10038000A4490AF1FF3048604FF0070AF02083F8D3
:100390002300C1F808906420C1F800A001F099FC86
:1003A0009D4B039A93E8030086E80300A96913981C
:1003B00041F00801A9610821116114A9029302F01A
:1003C0005FFA4FF40042ADF84C2014228DF84E2015
:1003D000AA694FF0020C42F004028DF84FC0874822
:1003E000AA613146CDF80CC002F04AFA8B4A8C491A
:1003F0004846116001F077FC029B083393E8030044
:10040000AB6986E8030043F00803AB61139814A9B5
:1004100002F036FA07F04EFDDBF80830102203F444
:10042000006308F10C00494602930EF01AF984F8B3
:100430000FA0029B0122A273DDF80CC043B188F823
:10044000182088F8192088F81A2088F81BA000E0E6
:1004500094466A49E0460A6800230846012199400B
:1004600001EA0C0E8E4506D199004FF00F0E0EFAE0
:1004700001F122EA01020133082BEFD102606B691E
:10048000684843F001036B61AB69DFF8989143F46E
:100490000073AB6105F035F8634B00251393634B94
:1004A000B8F1020F149314BF2B46802318934FF416
:1004B000807319934FF480631A93202331461B9362
:1004C00048464FF400531C931595CDF85880179566
:1004D0001D9504F0F8FFD9F80030B8F1010F43F092
:1004E0000103C9F80030524B98BF00215A6888BFF9
:1004F000012122F4702222F4807242EA01225A6021
:1005000099684C4A28460A4042F4602242F00202AE
:100510009A60D96A08F1FF3221F47001D2B241EA3F
:100520000252DA620123444A11188D78002D5AD004
:10053000825C5D1C092A91F803E0EDB23C4911D9B7
:10054000A2F10A0606EB46064FF0070C0CFA06FC71
:100550000EFA06FED1F80C8028EA0C0C4CEA0E06C6
:10056000CE600EE002EB42064FF0070C0CFA06FCE0
:100570000EFA06FED1F8108028EA0C0C4CEA0E06A2
:100580000E61062B2A490ED8013B03EB83034FF083
:100590001F0E0EFA03FE9A404E6B26EA0E0646EA3E
:1005A00002034B6320E00C2B0ED8073B03EB8303C5
:1005B0004FF01F0E0EFA03FE9A400E6B26EA0E064F
:1005C00046EA02030B630FE00D3B03EB83034FF09E
:1005D0001F0E0EFA03FE9A40CE6A26EA0E0646EA7F
:1005E0000203CB6200E01D460430102828D02B46C1
:1005F00099E700BF0000000800ED00E0000801409E
:100600000005FA05000C0140001001400000014007
:1006100040420F0010E000E02C0201088021002081
:10062000A1170008080002404C2401409C0600204D
:1006300000240140FDF7F1FF8C0600208006002019
:10064000AD4B9A6842F480729A609A6842F0010257
:100650009A609A6842F008029A609968A64A090767
:10066000FBD4936843F004039360A34A936813F0A8
:100670000403FAD19168BBF8E60041F4A00191604F
:100680009E4A50B9B2F9E83033B9B2F9EA30D3F141
:10069000010338BF002300E0034613F0010340F0DC
:1006A0008C803B7500B20AF071FD91A3D3E9002361
:1006B0000AF0D2FD0BF02AF8904F0646B7F9E80091
:1006C0000AF064FD8AA3D3E900230AF0C5FD0BF00C
:1006D0001DF80546B7F9EA000AF058FD84A3D3E9EE
:1006E00000230AF0B9FD0BF011F8814630460EF0F8
:1006F000E7F9074630460EF057FA804628460EF0D6
:10070000DFF9064628460EF04FFA054648460EF039
:10071000D7F9824648460EF047FA39468146504698
:100720000BF052F93946834648460BF04DF95146D5
:10073000049040460BF048F94946069040460BF0BD
:1007400043F93146079050460BF03EF94946606246
:1007500006F100400BF038F92946A062E5620698E0
:100760000BF032F9014604980BF026F82946206375
:1007700007980BF029F9014658460BF01BF8314653
:10078000606308F100400BF01FF92946A06358464A
:100790000BF01AF9014607980BF00CF82946E063B4
:1007A00004980BF011F9014606980BF005F839464C
:1007B000206430460BF008F96064514E4F4D3368A9
:1007C000DFF85CA143F0020333604E4B4FF0000BA7
:1007D0001B68B5F8EE90B3F8523095F8ED700493BD
:1007E0008AF800B008F0B4FE8046002800F00081CE
:1007F00094F84A30A4F848B00BB907F019FEB9F1E3
:10080000140F19D009D8B9F1050F19D0B9F10A0F91
:1008100014D0B9F1000F0DD114E0B9F1BC0F13D011
:10082000B9F5807F04D0B9F1620F03D102210CE049
:1008300000210AE0032108E0042106E0052104E08C
:10084000062102E0072100E001212F4B1A201A881F
:1008500022F040021204120C1A801A8822F0380288
:100860001204120C42F030021A801A8892B242F03E
:1008700040021A8007F0CEFD012001F01FFA13A8F4
:1008800008F0A8FC9DF94E30013303D19DF94C309E
:10089000013303D0B4F848309BB21BB10023A4F855
:1008A0004830A5E0194C1A4B64202360194BA1462F
:1008B0006360194BE36001F00CFAB8F1000F00F02F
:1008C000978004238AF80030144C0023062F2370ED
:1008D000DFF850B028D0092F02D0002F3DD123E0FF
:1008E000336823F00203336037E000BFAFF30080CA
:1008F000399D52A246DF913F00240140D8190020C3
:100900008802002018020020003001401C02002054
:10091000F11A0008D591000890C1793D9E0200208F
:10092000320200207D21002008F012FEA8B1324BD7
:100930000022A3F8482093F84A300BB907F078FD5D
:100940002E4B2F4A64201A602E4A5A6001F0C1F9DA
:1009500006238BF80030042323709BF8003033B952
:100960000FB11F46B0E7336823F0020333603368EA
:1009700023F00402326095F8E2200AB18AF80020E0
:1009800095F8E3200AB120490A7095F8E4200AB1ED
:100990001E490A709F0702D5184B1B689847D9F863
:1009A000003098473368144C13F0080F1DD0049A98
:1009B0004FF0640A0FFA82FB9BFBFAF738460AF005
:1009C000AFFF03460AFB17B000B202930AF0A8FF7C
:1009D0000F490AF0F9FF029B014618460AF0ECFEA7
:1009E0000C490AF0F1FFE06416E00023E36413E031
:1009F000032001F0A5F900BF800600208C02002032
:100A0000E11A0008399200089E020020842100208B
:100A10008988883C00002041C94B08221A614FF0A8
:100A20000A0AC74F1920FB680AF1FF3A83F008034E
:100A3000FB6001F04EF9012001F055F9192001F099
:100A400048F9002001F04FF91AF0FF0AE9D1082314
:100A50003B61BC4BBC4F1B68DFF81CB393F90C0027
:100A60000AF094FBB2A3D3E900230AF0F5FB0AF0E5
:100A70004DFE0EF025F8824638880AF051FF5146A7
:100A80000AF0A2FF0EF052F8B04BDFF8E8A218808F
:100A900038880AF045FF0146AD480BF049F8AD49EA
:100AA0000BF046F82065D9F80C000AF081FBA0A3F2
:100AB000D3E900230AF0D0FB9FA3D3E900230AF077
:100AC000CBFB0AF023FEA44B6979A44AA44F18601B
:100AD000A44B117007EBC101497C6365A24B4FF435
:100AE000A0721960A9681F4611F0200F18BF0123DA
:100AF0004FF000010AF1580018BF3B600DF0B1FD46
:100B00009A4A536823F4406343F0706343F40063EC
:100B10005360974BDA6942F00702DA619A6942F44E
:100B2000006242F00C029A61C4F898B104F01CFC17
:100B300016220AF5CE70FF210DF093FD002384F8F4
:100B40009C31336801229E0784F8B22107D58AF8C8
:100B50009D2103228AF8B22102228AF89E21580799
:100B600008D594F8B221511C84F8B2112244032113
:100B700082F89C1113F00A0F14D094F8B2310421BA
:100B8000E21882F89C115A1CD2B22244052182F844
:100B90009C11DA1C0233DBB284F8B2212344062212
:100BA00083F89C21AB68990608D594F8B221511CB2
:100BB00084F8B2112244072182F89C111A060ED53E
:100BC00094F8B2210920A11881F89C01911C0132EE
:100BD000D2B284F8B21122440A2182F89C116A79B7
:100BE000082A01D00E2A08D194F8B221511C84F8A9
:100BF000B21122440B2182F89C1194F8B2214FF0DB
:100C00000C0EA618511CC9B286F89CE15E07594823
:100C100084F8B21106D5023280F8B22101441022C4
:100C200081F89C2194F8B2214FF0120EA61886F894
:100C30009CE195F84561511CC9B2002E0CBF0026FD
:100C400003F001064B4884F8B21136B1023280F845
:100C5000B2210144132281F89C2194F8B2214FF073
:100C6000140EA618511CC9B286F89CE19E05414895
:100C700084F8B21106D502320144152380F8B2215E
:100C800081F89C313B4E0021982206F5DA700DF078
:100C9000E8FC39480AF066F8022000F069FFD4F851
:100CA00098A10146C4F84C0240B90090DAF8082037
:100CB0000220032306F022FFC6F84C020EA80021F2
:100CC00014220DF0CEFC6B790E2B01D0082B02D133
:100CD00001238DF842300025284A0023A85CD65C09
:100CE000D118864203D01033602BF8D1002108F0D0
:100CF00055FC83681B78012B04D01035602DEBD197
:100D00004FF000081E4A38689368003018BF012071
:100D1000C3F340018DF840001A488DF83D10C3F32D
:100D200080118DF83E100068C3F340312CE000BF05
:100D3000399D52A246DF913F000000A0F7C6B03EA9
:100D4000000C0140D802002000000020FC0200201E
:100D50000AE81C4100401C46D4020020EA0300209F
:100D60002C020108E81900200C05002000000140B9
:100D70000010024080060020041B0020F40201083D
:100D8000D8190020180200208DF83810C3F3C031A4
:100D90008DF83A1090F8B001C3F3C0218DF83B10E4
:100DA000C3F30041B2F8E050C0F380008DF83F106B
:100DB00003F00101DB0448BFB2F8DA308DF84100DE
:100DC000B2F8DE00ADF846504FF47A75ADF84850F1
:100DD00048BFADF84830B0F5FA7F84BF0023ADF8C6
:100DE0004830B2F818318DF83C80ADF84A3092F8AE
:100DF0002031BB4A84F85032002384F851325370BA
:100E00009DF842308DF83910002BADF8440014BF26
:100E10000223002301B10133B2494FF0000901EB75
:100E20008303D3F82831CA460493049A4FF6FF731C
:100E300032F809609E42F2B20CD1AB4B94F85122C9
:100E40001A70AA4B93F80090B9F1160F40F0708118
:100E5000002537E1A64F9DF83C104FEA021B07EB37
:100E60000B0519B1911E012940F217819DF83E1022
:100E700029B157F80B109F48814200F00E819DF870
:100E80003F1029B157F80B109A48814200F00581B4
:100E90009DF83A1011B1012A00F0FF809DF83D1035
:100EA00011B1042A00F0F9809DF83B1011B1052A18
:100EB00000F0F380360A022E9DF8381003D1002985
:100EC00008BF002603E0012E08BF9DF839609DF899
:100ED000400038B19DF8420020B9A2F10800012875
:100EE00098BF04269DF8410030B19DF8420018B922
:100EF000043A032A98BF0426A9B1F21ED2B2012AED
:100F000009D857F80B20B2F1804F00F0C68079491C
:100F10008A4244D1C1E0022E05D157F80B20764910
:100F20008A423ED1B9E0012E39D1744A4FF000080F
:100F3000FF2182F85482C2F85882C2F85C82C2F85B
:100F40006082C2F8948282F8981282F8991282F82C
:100F50009A82E97B82F89B8282F89C82C2F8A8522E
:100F6000AA686868ADF84C208DF84E10022213A9CB
:100F70008DF84F2001F084FC57F80B00297B424686
:100F800004F0AEFC284632464FF6FF7107F034FFFE
:100F9000284641465A4A5B4B05F0A2FE7DE0022EF0
:100FA00030D1594B5FFA8AF63001191800224FF000
:100FB00001088A708A724E7003F80080CD60A968BB
:100FC00095F80FE0ADF84C10022168688DF84F10CD
:100FD00013A98DF84EE0039201F052FC57F80B0074
:100FE000297B039A04F07CFC28464FF6FF714246A9
:100FF00007F002FF28463146444A454B05F070FE93
:10100000C2444AE0032E2ED1BDF844303B4EB3F526
:10101000FA7F96F852820FD93E4A2846B2FBF3F285
:101020000821BDF8483092B207F0AEF806EB88060A
:10103000C6F81C03384B0EE0384A2846B2FBF3F2E0
:101040000121BDF8483092B207F09EF806EB880601
:10105000334BC6F81C038360284B93F852220132AD
:1010600083F8522219E0042E17D1BDF846302B4ADE
:10107000224E92FBF3F22846BDF84A30012192B28B
:1010800096F8518207F080F806EB8803C3F84C030A
:1010900096F85132013386F8513209F10209B9F15B
:1010A000180F7FF4C2AEC8E61E4E97E80F002E441C
:1010B00086E80F001C4B10351A78C02D02F1010292
:1010C0001A7007D0636D002158595F190AF010FE9D
:1010D0000028E9D0154EB368DF0446D43FE000BFD6
:1010E000D10800202C020108C8040020EA030020D7
:1010F000D0180108000400400008004080060020CD
:10110000951900089D1A00081C0900201D590008A7
:10111000711A000800127A00BD1A000840420F0040
:10112000AD1A0008F003002050210020D81900203B
:10113000AB49AC4B01EBC90797F810E07F6983F826
:1011400000E0002FC6D000257545C3DAA64E2B015E
:101150001E443B440FCB013586E80F00F4E7B9F19C
:10116000080FDFF8F08226D128E09E4B93F800802C
:10117000B8F1010FF3D99D4D0027474505F1100542
:10118000EDDA55F8100C4FF07C510AF01DFC4FF0D1
:101190007C5145F8100C55F8140C0AF015FC4FF072
:1011A0007C5145F8140C55F80C0C0AF00DFC013775
:1011B00045F80C0CE1E7B9F10E0F04D198F80030B6
:1011C00043F0100303E098F8003023F0100388F890
:1011D000003007F09DFA8649864B8748874AC4F855
:1011E000703301600023B6F81801C4F86C13A4F83A
:1011F000763384F87833C4F87C23C4F8802380499C
:1012000058520233242BFAD17E4B7F4C1A60B368BC
:1012100013F0080F00F081807C4B002293F8163108
:10122000042B74D8DFE803F003032A505F00012B7E
:101230004FF0030208D184F88423072284F8863310
:1012400084F885230C2308E0022384F884330023E8
:1012500084F8863384F88523072384F887330023B2
:101260000093082001236A494FF4E13206F046FC5E
:10127000684BC4F88C03C4F8903344E00123664AF9
:10128000664900930820052306F038FCC4F894034F
:101290000546B6F818010AF043FB61490AF094FBD1
:1012A00060490AF087FA0AF07BFD00235E4A9850F5
:1012B0000433402BFAD15D4B281CC4F890334FF017
:1012C000100384F887331FE0009201230820584957
:1012D0004FF4E13206F012FC564BC4F89803C4F800
:1012E000903310230DE000920123082052494FF45F
:1012F000E13206F003FC514BC4F89C03C4F8903370
:10130000082384F88733003018BF012028B908204B
:1013100001F0E9F80023C4F89033B3685D0405D503
:10132000082284F88723464AC4F8902342F2010237
:101330001A4003F0010103F400505AB1414AC4F8C5
:10134000902318B1304A082082F8870311B10C228B
:1013500084F8872394F887231806A2F1040284F8FE
:10136000882340F18580284B374AD6F83811C3F8D6
:10137000A02300231A4A02EB0310D0F8640115469B
:10138000884204D00133DBB2042BF3D9002384F864
:10139000A5332E4B0020C4F8C03307F01FFD2C4BA3
:1013A00094F8A5231B680021C4F8AC3396F82631C5
:1013B00005EB02128B42C4F8A8134FF01000009105
:1013C000D2F864210CBF0123032306F097FBC4F875
:1013D000C403002840D1802001F085F83FE000BF21
:1013E0002C02010850210020F0030020F803002007
:1013F000E61A00206403010804010020F00900201F
:10140000CA0400200802002080060020D81900200D
:1014100045500008594F0008A086010051510008AE
:10142000CDCCCC3F0000B044240100200D5000087A
:10143000DD500008FD4F000891500008E94F0008FA
:101440003950000881170008041B0020FE1A0020F4
:10145000D4190020FE020020012007F0BFFCAB4B96
:101460001868AB4B00F5D97204301A6001F04EF9E0
:10147000A84BA949D4F87C230B608033C4F8C83347
:10148000A64BA74F1A60B3680025D9033D7040F101
:10149000B48001F077F801F0B1F801F08BF8012386
:1014A0002946A04840F22A323B700DF0DAF89E48F7
:1014B0002946836943F0080383619C4B1B68012222
:1014C0008A4002F01005954208D18A000F25954008
:1014D00023EA05030B2505FA02F21343013108291B
:1014E000EDD1924A924D1360C3694FF0010943F068
:1014F0000203C3618F4B00271A688F4BDFF87CA271
:10150000B2FBF3F22B88013A23F45C731B041B0C2F
:101510002B8092B21D23AB852A85A5F814902B8CC5
:101520004FF0100B23F001031B041B0C2B842B8C9E
:10153000A9882A8B23F0020322F0730212041B04F1
:10154000120C1B0C89B242F0600243EA0903A98025
:101550002A83AF862B842B8B23F008031B041B0CE0
:1015600043F008032B83B5F844306FEA43436FEA36
:1015700053439BB2A5F84430436943EA09034361EE
:10158000504603F0BEFF6D4B50461393654B13A9B5
:10159000149340F22A331693802318934FF48073E8
:1015A00019934FF400531C93CDF854B017971A9722
:1015B0001B971D9703F087FFAB890DA89BB243F4DF
:1015C0000073AB81DAF8003043F00203CAF8003050
:1015D0008DF834B08DF835908DF836708DF83790E1
:1015E00005F0C0FB564B1A68564BFA500437802F53
:1015F000F8D107F0AFFC07F0ADFCB3685A0546D54B
:1016000008F00EF8504B84F8F606986810F48060E5
:1016100009D0042006F028FD0146042007F0BEFF93
:10162000003018BF0120494B1870494B1D682B78BA
:1016300013B9484B1D6023E0012B21D1464F0021F7
:1016400038462C22C4F8F8560DF00BF88E237B7028
:101650004FF07C0AE0234FF07D09FB7087F800A073
:1016600087F82B903D4F002138462C220CF0F9FFD3
:101670008A237B70A02387F800A0FB7087F82B904B
:101680002B78022B08BFC4F8FC5606F099FA00F03C
:10169000FBFA334B18607379052B03D1314B4FF4B0
:1016A000C8721A80304B4FF47A721A8098F8003062
:1016B00043F0080388F800302C4B1A7822F002021D
:1016C0001A70B3689B071ED5294BC4F8003704F085
:1016D0001BFA282000F0FDFA059B013B0593F6D18B
:1016E000244B96F8051118780A460123904203D33B
:1016F0000133082B0A44F9D11F4A137096F80621CA
:101700005343A4F804371FB0BDE8F08F180200203F
:10171000D40300202C1B0020DC05002064060020E0
:10172000CC0500204C0A002000100240000C0140B3
:10173000000400408400002000366E0134040040A4
:10174000EC010108E0050020D81900201005002058
:101750001405002024050020480500207405002001
:1017600048030020A0020020782100207C210020D6
:10177000DC1A002028050020800000206C000240B8
:10178000014B33F81100704726110020034B4FF432
:10179000004208B11A6170475A6170470008014061
:1017A000034B4FF4004208B15A6170471A61704709
:1017B00000080140032810B50F4B0DD80F4A1268DE
:1017C00094888C4208D2D2888A4205D9012202FA32
:1017D00000F01A78104318701B780F2B0BD1064BB2
:1017E00000221A70064B998808B2142802DD1439B9
:1017F000998010BD9A8010BD880D0020D01900205E
:10180000F0090020024B9A8801329A80704700BF8D
:10181000F0090020074B1A68074B1178B3F9040050
:1018200053780B4403EB83039842D4BF002001207C
:10183000704700BFD0190020F0090020064BB3F913
:101840000400064B1B681B7803EB83039842D4BF4C
:1018500000200120704700BFF0090020D0190020AF
:1018600010B50446FFF7EAFF002814BF2046002009
:1018700000F0010010BD024B01221A72704700BF38
:10188000F0090020014B187A704700BFF0090020D2
:10189000034BB3F90400D0F1010038BF00207047BA
:1018A000F0090020014B00229A807047F0090020C7
:1018B00003685A1C026019707047016B0346C268C6
:1018C00010B5406941B1196C541A005D013918BF57
:1018D0000A46C0B21A6410BD196A405C0131B1FBFE
:1018E000F2F402FB1412C0B21A6210BD026B03695B
:1018F0001AB15168013B026C02E0C169026A013B06
:10190000881A1840C0B27047436B13B190F8440076
:101910007047826A436AD31A5842584170474379E4
:101920009B070AD5436A8269D154426A036901322E
:10193000B2FBF3F103FB112343627047437913F0C9
:10194000010307D0C368C169026A013B881A1840C5
:10195000C0B2704718467047437910B513F00103C1
:1019600004460DD0FFF7EAFF58B1226A6369985C1C
:10197000E3680132B2FBF3F103FB1123236210BDD4
:10198000184610BD426A806A131A5842584170477F
:1019900041717047334A10B5136C90681944081AA6
:1019A00040F68C2398429160D060516013463CD938
:1019B000127893F945108A420BD1111F082908D8D3
:1019C00093F84610182901D8013103E083F8442028
:1019D00002E0002183F8461093F944108A421CD19A
:1019E000204991F84710C1B1002191421E4806DA02
:1019F00003EB8104246920F811400131F5E7511E01
:101A000000EB41011630814203D0002421F8024F3F
:101A1000F9E7164908780130087083F8452000225C
:101A200001211A7083F8471010BD92F84710B9B120
:101A3000A0F2EF2440F2DA518C4208D811780B2939
:101A400005D80B1D0131117042F8230010BD002292
:101A500083F84720991804320020302A0861F9D110
:101A600010BD00BFD408002026110020CC15002096
:101A7000084B03EB0010837A0133DBB20A2B83722D
:101A800007D983781BB94178034A22F81130002323
:101A9000837270471C09002026110020024B1A6C2B
:101AA00011441964704700BFD4080020024B53F85A
:101AB00020301B68198070479C090020074BA1F556
:101AC0007A7153F820304FF47A701A689B884B4330
:101AD00093FBF0F39BB21380704700BF9C0900207A
:101AE000024B4FF480521A80704700BF0000002064
:101AF000704738B50C68054620460CF0F3FD2146CA
:101B000002462868BDE838400CF0F4BD034B1B6862
:101B1000DA79511CD9711344187A7047C005002036
:101B200010B5FFF7F3FF0446FFF7F0FF04EB0020CA
:101B300080B210BD10B5FFF7F3FF0446FFF7F0FFCA
:101B400004EB004010BD094B5A6882420AD01A6962
:101B5000824206D0DA69824208BF183302D00023DD
:101B600000E00C3300225A725A607047480000208F
:101B70000E4B1A7A824215D01A7D82420FD093F80A
:101B8000202082420DD003F124011A7A024001D0B4
:101B900043B909E00C338B42F7D1104670470C3340
:101BA00000E0183358687047184670474800002016
:101BB0002DE9F0478278C6781E4BC2F1640802EB2B
:101BC000820C54425FFA88F84FEA4C0CC6F1640963
:101BD000A4B203F11807A5B228B2002804DC002D36
:101BE00014BF1546012500E0454600FB00FA6D4391
:101BF0000AFB06FA9AFBF5F54D4468434FF00A0AD2
:101C000090FBFAF0604480B258800D88B1F802A0D1
:101C100000B2C5EB0A0A00FB0AF04FF47A7A90FB97
:101C2000FAF0054423F8025F0A34BB42A4B2D2D1D1
:101C3000BDE8F087AE0E002010B544780078002390
:101C400003FB03F11939614301F6C41159434143C0
:101C500040F6C41291FBF2F1034A22F8131001334B
:101C6000072BEDD110BD00BF980E002010B5044C1D
:101C70002068FFF7E1FF20680249BDE8104097E7C0
:101C8000E0030020A81A002010B5094A094913688A
:101C90008C6812689342F8D1074A106811684FF4B3
:101CA0007A725043001BB0FBF1F002FB030010BD41
:101CB000D419002010E000E08806002038B5044662
:101CC000FFF7E2FF0546FFF7DFFF401BA042FAD314
:101CD00038BD10B504462CB14FF47A70FFF7EEFF13
:101CE000013CF8E710BD08B5014B1B68984708BDDB
:101CF000802100202DE9F04106460F469046002540
:101D0000EBB2434518D20024E3B2B3420FD20B4BDF
:101D10000120DA68013482F00802DA60FFF7E3FF9D
:101D20003846FFF7D6FF0020FFF7DDFFECE73C2049
:101D3000FFF7CFFF0135E3E7BDE8F081000C01407C
:101D400040F2DB14604308B50A4B08221A61841E76
:101D5000084B2046DA6882F00802DA60FFF7B9FF24
:101D60000120FFF7C0FF1920FFF7B3FF0020FFF7A6
:101D7000BAFFEDE7000C014008B503685B699847BE
:101D800008BD08B503681B69984708BD08B5036816
:101D9000DB68984708BD08B503689B68984708BD8D
:101DA00008B503685B68984708BD10B5044C206807
:101DB000FFF7F6FF18B12068FFF7EDFFF6E710BD5B
:101DC000A805002008B503681B68984708BD064BA6
:101DD00010B5044621461868FFF7F4FF034B1B6853
:101DE0009A7954409C7110BDC4050020C0050020A4
:101DF00038B5044624200D46FFF7E9FF4D20FFF7D4
:101E0000E6FF002C084C0CBF3E202120FFF7DFFF2F
:101E10002368002228469A71FFF7D9FF236893F8B8
:101E20004900BDE83840D2E7C00500200146002047
:101E3000DEE7F8B50C4E0D4C0D4DC1B207463068CB
:101E40006170FFF7BFFF2B6861789A7930684A406C
:101E50009A71C7F307216170FFF7B4FF2B686178AF
:101E60009A794A409A71F8BDC4050020880D002077
:101E7000C0050020F8B5174D174C184F0646C1B2E3
:101E80002868A170FFF79EFF3B68A1789A792868BF
:101E90004A409A71C6F30721A170FFF793FF3B6890
:101EA000A1789A7928684A409A71C6F30741A170CF
:101EB000FFF788FF3B68A1789A7928684A409A71B1
:101EC000310EA170FFF77EFF3B68A1789A794A40F6
:101ED0009A71F8BDC4050020880D0020C0050020BF
:101EE00010B5441E14F8011F21B1034B1868FFF709
:101EF00069FFF7E710BD00BFCC080020014B186850
:101F000060E700BFFC11002038B5054C05465E2196
:101F10002068FFF757FF20682946BDE8384051E7A1
:101F200018050020014B5E2118684BE718050020BA
:101F300010B50A4C5E280146206805D15D21FFF7E7
:101F400041FF20683E2105E05D2903D1FFF73AFFFC
:101F500020683D21BDE8104034E700BF180500208F
:101F600010B50446C0B2FFF7E3FFC4F30720BDE895
:101F70001040FFF7DDBF10B50024094BE0B21B781D
:101F800083420CD9074B33F81010074B53F820301D
:101F90001BB10B2801D89B6898470134EDE710BDB1
:101FA00050210020522100209C090020054B1B6875
:101FB00003EBC00090F9063019420CBF01204FF02E
:101FC000FF307047B00400200A4B1A6802EBC002D1
:101FD000D379FF2B07D008490978994203D9074ADA
:101FE00032F8130004E00728D4BF908840F2DC5098
:101FF00000B27047B0040020070A0020CA04002085
:102000002DE9F04F0C68836889B0D0F800A0D0F8B3
:1020100004800646204603938B460CF051FD07468C
:1020200020460CF0C1FDDBF80440814620460CF050
:1020300047FD054620460CF0B7FDDBF808200446B6
:10204000104601920CF03CFD019A834610460CF0BC
:10205000ABFD39460290584609F0B6FC394604906B
:10206000029809F0B1FC59460590484609F0ACFCCD
:1020700002990690484609F0A7FC29460790584661
:1020800009F0A2FC0146504609F09EFC2146834619
:10209000069809F099FC0146059809F08DFB014668
:1020A000404609F091FC0146584609F085FB21465F
:1020B0008346049809F088FC0146079809F07AFBEA
:1020C0000146039809F080FC0146584609F074FB6C
:1020D0003060029905F1004009F076FC0146504657
:1020E00009F072FC21468346079809F06DFC014611
:1020F000049809F05FFB0146404609F065FC014683
:10210000584609F059FB21468346059809F05CFCC6
:102110000146069809F050FB0146039809F054FC6B
:102120000146584609F048FB21467060504609F0C8
:102130004BFC2946044609F1004009F045FC0146E4
:10214000404609F041FC0146204609F035FB39467E
:102150000446284609F038FC0146039809F034FC8F
:102160000146204609F028FBB06009B0BDE8F08FB9
:102170002DE9F84F384E0446376838460CF0A0FC7D
:10218000054638460CF010FD7668804630460CF067
:1021900097FC834630460CF007FDD4F804900646C1
:1021A0002946484609F010FCA76882464146384651
:1021B00009F00AFC0146504609F0FCFA2168824603
:1021C000584609F001FC41460446484609F0FCFB2C
:1021D000314609F0F9FB0146204609F0EDFA314697
:1021E0000446384609F0F0FB294609F0EDFB0146AC
:1021F000204609F0E1FA014650460CF063FD17490C
:1022000009F0E2FB08F0D4FF11A3D3E9002309F0A1
:102210004DF9134B044618680D4608F0C9FF0246F5
:102220000B462046294608F065FE00220D4B09F0BA
:102230003DF909F06BFA0CF079FC83B21A0444BF43
:1022400000F5B4739BB218B2BDE8F88FAFF300800D
:10225000182D4454FB210940000300200000E144F4
:10226000CC06002000002440064B1B7803F004033A
:1022700003F0FF001BB1044B1888C0F3C01000F03E
:10228000010070477C210020500300202DE9F0411F
:1022900002780346202A00F10100F9D0092AF7D07C
:1022A0002D2A02D10346414D04E02B2A08BF0346E4
:1022B0004FF07E551E460024334616F8012BA2F13E
:1022C0003007F9B209290DD83949204609F07CFBBD
:1022D0000446384609F024FB0146204609F06CFA12
:1022E0000446E9E72E2A17D1314F334616F8010B81
:1022F0003038C2B2092A0FD809F012FB394609F06A
:1023000017FC0146204609F057FA29490446384689
:1023100009F05AFB0746E8E71A7802F0DF02452A7F
:1023200038D15A782D2A02D10233012604E02B2A13
:1023300014BF013302330026013B002713F8012F9D
:10234000303AD1B2092903D80A2101FB0727F5E762
:10235000B7F59A7F28BF4FF49A77B8464FF07E5171
:10236000B8F1070F07D90846124909F02DFBA8F16B
:1023700008080146F4E707F0070737B108460C499B
:1023800009F022FB013F0146F7E72EB1204609F094
:10239000CFFB04E04FF07E51204609F015FB0146CB
:1023A000284609F011FBBDE8F08100BF000080BFA6
:1023B0000000204120BCBE4CF0B50124B0FBF4F578
:1023C0008D4201D34C43F9E70026DCB1B0FBF4F5B4
:1023D00004FB1500B4FBF1F41EB9002D01DC002C48
:1023E000F3D1092D03F101075FFA85FC04DD002A12
:1023F0000CBF5725372500E0302565441D70013698
:102400003B46E2E71C70F0BDF0B50124B0FBF4F5EB
:102410008D4201D34C43F9E70026DCB1B0FBF4F563
:1024200004FB1500B4FBF1F41EB9002D01DC002CF7
:10243000F3D1092D03F101075FFA85FC04DD002AC1
:102440000CBF5725372500E0302565441D70013647
:102450003B46E2E71C70F0BD70B50646B6FBF2F4F1
:102460000846154614B12046FFF7F6FF05FB146435
:10247000024B1B5D00F8013B70BD00BF6A1A0108EA
:102480002DE9F041069C002B06460F460CBF4FF08D
:1024900020084FF03008234613F8011B09B91546F0
:1024A00003E0002AFBDD013AF6E7002D04DD3046AB
:1024B0004146B847013DF8E714F8011B11B1304619
:1024C000B847F9E7BDE8F08180EAE073A3EBE07379
:1024D0008B4206DB002801DD401A704702D0084419
:1024E000704700207047034B9A6822EA000098600A
:1024F000704700BFD8190020114A30B50028B8BF76
:102500004042104C90FBF2F304FB03003C2568436F
:102510000D4D90FBF2F22D682D7B25B903EB830363
:1025200003EB830301E0C3EB031302EB830304FB20
:1025300002020B804FF47A7392FBF3F24A8030BDB3
:1025400080969800806967FF24050020094B1B785E
:102550006BB1094B1B685B7823B1084B1868C0F35B
:10256000C0407047064B1878C0F3800070470120C8
:10257000704700BF760D0020140500204C0300209A
:102580007C210020094A0A48002310B51168037015
:102590001A46CC1864880CB9CC5C24B104330132DF
:1025A000802BD2B2F5D1027010BD00BFDC05002037
:1025B0006006002010B50B4B0B4819780B4BDA78EE
:1025C0004B085C1E047001F0010109480B440370C4
:1025D00008495308581E087002F0010206491344C6
:1025E0000B7010BD7506002070060020880D0020BD
:1025F000720600207306002071060020F0B50F4A15
:102600000F4816780F4A00231768C3701A461946F8
:102610000546D0B2B0420CD217F8220001320409AC
:102620009C4200F00F00A8BF631C8842A8BF411C59
:10263000EFE7EB70044B1970F0BD00BF600600209F
:10264000880D0020DC05002075060020F8B5101A62
:102650000C461F4609F064F90546381B09F060F97D
:10266000174B079E196809F0AFF92946044628461A
:1026700009F0AAF921460746204609F0A5F90146C6
:10268000384609F099F80CF01FFB0E4909F09CF947
:1026900009F086FB069B2146186005F100400CF00E
:1026A00011FB094909F090F9084909F085F809F08A
:1026B00051FB0028BCBF00F50C40A0303060F8BDD5
:1026C000300000202C7D8E3FA00CB34500A00C46AE
:1026D00010B509F025F90021044609F031FB08B1D5
:1026E000204601E004F10040054909F021FA0549BE
:1026F00009F06AF90CF0E4F9034B186010BD00BF53
:102700008096184B35FA8E3C3000002070B5044698
:10271000007909F001F91E4909F00AFA1D4D1E4E13
:102720002860A07B09F0F8F8194909F001FAEE6079
:102730006860607909F0F0F8184909F0F9F9184D66
:102740002860E07B09F0E8F8114909F0F1F96860C8
:10275000607E09F0E1F8134909F0EAF9EE60A8603B
:10276000A07909F0D9F80D4909F0E2F90E4D286079
:10277000207C09F0D1F8064909F0DAF96860A07EFA
:1027800009F0CAF8074909F0D3F9EE60A86070BDF6
:102790000000C842781000200000FA4400002041E8
:1027A0008810002000007A44AC10002044F25063EE
:1027B000984203DDA0F50C40A0387047034B9842C7
:1027C000BCBF00F50C40A030704700BFB0B9FFFFA0
:1027D00010B50023094CDAB254F822400133844288
:1027E000F8D10023064CD8B234F8104001338C42A3
:1027F000F8D102EB8000C0B210BD00BFB4080108E0
:10280000080B010890F83B3210B57BB990F83A32CA
:1028100090F83922934209D201219940B0F8404200
:1028200001332143A0F84012DBB2F3E710BD8379F6
:10283000012B03D1D1F1010138BF0021D0F834318F
:102840005A681B8909B11361704753617047044B83
:1028500053F820301BB107289CBF1B6819807047B4
:10286000CC09002010B5054C00202188FFF7EFFFB0
:1028700061880120BDE81040E9E700BF6C0000203E
:102880002DE9F0410F88002347FA03F2D2072BD538
:102890008A7803F0070512F0100F18BF91F803C0F3
:1028A00002F00F0618BF46EA0C06AD004FF00F0C01
:1028B0000CFA05FC06FA05F5DC0850F82480282AF5
:1028C00028EA0C0C45EA0C0540F8245005D10122F9
:1028D0009A40C46824EA020205E0482A04D1012291
:1028E0009A40C4682243C2600133102BCCD1BDE8AA
:1028F000F081034B1A88013292B21A80704700BFF0
:10290000C8060020AFF30080A14A2DE9F04F1368FC
:10291000A04903F59C43A04D20330B60AB6885B004
:1029200013F4807F174604D09C4B1B681B681B69FF
:102930009847AB6842F201041C405CB9984E33786A
:1029400073B1964B1B681B681B68984705F0FCFD2C
:10295000347005E0934B1A7801321A7005F0F4FDDB
:10296000AB68DA0405D5904B1B68DB0701D408F08F
:1029700023FA8E4B3C681868037CCBB18C4A013B30
:1029800032F91300A0F57A70B0F57A7FA8BF4FF442
:102990007A7020EAE07008F0C3FF864909F0C8F8B1
:1029A000854909F011F809F0FBF97E4B588039E0B0
:1029B000AA68160436D57B4A5168611A002931DBB2
:1029C00004F59C41203151607C494E797C4931F8B5
:1029D0001660417CB6B296FBF1F0117A013101F03C
:1029E0000F0111720A44507218466E4E06F1090228
:1029F0009A5C01331044102B80B2F6D100B290FBE8
:102A0000F3F000B26428A8BF642020EAE07008F068
:102A100087FF6C4909F08CF8674908F0D5FF09F089
:102A2000BFF97080AB68D80510D5674B9C42674CE6
:102A300008D923681B681B6A984718B923681B6864
:102A40005B6A984723681B685B699847AA68DFF848
:102A500060A112F4805F504BB5F8DC10BAF9062083
:102A600007D0B3F81831581A824207DD19448A4258
:102A700002E0B3F81A319A42C0F228840122002100
:102A800095F8218195F82201B5F81A61B5F81C7105
:102A90000B463AF901409B08B442C4BF63F07F0380
:102AA000DBB20231BC42B8BF43F040030829F0D189
:102AB0003C4C617E994204D1A17EF92903D80131B1
:102AC00000E00021A1766376414B374F1978A1B918
:102AD0003B68D90707D582B93E4B1B78DB070CD57D
:102AE00006F0ACFD09E03B4B1B785E0705D510B145
:102AF00008F062F901E0002AFAD0A37E294A142BDB
:102B0000354E40F09980334B18F100081B7818BF00
:102B10004FF0010803F0040303F0FF0093B12C49C8
:102B20000B78002B00F08880537E5F2B01D108F0DA
:102B300043F9B8F1000F7FD0637E7D2B7CD108F084
:102B40003BF979E0537E572B0BD1244B4FF47A722B
:102B50001A80234B1B6813F008036DD1214A1380A0
:102B60006AE0A968490745D55A2B43D11E4B19780D
:102B700019B1187001221D4B4DE0D17E1C4B81F024
:102B80000101D17609B1042245E0062243E000BFED
:102B90006C2100200C020020D8190020080200201F
:102BA000000100208C0D00204C03002004010020B7
:102BB000CA04002000007A4400C07F448C06002034
:102BC0009C0600200000C842404B4C00FC0900203D
:102BD0002C0000207C2100201802002078210020F9
:102BE0008802002018030020CD020020CF02002020
:102BF000CE0200205D2B00F0EF825B2B00F0EE8216
:102C00005E2B0AD10322EAE2A72B40F00783AA4BEE
:102C10001A7842F004021A700EE0562B01D107F028
:102C200083FEA64A1378002B00F0EF82637E6F2BA1
:102C300040F0E58206F002FDAB68590731D5E37E2E
:102C40009BB19F4B1B785A070FD59E4BBAF90620B4
:102C5000B3F81A319A4208DD3B6813F0010304D13E
:102C6000994A32211180994AD3763B68DB030AD511
:102C7000974B1A782AB9974A127812B9924A322198
:102C8000118001220CE0934B1A7852B18C4A1278D1
:102C900002F0040202F0FF011AB919708E4B0122F2
:102CA0001A70D6F80090002309F1750B3B6009F10A
:102CB000770698460BF1020303EB080113F808208E
:102CC0004B7816F8010C9A420AD2314605F0E8FF1B
:102CD00030B116F8023C01229A403B6813433B6036
:102CE00008F10408B8F1A00F06F10406E2D17B4B0D
:102CF0001B7843B13B68DFF8FC8113F0020F784E7C
:102D000040F09A818FE109F21512019209F58B7654
:102D10009846019A16F8010C531C03EB080113F8AE
:102D200008204B789A4228D2314605F0B9FF20B3EB
:102D3000B0786C4B013800EB400096F804B01844B2
:102D40004FF00C0CF3780CFB0BFC00935F4B03F182
:102D50001C0909EB0C014A6882420ED0009A09F85E
:102D60000C2000228A60012202FA0BFB93F84C200F
:102D7000486022EA0B0B83F84CB008F10608B8F162
:102D8000480F06F10606C4D1574BDFF86C811E6868
:102D9000564B4FF00009D3F800B0D8F80030002BA4
:102DA00000F038811978002900F03481D8F8042027
:102DB000C2EB0B02002A0CDB0BF5FA72C8F80420F8
:102DC000012202FA09F294F84C0020EA020284F887
:102DD0004C2018F8040C5A780430C0B2002A40F095
:102DE000E1803AF91020B5F8180100F1C80C6245ED
:102DF00001DD9B7813E0C838824202DA9B785B429F
:102E00000DE0012303FA09F394F84C2022EA0303AE
:102E100084F84C300BF5FA73C8F80430FAE094F8F3
:102E20004C2042FA09F2D00700F1F480002B304A1E
:102E3000CCBF02200120013910700A2900F2E28083
:102E4000DFE801F0060F1B28315C6E80929CA60023
:102E500032781344FA2BA8BFFA2323EAE3733370C2
:102E600007E072781344642BA8BF642323EAE3735A
:102E700073703046FEF7E0FEC4E0F278304613444B
:102E8000642BA8BF642323EAE373F370216DFEF77C
:102E90008FFEB7E032791344642BA8BF642323EA82
:102EA000E3733371AEE072791344642BA8BF6423DB
:102EB00023EAE3737371A5E0FE0200202C000020DA
:102EC0007C210020D8190020B40200208C0D0020A5
:102ED000CC020020CD020020CF0200207B21002068
:102EE00050030020C4080108E0030020D41900208A
:102EF000CE02002088020020AC0D0020616D4A78CF
:102F00001A44C82AA8BFC82222EAE2724A700A7884
:102F10001344C82BA8BFC82323EAE3730B7071E0E6
:102F2000616DCA7A1A44C82AA8BFC82222EAE2728E
:102F3000CA728A7A1344C82BA8BFC82323EAE37352
:102F40008B725FE0616D4A7D1A44C82AA8BFC8220F
:102F500022EAE2724A750A7D1344C82BA8BFC8232F
:102F600023EAE3730B754DE0626D91780B44C82B37
:102F7000A8BFC82323EAE373937043E0626D117B1B
:102F80000B44C82BA8BFC82323EAE373137339E0AB
:102F9000626D917D0B44C82BA8BFC82323EAE3735D
:102FA00093752FE0012A2DD13AF910009B784FF448
:102FB0009662B0F5617F92FBF3F305DB40F63302D6
:102FC0009042B8BF024601E04FF46172A2F561720F
:102FD00092FBF3F3DBB2AB4A581C0C29107011D1F1
:102FE00094F858209A420DD0A74A042B28BF0223F8
:102FF0000A2184F8583001FB0323A44A06331360E6
:10300000FEF734FE012303FA09F394F84C2013432E
:1030100084F84C3009F10109B9F1040F08F10C08EA
:103020007FF4BBAE66E6AB68DB0514D5984B1B6836
:103030001B689B68984770B1D8F800309A070AD58A
:10304000338813F001020CD1924943F00103E26589
:1030500022660B8006E03388012223F001033380CF
:1030600000E000223B68580710D57AB1328822F080
:10307000010102F0020289B292B2318052B9E265D6
:103080002266844A41F00201118003E0328822F076
:1030900002023280D8F80020910640F188807E4AF2
:1030A000127892077CD57D4A1278042A78D913F4D5
:1030B000007C328812D002F010039BB2002B76D134
:1030C000744922F0200242F0100275480A80754AC5
:1030D000011D537006F0F7F9022366E022F010019B
:1030E00089B2580531802ED56F4B1B6858896F4BBC
:1030F000B3F90080B8F1000FB8BFC8F100088045EF
:1031000009DAB3F90230002BB8BF5B428342ACBF8F
:103110000023012300E06346DB0714D502F0200200
:1031200092B2002A43D15F4B61485A70614B41F023
:1031300020011A685B683180011D6367226706F011
:10314000C2F9012331E022F030023280554A53782F
:103150006BBB012151701A46574900205052574904
:10316000574C5052574904EB030C5052002119514F
:103170000232CCF80400CCF8081004F1280C5034CA
:1031800043F80C1019519C441C44042ACCF8040048
:10319000CCF808106060A16003F11403DCD106E0F4
:1031A000338823F030033380002384F86C303B688D
:1031B00013F4006F338814BF43F4807323F48073D7
:1031C00033806B79082B02D00E2B40F0928033882D
:1031D00023F0400333808CE0012200E002225FFAFA
:1031E00082F808F1FF3385F8543706F053FB07F0F7
:1031F000D5F9022028214246FEF77CFD1CE5B8F1F6
:10320000000F02D07E2B3FF415AD637E972B7FF429
:10321000FBAC2D4B4FF4C8721A800DE50022BB2B7E
:10322000039201D1022303E0B72B04D14FF6FE73C2
:10323000ADF80E300AE0BE2B01D1022304E0BD2B15
:103240007FF4FAAC4FF6FE73ADF80C303368BDF87E
:103250000C10B3F854200A44A3F85420BDF80E1003
:10326000B3F856200A44A3F8562006F013FB07F0E3
:1032700095F90F2014210122FEF73CFD0023A376CF
:10328000DAE400BFCE02002028210020E003002065
:10329000FC09002050030020FE0200203805002019
:1032A000F00D00202C000020D4030020C6030020D5
:1032B000FC0D00203C05002070210020D8030020D8
:1032C000040E0020DC030020A00200200A4B002294
:1032D0000021DA651A66C3F8F020C3F8F420C3F8B9
:1032E000F820C3F8FC10C3F80011C3F80411FFF76D
:1032F000C6BB05B0BDE8F08F8C0D002000000000BB
:10330000664B2DE9F04FB3F90600654B87B01D6899
:103310002B8998420EDBB0F5FA6FAF7907DAC21A43
:103320005743A3F5FA6397FBF3F7643703E0C7F15C
:10333000640700E064275B4B5B4AB3F8181193F90C
:10334000EC3016685B4204919BB200210593344631
:103350000A46524BDDF810C0CB5E40F2E63E0393C6
:10336000CCEB030303F2F31CF44503D8002BB8BFE6
:103370005B4201E04FF4FA73022ADFF8388131D062
:1033800096F85DE1BEF1000F04D07345CCBFCEEBE3
:10339000030300234FF0640EDFF814A193FBFEFC3F
:1033A0006FF0630B3AF81C900BFB0C3B0CF1010C1B
:1033B0003AF91CA00FFA89FCCCEB0A0C0CFB0BFCB5
:1033C0009CFBFEFCCC4428F801C095F804C003FB2C
:1033D0000CFC364B9CFBF3F373449BB27B4393FB97
:1033E000FEFE1BE096F85EE1BEF1000F04D07345CF
:1033F000CCBFCEEB03030023DDF814C003FB0CFEAF
:10340000A8F804E095F805E0002BB8BF5B4203FB89
:103410000EFE264B9EFBF3FE0EF1640EB31893F8DE
:103420000480DFF894C00EFB08F8642398FBF3F8DF
:1034300002F80C8094F80E900CF103080EFB09F9C9
:1034400099FBF3F902F8089094F818800CF1060C37
:103450000EFB08FE9EFBF3F302F80C30DDF80CE0E7
:10346000049B9E45DFF84CE004DA3EF801305B42F5
:103470002EF801300132032A01F1020104F10104A6
:103480007FF467AF074DB5F81A31984216DBB0F5F7
:10349000FA6FA8BF4FF4FA6011E000BFCA04002021
:1034A000E0030020D8190020180200200CFEFFFFC6
:1034B000980E0020C6030020A60E00201846C01A51
:1034C0004FF47A725043C3F5FA63B0FBF3F3642709
:1034D000A54C93FBF7F204EB42016FF0630000FB95
:1034E0000233098B04EB4202B2F91A000AB2821AC3
:1034F000534393FBF7F79D4B39441A889C4E500673
:10350000AEF806103ED59B4B1888238EC01A00B229
:1035100007F03CFE92A3D3E9002307F09DFE08F0DC
:10352000F5F807460BF0CCFA804638460BF03CFB2A
:103530000746B6F9020008F0F3F98146B6F9000033
:1035400008F0EEF94146824608F03EFA39468346D5
:10355000484608F039FA0146584608F02BF908F0B9
:10356000F9FB41463080484608F02EFA394680463D
:10357000504608F029FA0146404608F01DF908F0C7
:10358000E9FB7080AA6840F602031340002B53D079
:10359000794B06211E88636B1E4494F838306663AD
:1035A0000133DBB2B3FBF1F084F8383001FB1033A8
:1035B00013F0FF0F40D1910706D502F0A5FA02F0F3
:1035C0008DFA694B83F83900AB681A0532D56B4B1D
:1035D000E16B5A7B6A4B33F81200082391FBF3F23C
:1035E00080B28A1A0244E26392FBF3F292B240F68E
:1035F000E4435A43634B40F6FF71B2FBF1F21968A2
:103600004FF47A73C8888988121A5A4392FBF1F2F0
:1036100056435D4996FBF3F30A60D4E91001C018E4
:1036200041EBE371C4E910010023584A08F0D8FBCC
:10363000574B18600023636356494B4A0B6894F854
:10364000397013F4805318BF012382F84830AB68F7
:10365000894613F4807F504E2CD0DFF850813078AB
:10366000D8F80030C0F380001B685B68984760B1F1
:10367000012384F84930D8F800301B68DB6898478C
:1036800018B1394B022283F84920D8F800301B6862
:103690009B68984728B133785B075CBF022384F8A6
:1036A0004930D8F800301B689B69984710B1002357
:1036B00084F84930394B1A6890060DD5D9F8003096
:1036C00013F4C06F05D0364B1B78990701D4012342
:1036D00000E0002384F84A3094F84920224B022A63
:1036E00002D14C204E211CE0012A06D153204D214D
:1036F0004C220B4605F024FB2AE093F84A20012ACD
:1037000003D1532001464E2206E093F84820012AB7
:1037100004D15320014602464D23EBE727B1532045
:103720004D210A464423E5E710490A88120603D5CD
:1037300053204D210246DCE71A4A12781AB11920AB
:1037400005F0D2FA04E0384683F84B70FEF7CBFA66
:10375000327850072CD5144B08225A617EE000BF06
:10376000399D52A246DF913F980E00205003002061
:10377000C603002018030020440300208C0600200C
:103780009C060020800D00202C050020407E0500B6
:10379000300500204C0300207C21002088020020FE
:1037A000FE020020CE020020000C0140000A002092
:1037B000D9F80030D90703D4B64942F001020A70A3
:1037C000B54A12881AB1B5490A68920705D4B44AB5
:1037D0001288003218BF012200E0012242B1B14A32
:1037E000D16881F00801D160327822F00102327094
:1037F000AD4A1278170703D4327822F001023270F2
:10380000D80203D5337823F0010333703378A74A05
:1038100013F0010F05D00023E364A24B08211961C6
:103820000BE0E16C136841B9A14903F5F42303F5FA
:103830009073CB649B4B08215961E36C12686BB1A8
:10384000D21A002A0ADB974A03F5F423D16803F55C
:10385000907381F00801D160954AD36404F0B0F907
:10386000944B1B7813B102F099FEFBE3DFF86C82F6
:1038700098F84A30012B40F0EE838F4A8F4BD8F8EE
:103880000010C2F80080196091468C4B1868FEF752
:1038900087FA002800F0D983884B1868FEF77BFA76
:1038A000D9F8003093F84820DAB9B0F124014A423F
:1038B0004A4183F84820002AE7D133785B07E4D4F3
:1038C000232802D102F06AFEDFE77D4B1B681B7DD7
:1038D0008342DAD17B4A7C4B1A607C4A7C4BDA60AB
:1038E000D3E7012A04D14D2814BF00220222A9E304
:1038F000022A04D13C2814BF00220322A2E3032A97
:103900000AD140284FF0000200F29C831A71DA714C
:1039100058719871042295E3042A06D19A7983F8A4
:1039200049005040987105228CE3052AADD15979A0
:103930001A799142997906D941409971511C1971AE
:1039400013441872A1E7814240F0798393F849004B
:1039500006F040F8002840F06D83D9F8003093F865
:103960004930C82B00F0D98043D82D2B00F0F882C5
:1039700024D8252B00F0D68206D8212B00F02B82EC
:10398000232B00F06E8187E3292B00F0D6822B2BAE
:1039900000F0DF82272B40F07F830020FEF746FAFD
:1039A000FEF7BEF84B4FA7F8E600FEF7B9F8A7F808
:1039B000E800FEF7B5F8A7F8EA0038E3332B00F08B
:1039C000E3820CD82F2B00F0F482312B40F064837B
:1039D000404FC020FEF72AFA07F1800BFFE2412B8F
:1039E00000F0DA82442B00F01C83352B40F0548326
:1039F00059E1D02B00F0FD813FD8CC2B00F0818124
:103A000006D8C92B00F01782CA2B00F09E8043E332
:103A1000CE2B00F0028240F2F781FEF781F8FEF72C
:103A20007FF8A5F8D000FEF77BF8A5F8D200FEF7E6
:103A300077F8294FA5F8D400D7F800B0FEF770F852
:103A4000ABF8A801FEF76CF8FEF774F83F68FEF7D4
:103A500067F800EB80004000A7F85200FEF756F828
:103A600085F80401FEF752F885F80601FEF74EF8D6
:103A700085F80501FEF74AF8D9E2D42B00F07381EE
:103A80002ED8D22B36D040F21482FEF749F8A4F893
:103A90005000CCE27C210020A002002088020020FF
:103AA00078210020000C0140FE0200206C21002043
:103AB000980E00207B210020C0050020C4050020B6
:103AC00018080020EFBEADDEF04F00200400FA051C
:103AD00000ED00E0D8190020180200203408002072
:103AE000EF2B25D0FA2B00F0A281D62B40F0D48208
:103AF000002730E1337803F0040303F0FF07002BC5
:103B000040F09582FEF702F8022885F8540740F24B
:103B10007681CD4B83F8547771E10027FEF700F8EA
:103B2000CA4BD8530237102FF8D10122C84B7CE181
:103B3000C84FD7F800B0FDF7F3FFABF856003F6869
:103B4000FDF7EEFFA7F8540071E2C24F3B681B7807
:103B5000022B69D10027DFF8FCB2DBF800A0FDF7EB
:103B6000D5FF07F108020AEB820A07F0D5FEBA4931
:103B700007F0DEFFCAF80400DBF800A0FDF7C6FF7F
:103B800007F10A020AEB820A07F0C6FEB34907F002
:103B9000CFFFCAF80800DBF800A0FDF7B7FF07F178
:103BA0000E020AEB820A07F0B7FEAD4907F0C0FF2C
:103BB0000137032FCAF80400CDD1072F1BD1DFF83E
:103BC00094A2DAF800200192FDF7A0FF07F0A4FE0E
:103BD000A14907F0ADFF019ADAF800A09064FDF763
:103BE00095FF07F099FE9C4907F0A2FFCAF84C0028
:103BF000FDF78CFF14E0DBF800A0FDF787FF0AEB70
:103C000007031871DBF800A0FDF780FF0AEB07033C
:103C10009873DBF800A0FDF779FF0AEB070318762D
:103C200001370A2FC9D102E24FF0000BD7F800A0EC
:103C3000FDF76CFF0AEB0B031871D7F800A0FDF736
:103C400065FF0AEB0B039873D7F800A0FDF75EFF42
:103C50000AEB0B030BF1010BBBF10A0F1876E5D150
:103C6000E5E1FDF753FF272821D87A4B00F11C0B23
:103C70001B6803EB8B0BFDF749FF7A4B0BF1050734
:103C800003F58A72197A814203D00C339342F9D139
:103C90000DE01B788BF80530FDF738FF7870FDF7E5
:103CA00035FFB87053E0FDF731FF0B2804D9012030
:103CB0000021FEF79DF8BAE14FF0060B0BFB00F078
:103CC000644B00F588701B6803EB000BFDF71EFFCB
:103CD0000328ECD88BF80A00FDF718FF8BF80500D5
:103CE000FDF714FF8BF80600FDF710FF8BF80700B7
:103CF000FDF70CFF8BF80800FDF708FF8BF80900B3
:103D000095E1594FD7F800B0FDF700FF8BF80000A0
:103D1000D7F800B0FDF7FAFE8BF80100D7F800B035
:103D2000FDF7F4FE8BF80400D7F800B0FDF7EEFEC7
:103D30008BF80500D7F800B0FDF7E8FE8BF8060019
:103D4000D7F800B0FDF7E2FE8BF802003F68FDF700
:103D5000DDFEF8706BE1FDF7E3FE444BD85302370C
:103D6000102FF8D163E10027DFF8E8B0DBF800207E
:103D70000192FDF7D5FE019A07F12C034FEAC30A21
:103D80005244D080DBF800200192FDF7C9FE019A71
:103D900052441081FDF7C4FE072804D8DBF8002048
:103DA00002EB0A035873A0F57A739BB2B3F57A7FDE
:103DB00005D8DBF8003003EBC703A3F86A01DBF892
:103DC00000B0FDF7A3FE0BEBC7030137082F83F804
:103DD0006C01C9D12BE100271E4BD3F800B0FDF7D1
:103DE00095FE0BEBC7030137082F83F86D01F3D164
:103DF0001DE133785F0700F11A8102F0F3FC05F052
:103E000049FD06F0CBFB12E13378580700F10F8132
:103E1000174B4FF4C8721A8009E13378590700F143
:103E20000681144B1A7842F004021A70FFE03378CE
:103E30005A07E4D530E1FDF769FE0E4B1A78D8B188
:103E400042F002021AE000BFD8190020CA04002084
:103E50000402002018020020000020410000C84297
:103E600000007A44E8080108E0030020F404002080
:103E7000A0020020FE02002022F002021A70FDF7CC
:103E800045FE894B894F1870FDF754FE3860FDF7E9
:103E900051FE7860FDF744FE854B1880FDF740FE2B
:103EA000844B188094F8523043F0020384F8523067
:103EB000BDE0FDF72BFE0190FDF73CFE0290FDF703
:103EC00039FE8346FDF736FE0746FDF729FEFDF76E
:103ED00027FEFDF71BFE019A029B92B9764A82E803
:103EE0000808764A138823F010031380744B1A785D
:103EF00042F001021A70002F00F09980714B5F654B
:103F000095E0102A40F093806F4A82E808080FB1CC
:103F10006C4B5F656C486D4B0222011D1A7005F0F9
:103F2000D2FA84E00020FDF781FF0023AB60FDF7AB
:103F300001FEAB681843A86079E00020FDF776FF2A
:103F4000FDF7EEFDA5F80801FDF7EAFDA5F80A0169
:103F50006DE00020FDF76AFFFDF7D8FD687166E0AF
:103F60000020FDF763FFFDF7D1FD85F81601FDF791
:103F7000D7FDA5F81C01FDF7D3FDA5F81801FDF745
:103F8000CFFDA5F81A0152E00020FDF74FFFFDF725
:103F9000BDFD85F81E014AE00020FDF747FF002720
:103FA000FDF7B4FDEB190137082F83F80E01F7D1A7
:103FB0003DE00020FDF73AFF454F07F1400BFDF7CC
:103FC000AFFDA7F8D401FDF7A1FD87F8D601FDF7F5
:103FD0009DFD043787F8D3015F45F0D127E0FDF759
:103FE0009FFD00F03F00A7F85601FDF799FDB7F8D7
:103FF0005621800100F4F8631343A7F85631FDF70A
:1040000085FD000187F85401FDF780FD97F85431D4
:1040100000F00F00184387F8540104375F45DED1E4
:1040200005E00020FDF702FF012384F8583000204E
:10403000FDF7FCFED9F800309879FDF7C8FED9F8F5
:104040000030002283F848201FE494F8583013B160
:10405000204A214BDA60DFF894C008F14C08E045B3
:104060007FF406AC1D490B689B060FD51C4BE26D17
:104070001B689A1A002A09DB0B4A1278042A05D910
:1040800003F512330F4A03F5F873D365154B9B689C
:104090003BB11548984704E001200021FDF7A8FE38
:1040A000C8E707B0BDE8F08F380500203C050020C8
:1040B0003605002034050020F00D002050030020BC
:1040C000FE020020980E0020FC0D0020F80D0020BC
:1040D000D81900200400FA0500ED00E08802002055
:1040E0006C2100201C02002022050020CC080020AA
:1040F0002DE9F04F974B91B01B68BBB9964C2378D4
:10410000013B042B00F20487DFE813F01D061D06B7
:104110001D06F206D8062068FDF73DFE8F4B0446CB
:104120001B681B784BB1012B00F0ED80894C206897
:10413000FDF736FE0028EED1E0E72428884D0CD0AC
:1041400006D80A2800F08E800D2800F08B80C6E08B
:104150002A2806D02C2804D0C1E02B706B70AB70DD
:10416000CEE06A782E782A4400217D4BD170EEB9DA
:10417000DA789E74472A19D11A79502A16D15A79B9
:10418000472A07D19A79472A04D1DA79412A01D1FD
:1041900001229A746A79724B522A07D19A794D2A70
:1041A00004D1DA79432A04BF02229A74AB7C6C4FA3
:1041B000012B02D0022B36D049E0B31E072B46D884
:1041C000DFE803F0040810141C27452C02F03CFE25
:1041D00068613CE0EA78624B532A38D15A6952420E
:1041E0005A6134E002F030FEA86130E0EA785C4BBE
:1041F000572A2CD19A6952429A6128E0EB78302BE9
:10420000584B1A788CBF42F0020222F002021A7058
:104210001DE0002002F072FE287718E0002002F076
:104220006DFEE88313E0072E06D0082E0FD1012083
:1042300002F064FE78840AE0012002F05FFE41F2A1
:10424000184358434FF47A72B0FBF2F33B840136C3
:1042500000232A2C424A2E706B704CD1012182F827
:1042600024104DE095F82430002B34D03C4BDB7803
:10427000402B04D9A3F137021201D2B202E01B0194
:1042800003F0F0022B79A978402B8CBF373B303BF1
:10429000DBB21344DBB29942314A1BD1937C012B30
:1042A00008D0022B16D1118C2F4B528C19802F4B1A
:1042B0001A800FE02B4909788E070CD52C495069DC
:1042C000086090694860107F2A490870D18B2A4A9B
:1042D000118000E00023002285F8242010E06B7894
:1042E0001F4A0E2B03D8591C13445170DC7095F8EB
:1042F00024301B4A1BB991784C40947000E0002395
:1043000003F0010361E1164B002193F82520082AF0
:1043100000F25A81DFE802F00B0514324353718D2D
:104320009A00622801D1022207E083F82510B52CFB
:1043300040F04A8193F82520013283F8252043E19B
:10434000032283F8252083F8260083F8270083F8CA
:10435000280039E1440A0020240A0020400A0020F5
:10436000F80E0020FE02002034050020BC180020BA
:104370003C0500203805002036050020042283F883
:10438000252093F8272093F828100244D2B283F80E
:1043900027200A4483F8282083F8290014E1052205
:1043A00083F8252093F8272093F828100244D2B2EE
:1043B00083F827200A4483F82820588504E1062141
:1043C00083F8251093F8271093F828002144C9B2E8
:1043D00083F82710014483F82810598D6C4A01EBAB
:1043E0000424A4B2B4F5007F89BF0021548551850F
:1043F00082F8251000229A85E6E093F8272093F8AA
:1044000028100244D2B283F827200A4483F82820D7
:104410009A8DC72A03D85E49114481F830000132D1
:1044200092B29A855B8D934240F0CE800722584B22
:1044300083E7082283F8252093F82730834200F091
:10444000C380534A002382F82530BEE083F825104C
:1044500093F828104E4A814240F0B68092F8291015
:10446000062947D004D8022912D003292CD0ABE06A
:1044700012295CD0302940F0A78092F83410454AC8
:10448000102988BF102111701078434900225CE088
:104490004249506B4860906B0860116C4FF47A7021
:1044A00091FBF0F13E48018092F8F8103D4A19B1B5
:1044B000117841F0020102E0117821F0020111703F
:1044C000012283F8F92055E092F8351011F001012E
:1044D00005D092F83420D41E6242624100E00A46C0
:1044E00083F8F820002A45D12E4A117821F00201E4
:1044F00011703FE092F83B1011F0010105D092F8E5
:104500003A20D01E4242424100E00A4683F8F82099
:1045100022B9244A117821F00201117093F85F103A
:10452000214A1170B3F85C10204A118022E0516CCE
:104530001F480180916C42F2107091FBF0F11D4810
:104540000180012182F8FA1014E0824201F10C018D
:1045500010DA11F8045C184C155511F8035C174C6F
:10456000155511F8015C164C15550D78154C15555F
:104570000132EAE793F8F930054A2BB392F8FA30A2
:1045800013B3002382F8F93082F8FA3001231CE0DB
:10459000F80E0020BE180020280F00203C05002047
:1045A00036050020FE020020380500208200002091
:1045B00034050020BC180020BF180020CF180020B0
:1045C000DF180020EF1800200023002B3FF4AEADD1
:1045D000A54BA64E9A68DA6032689A60A44B1A68B6
:1045E00042F020021A60A34B1A78012A0CBF002265
:1045F00001221A70A04B1A7891077FF597AD9F4959
:10460000097804297FF692AD9D49097801F00401EB
:1046100001F0FF0011B922F001021A701B78964FC9
:1046200013F0010F974C984D11D180B19B070ED517
:10463000964B28686A6818605A60FEF749F8944BF0
:104640001B88A4F8FC303B7843F001033B7094F8DE
:10465000FE304FF00509013393FBF9F909EB8909A5
:10466000C9EB03098B4B8C481B7884F8FE900593AB
:10467000831D03EB890907900023DFF80CE2874ACA
:1046800053F80E00864F985090FBF7FC02F1080794
:1046900043F807C0834F03EB0E0107FB0C0742F200
:1046A000107097FBF0F00691079980B221F8020F85
:1046B00002F1100A03EB830B0490079153F80A00F0
:1046C00059F80B1049F80B70C1EB000808EB070014
:1046D000734F4FF0050843F80A0090FBF8F007FB12
:1046E0000C000599183201299850774608D1DDF859
:1046F00010E0AEF10202B2F5797F9CBF0699086026
:104700000433082BB9D1DFF87C813068D8F84C31FC
:10471000C01A07F001F9644907F00AFA33684FF04C
:104720007E51C8F84C31814607F0ECFA10B94FF0D1
:104730007E5000E048460CAAC4F85001534B00924A
:104740000DAA019297E803000CCBFDF77FFF0C9BAD
:1047500056496422B3FBF2F30D980B80544B90FB47
:10476000F2F21A80444A474E127812F0010208BF52
:104770001A8098F8543108BF0A80002B3AD0D6F836
:1047800050114FF07E5007F0D3F9D6F858318146DA
:104790002868C01A07F0C4F8494607F015F907F071
:1047A000D9FAD6F85C211FFA80FA68680FFA8AFAFB
:1047B000801A07F0B5F83F4B196807F005F949462C
:1047C00007F002F907F0C6FAB6F9623100B2C21872
:1047D000B6F960310221534492FBF1F293FBF1F3FD
:1047E00092B29BB2A6F86621A6F86431A6F86221BF
:1047F000A6F86031012388F854312F4B79681B8863
:10480000386803F030031F4D1F4EC8F85C11C8F81C
:104810005801002B3FF48AAC05F5B873009305F5F9
:10482000BA730193D5F86821D5F86C31FDF70EFF06
:104830007368D5F86C01C01A07F072F81D4B19683F
:1048400007F0C2F807F086FAD5F868313268C5F883
:104850007C019B1AC5F878310E4B1B78012B2DD0AB
:10486000022B00F0F98061E4240A0020D419002012
:1048700088020020EA0E0020FE02002038050020F9
:104880007C210020F80E00203C050020F00D0020C7
:1048900018030020F80D0020F60F0020241000203F
:1048A00080969800806967FF00007A44A005002088
:1048B000A20500203000002050030020D5F88071B0
:1048C000D5F89C410497D5F8907104F10040059704
:1048D000D5F89471D5F85061079707F03BFA8046F8
:1048E000204607F037FA904BD5F898511B688F4C4B
:1048F0000695089009930025DFF850A25AF8157024
:10490000AAF11403384635F8039007F009F8049922
:1049100007F05AF807F01EFAC9EB000080B20AF15E
:10492000280A25F80A000FFA80FA504606F0F8FF28
:10493000059907F049F807F00DFA1FFA80FB0AEB1A
:10494000070006F0EDFF079907F03EF8314607F043
:104950003BF8216806F030FF07F0FCF9404505DB25
:10496000DDF820E07045A8BF704600E0404606F044
:10497000D7FF206007F0EEF958441FFA80FB60680B
:1049800009F13109381A06F0CBFF314607F0D0F8AB
:104990000999206184468878D4F808A0CDF80CC025
:1049A00006F0BAFF06F004FC5DA3D3E9002306F08D
:1049B00053FC02460B4600205D4906F077FD06F0E9
:1049C000A5FE314606F0F8FE0146304607F0B0F885
:1049D000DDF80CC0034651466046039306F0EAFE3C
:1049E000039B0146184606F0EFFF0146504606F0CD
:1049F000E3FE1FFA89F9B9F1620F01462061676091
:104A0000A0600ED9069806F0DFFF07F0A3F9494B26
:104A1000B0F5FA6FA8BF4FF4FA609842B8BF1846D5
:104A200000E00020834440F6B8330FFA8BFB9B452F
:104A3000A8BF9B46404B0A229B45B8BF9B466A4392
:104A40003E4B54F8141B25F803B03D4B0235042DA2
:104A5000D1503FF46BAB4FE7334BD5F870B11F68C3
:104A6000B5F8A461B7F808904FEA5B03994528BFF1
:104A7000994633B2994502DC1FFA89F90BE03149B6
:104A8000D5F8500106F0A0FF07F064F930441FFA92
:104A900080F9A5F8A491D8F87451D8F8A861AE1B94
:104AA0003046FDF783FE0028D8BF404241F2931301
:104AB0009842CCBF00200120002849D0304606F0A3
:104AC0002FFF214906F080FF0AF06EF8064658468F
:104AD00006F022FF0146304606F076FF07F03AF96D
:104AE00080B240F6B83203B29342A8BF1346124ACE
:104AF000A8F8AC019342ACBFEB18AB1848F6A04243
:104B0000934203DDA3F50C43A03B04E0002BBCBFA4
:104B100003F50C43A033C8F8B0311BE0AFF30080BD
:104B2000182D4454FB211940D40300202C0E0020E2
:104B30000000F03F30F8FFFF48F4FFFFDC030020E7
:104B4000540E00200000C842D302373970100020F4
:104B5000C8F8B051D4F8B021C2F50C5028300492F6
:104B600006F0DEFEA44906F02FFF054609F0A8FF77
:104B70000F9028460AF018F8D4F8C051D4F8B43190
:104B8000D4F8B8E10E9005F100400793CDF828E085
:104B900007F0E0F80590284607F0DCF8D4F85081DB
:104BA000D4F8BC410B900994944C0025484606F07B
:104BB000B7FE0EAB53F8151006F006FFDFF874A22F
:104BC00006463AF9050006F0ABFE0146304606F00F
:104BD000F1FD07F0BFF88A4B06B2B6F57A7FA8BFA1
:104BE0004FF47A769E42B8BF1E46B0B20AF13C0A34
:104BF00025F80A0000B206F093FE0799824606F0F7
:104C0000E3FE07F0A7F880B208900A99504606F034
:104C1000DBFE414606F0D8FE216806F0CDFD07F028
:104C200099F80599884204DB0B9A9042A8BF104678
:104C300000E0059806F074FE824620606068143437
:104C4000301A06F06DFE414606F072FF54F80C3C37
:104C500044F8040C8446B8780693CDF80CC006F0EE
:104C60005BFE06F0A5FA62A3D3E9002306F0F4FA8E
:104C700002460B460020634906F018FC06F046FD8C
:104C8000414606F099FD0146404606F051FFDDF829
:104C90000CC0034606996046039306F08BFD039B08
:104CA0000146184606F090FE0146069806F084FD7F
:104CB00044F8106C014644F8040C44F80C0C0998B4
:104CC00006F082FE07F046F8089E0644504607F0BC
:104CD00041F8304440F6B83300B29842A8BF1846B5
:104CE000494B0A229842B8BF18466A43474BE852DC
:104CF000474B0235042D42F803A07FF457AF3B79B0
:104D00002BB104986422434B90FBF2F21A803B884B
:104D1000414C9B450ED9D4F8A831D4F87401C01A7F
:104D2000FDF744FD42F210730028B8BF404298429C
:104D30007FF7FCA9394B01221A70B4F8FC20354BDF
:104D40001A80FFF7F3B9364A116890460F7817B109
:104D5000012F0DD0AFE0012B00F2AD806278314B16
:104D600003EB0213304A59681068FDF70FF89FE013
:104D70002D4E3068FDF705F8B146002800F09B8005
:104D800023782A4D022B29D0032B55D0012B40F03C
:104D90009280274B1F686B69FB1A632B40F28B8054
:104DA0002B69042B18D8DFF87C80306808EB0313DC
:104DB0005968FCF7EBFF6B78366808EB03139D68C6
:104DC00015F8011B19B13046FCF7FCFFF8E7236921
:104DD0006761013323616EE002206AE06A78114B5B
:104DE000306803EB02135968FCF7D0FF032060E042
:104DF000182D4454FB211940D3023739540E00209A
:104E000018FCFFFF0000F03F48F4FFFFDC03002028
:104E10002C0E0020E80E0020F80E0020F80D0020D7
:104E2000400A00208C030108440A0020240A0020C4
:104E3000D41900205C1000202B7E03B92F76227E2F
:104E4000354B012A14D11A697B2A0DD8D8F80030C5
:104E50009B782BB9314BD9F80000995CFCF7B2FF75
:104E600023690133236103E000221A6102221A76CA
:104E7000227E294B022A18D11A690F2A13D8D8F892
:104E80000030997859B95B78244903EB03130B443C
:104E90001A44D9F8000092F87D10FCF793FF2369BB
:104EA0000133236101E003221A76237E022B02D90B
:104EB000042003F093FF0023636029E06368052268
:104EC00001336360637801200133DBB2B3FBF2F29C
:104ED00002EB82029B1A6370114B00221B68A360D5
:104EE000104B1A70104B1A7822F002021A700DE063
:104EF0000B4B1A68A368D21A40F6C4139A4207D91A
:104F00000A4B05201A6822F020021A6003F066FF9F
:104F100011B0BDE8F08F00BF240A0020FC09010891
:104F2000D419002038050020FE020020880200204D
:104F3000084BDA68D10709D4DA68520708D4DB686D
:104F400013F0100F0CBF042003207047012070479E
:104F500002207047002002401E4B2DE9F0431A78D2
:104F60001D460AB31C4B07781E781C4B93F800C0F3
:104F700002231B4A03F10108D45C344104F00F04FE
:104F8000BC420CD20B2C0AD812F8039012F80880FD
:104F900002EB840209EA0C0408EB042414610233D6
:104FA000102BE6D100232B7003788B420FD90C4BCA
:104FB00093F8400060B10B4A890012780B441869DD
:104FC00002B1400800F5777080B2BDE8F0830020A0
:104FD000BDE8F08308010020040A0020050A002033
:104FE000BC100020060A002007299ABF024B33F8A4
:104FF00021000020704700BFE4010020024B53F85D
:105000002100C0F3CF0070478C01002008B5074B8A
:1050100053F8210006F080FC054906F0D5FC05494F
:1050200006F0CAFB06F0BCFE80B208BD24010020D9
:105030000000203F00005C44014B33F81100704732
:10504000CA04002038B5104C0123054684F84030CE
:10505000FCF71AFE636C41F28832C31A9342A364D0
:1050600084BF002384F84C3094F84C30EDB20F2B01
:105070006064E55403D1054B01221A7038BD024A21
:10508000013382F84C3038BDBC10002008010020EC
:1050900010B50446FCF7F8FD0D4B41F288311A6D4E
:1050A0001865821A8A425A6584BF002283F8582004
:1050B00093F85830074A142BD45403D1064B0122DD
:1050C0001A7010BD024A013382F8583010BD00BF7B
:1050D000BC100020CD010020CC01002010B50446FA
:1050E000FCF7D2FD164AD36DD065C31AB3F57A6FBB
:1050F00084BF002382F8603092F8603023B9A82C76
:105100001CD110490B7006E0022B02D10E490C7025
:1051100001E0242B01D80D49CC540133DBB282F8D5
:105120006030094A127852000532934206D1044B8E
:10513000002283F86020034B01221A7010BD00BFCB
:10514000BC100020640100208A01002065010020BD
:1051500038B50446FCF798FD114B40F6C4115A6E61
:105160005866821A8A4284BF002283F8682093F826
:1051700068200AB90F2C11D10A480021017052B1E0
:10518000094D182A154405F8014C04D1012283F871
:105190006810027038BD013283F8682038BD00BF46
:1051A000BC100020090100200A0100202DE9F04F69
:1051B000064689B00F4615469B462978002900F01F
:1051C000B880252902D001353046B0E06C78302C0B
:1051D00003D002354FF0000903E0AC784FF001092D
:1051E0000335A4F13003092B4FF000081AD8A4F1BD
:1051F0003003DAB2092A07D80A2B13DC0A2202FB91
:10520000083815F8014BF2E7A4F16103052B02D829
:10521000A4F15703F0E7A4F14103052B02D8A4F150
:105220003703E9E76C2C03BF2C78012201350022FB
:10523000632C66D006D8252C77D0582C3FD0002C74
:1052400077D0BAE7732C63D002D8642C11D0B4E7BE
:10525000752C02D0782C32D0AFE70BF1040A05ACE4
:10526000DBF800000A2112B10022234613E0234696
:1052700020E00BF1040A05ACDBF8000072B1002855
:1052800006DA2D238DF8143040420DF1150300E0AD
:1052900023460A210022FDF7B7F80DE0002806DAC0
:1052A0002D238DF8143040420DF1150300E0234604
:1052B0000A210022FDF780F8D34600941AE00BF192
:1052C000040303930DF1140ADBF80000102132B13E
:1052D000583C624262415346FDF796F806E0B4F14D
:1052E00058035A425A415346FDF766F8DDF80CB0B0
:1052F000CDF800A03046394642464B46FDF7C0F88F
:105300005BE730469BF800100BF10404B8470AE055
:10531000DBF80030304600933946424600230BF15B
:105320000404FDF7ADF8A34647E730462146B847E9
:1053300043E709B0BDE8F08F70B50546441E14F888
:10534000011F61B1064E304609F0BFF90028F6D0C2
:10535000861B0448631B304480F80E31EFE770BDB4
:1053600090250108D8190020124870B50023047850
:105370001A46D1B28C4209D0057B8D4208D00D4D22
:105380002D7E8D4208BF02210ED102E0002100E0F7
:1053900001210C2505FB0101074D084E1D4495F820
:1053A0002C510133755D0D720132052A01D0022B9B
:1053B000DFD970BD48000020D81900204A1B010821
:1053C00030B587B005460C4603A800210C2209F031
:1053D00048F92846002106F0B3FC20B128462A49A6
:1053E00006F0EAF903E02846274906F0E3F92749E1
:1053F00006F0EAFA06F0AEFC054685EAE570A0EB99
:10540000E57069460A22FDF727F800239D420370E4
:10541000ACBF20232D2368468DF80C3009F062F9CB
:10542000012807D130238DF80D308DF80E308DF81E
:105430000F300CE0022805D130238DF80D308DF8A7
:105440000E3004E0032804BF30238DF80D30694688
:1054500003A809F02DF903A809F044F90338C5B2EF
:105460002A4603A9204609F067F900236355204620
:10547000074909F01DF903A92046294409F018F944
:10548000204607B030BD00BF6F12033A00007A44D7
:10549000481B0108826A8169436B1144D960416AE3
:1054A000914203D98A1A5A60816204E001698A1A1A
:1054B0005A6000228262002280F844201A6842F07A
:1054C00001021A6070478A6810B50C6A03681443B9
:1054D0000A6923F4FF4314434A6923F07003144319
:1054E0008A691443CA6914434A6A14438A6A224384
:1054F00013430360CB6843600B6883604B68C360F1
:1055000010BD02684FF6FE73134003600023036072
:1055100043608360C3602A4B984222D0294B984253
:1055200029D0294B984230D0284B984237D0284B6D
:1055300098423ED0274B984206D153F8682C42F44B
:10554000700243F8682C7047234B984206D153F8F9
:105550007C2C42F0706243F87C2C70471F4B9842C1
:1055600006D153F8042C42F00F0243F8042C704784
:105570001B4B984206D153F8182C42F0F00243F826
:10558000182C7047174B984206D153F82C2C42F434
:10559000706243F82C2C7047134B984206D153F895
:1055A000402C42F4704243F8402C70470F4B984215
:1055B00005D153F8542C42F4702243F8542C704710
:1055C000080002401C00024030000240440002403B
:1055D000580002406C000240800002400804024073
:1055E0001C040240300402404404024058040240BB
:1055F0001F4B10B55A6802F00C02042A03D0082A87
:1056000004D01C4A14E01C4A126811E05A68596818
:10561000C2F38342C90302F1020201D4174906E032
:10562000596811F4003F1449096818BF49084A43F2
:1056300002605968124AC1F30311545C0168E140E9
:1056400041605C68C4F30224145D21FA04F48460B0
:105650005C68C4F3C224145DE140C1605B68C3F3BD
:1056600081331A44137CB1FBF3F1016110BD00BF1B
:105670000010024000127A001400002000093D00D2
:105680003400002010B50446FFF752FC012806D173
:105690001CB1FFF74DFC013CF8E7052010BD002CC4
:1056A00008BF052010BD038A828911EA030092B267
:1056B00003D011420CBF0020012070470A88F0B5CA
:1056C0004B888F880E89CD88002A3AD1048C834A72
:1056D00024F001042404240C0484018B048C89B27A
:1056E00021F0F30141EA0616B6B29042A4B246EAAE
:1056F000070743F0010315D002F50062904211D074
:10570000B0F1804F0ED0A2F5983290420AD002F547
:105710008062904206D002F58062904218BF24F069
:105720000A0401D124F00204234307830384038B7A
:1057300023F00C031B041B0C0383038B9BB21D4340
:1057400044E0042A44D1048C644A24F01004240464
:10575000240C0484018B048C21F440710905090D8B
:1057600041EA063189B241EA07279042A4B2BFB2AA
:1057700012D002F5006290420ED0B0F1804F0BD0F3
:10578000A2F59832904207D002F58062904203D091
:1057900002F58062904207D124F0200444EA03130A
:1057A0009BB243F0100304E024F0A00443F0100384
:1057B000234307830384038B23F440631B041B0CE4
:1057C0000383038B9BB243EA0525ADB20583F0BD8D
:1057D000082A018C3ED121F480710904090C01844E
:1057E000818B3E4A89B221F0F301048C41EA06160E
:1057F000B6B29042A4B246EA070712D002F50062A0
:1058000090420ED0B0F1804F0BD0A2F5983290426A
:1058100007D002F58062904203D002F58062904288
:1058200007D124F4007444EA03239BB243F4807349
:1058300004E024F4206443F48073234387830384C7
:10584000838B23F00C031B041B0C8383838B9BB281
:105850001D4341E021F480510904090C0184828B2D
:10586000048C22F440721205120D42EA072242EA29
:1058700006361A4AA4B29042B6B212D002F50062BD
:1058800090420ED0B0F1804F0BD0A2F598329042EA
:1058900007D002F58062904203D002F58062904208
:1058A00007D124F4005242EA033292B242F4805209
:1058B00005E047F6FF52224043F480531A438683A3
:1058C0000284838B23F440631B041B0C8383838B30
:1058D0009BB243EA0525ADB28583F0BD002C0140A3
:1058E0001FB50123ADF808300023ADF80C30ADF83A
:1058F0000A30094BADF804101B7801A9012B08BF31
:105900000323ADF8062008BFADF80C30FFF7D6FE34
:1059100005B05DF804FB00BFD008002038B5114C7D
:1059200004EB0014A278E36842B90122A270A180BE
:105930001868197B0222BDE83840D1E7A288E180CF
:105940006078891A084A89B202EB40020025A2F861
:105950006A10A57021811868197B2A46FFF7C0FFDD
:10596000A57238BD1C090020BC1000202DE9F843A9
:10597000574B0C460168013AC3F882108188A3F89E
:105980008610072A42D8DFE802F0040A10182229FC
:105990002F35B3F882202280B3F8842013E0B3F8C7
:1059A00084202280B3F8822005E0B3F8822052429E
:1059B0002280B3F88420524205E0B3F8842052429A
:1059C0002280B3F882206280B3F886301DE0B3F8FD
:1059D000822052422280B3F8842012E0B3F884205F
:1059E0002280B3F882200CE0B3F882202280B3F842
:1059F000842005E0B3F8842052422280B3F882204C
:105A000052426280B3F886305B42A380314B1B78F0
:105A1000002B5AD1B4F9000005F082FF8046B4F99A
:105A2000020005F07DFF0746B4F9040005F078FF99
:105A3000294D06462968404605F0C6FFE9688146BB
:105A4000384605F0C1FF0146484605F0B5FEA96994
:105A50008146304605F0B8FF0146484605F0ACFEE9
:105A600009F064F869682080404605F0ADFF2969B7
:105A70008146384605F0A8FF0146484605F09CFEE1
:105A8000E9698146304605F09FFF0146484605F02A
:105A900093FE09F04BF8A9686080404605F094FF3A
:105AA00069698046384605F08FFF0146404605F09B
:105AB00083FE296A0746304605F086FF01463846D0
:105AC00005F07AFE09F032F8A080BDE8F88300BF47
:105AD000BC10002028000020A4060020074B084A24
:105AE0001B7812889A4207D3064A12689078984227
:105AF0008CBF00200120704700207047280500203F
:105B0000840D0020800D002010B5194B93F88820DB
:105B1000511C83F88810174902F00702487816498B
:105B200003EB420331F81010A3F88A100023184643
:105B3000124A9A5A02331044102B80B2F8D1C0088E
:105B400005F0EEFE0E4905F03FFF0E4905F0F0FFAF
:105B50000D4B04461B68187805F0E2FE014620460E
:105B600005F032FF06F01CF9084B187010BD00BF9D
:105B7000BC1000208C0600209C060020461100204E
:105B80003333534000F07F45800D0020280500206E
:105B9000A14B2DE9F04F1B7885B0013B012B00F2A2
:105BA00037819E4B1D78854240F032819C4B1B789B
:105BB000022B00F02D819B4E002333809A4B13F86B
:105BC00005B09A4B83F800B0994B1A7803921AB13A
:105BD000984B33F9150008E0974B1A6802F1004220
:105BE0001A60944A32F91500404205F099FE934933
:105BF00005F09EFF9149044605F0E6FE06F0AAF87E
:105C00008D4F8E49D7F800A01FFA80F85046A6F8AD
:105C1000028005F0D9FE06F09DF8DFF84092B080D2
:105C2000D9F8002000211046029206F061F8002702
:105C3000834B029A002857D01A68204611460292D8
:105C4000019306F07DF8029A019B38B11C607D4BF0
:105C5000C3F800A0734BA3F80680BFE01046394696
:105C600006F06EF8002800F0B980774B1A78984655
:105C7000002A31D12046514605F09CFD4FF07E515F
:105C800006F040F8714C28B16068714905F09CFE3F
:105C900060600FE06F49606805F096FEDFF8D09114
:105CA0008246494606F02EF810B9C4F804A001E077
:105CB000C4F80490012388F80030674B00221B6869
:105CC0005B449A72039A82F00103594A1370634B42
:105CD0001F605B4B1F6081E0614BC9F800401A6890
:105CE000584BFA325A6079E020461146019306F08B
:105CF00009F8019B20B1594A14604A4AA2F806806B
:105D0000D3F80080554B4046D3F80090494605F043
:105D100051FD534B824619684A4B5A688A1A002A29
:105D20000BDA4FF07E5106F00BF8002856D02046D3
:105D3000494606F005F8002850D0424A404611680E
:105D400005F0FEFF414C48B10123206841493380F2
:105D500005F03AFE3E492060A06809E00223504663
:105D60004FF08041338005F0EBFF28B1A06839493E
:105D700005F02AFEA06004E02068354905F024FE05
:105D80002060354B2D492068D3F8008005F01CFEBB
:105D900006F006F808F80B00A06806F001F8039A70
:105DA000D84482F00103224A88F8140013702B4B68
:105DB0001F60234B1F60244B1A780132D2B2032A92
:105DC00001D01A700AE000221A70204B2549586849
:105DD00005F0FAFD05F0E4FF88F80A0015B93388EC
:105DE00064333380124A13780BB11F4B00E01F4B12
:105DF000114A13600F4B33F9150005F091FD0F495F
:105E000005F096FE0C4A0146106805F0D3FC00E050
:105E1000084605B0BDE8F08F52030020A40300201F
:105E2000B40300200019002098010108B5030020E8
:105E3000A503002008030020540300200000204197
:105E4000AC03002058110020A6030020B803002056
:105E50000AD7833FEC51783FB0030020A80300200D
:105E6000D419002000007A440000A0410000A0C125
:105E70006F12833A10B50848FCF732F8074B1C68DC
:105E80002046FBF77EFF18B90A20FBF722FFF7E751
:105E9000034A044BDA6010BD531B0108CC080020F4
:105EA0000400FA0500ED00E008B50748FCF718F813
:105EB000064A002313729363054A137002F028FC0C
:105EC000BDE80840FFF7D6BF5F1B0108581100204E
:105ED0007B21002008B50448FCF702F803F0DAFC47
:105EE000BDE80840FFF7C6BF8B1B01082DE9F04F46
:105EF000002485B0074601919246029380462546CC
:105F0000022DDFF878914FEA450607D1019AB9F9D9
:105F1000040053791B3343435B1148E04C4B39F980
:105F2000151033F9153003EB4101CAF10003994212
:105F300003DB5145B4BF0B4653464649029A31F93B
:105F400006B0915FCBEB030303EB010BFCF78CF97D
:105F500098B1414B58465B5D009305F0E1FC3F4929
:105F600005F0E6FD009B01461846FFF711FE3B4990
:105F700005F02AFD05F0EEFE8346394B1988C80767
:105F800011D4019A39F9060013798A0703F11B032A
:105F900000FB03F34FEA231309D57A7C02FB0BFBCA
:105FA00003EB2B2303E0FB7903FB0BF31B112D4ABF
:105FB00098F80AB0905F042290FBF2F0181A7B5D0B
:105FC000294A43430393294BA158B3F800C0013534
:105FD0000CFB00F3DB120BFB03132549B3F5001F89
:105FE000A8BF4FF400138B42B8BF0B462149A35002
:105FF00062584FEA1C1C6050821A4FF6FF70B0FBCB
:10600000FCFC0CFB02F201F10C0C183154F80CB042
:10601000605892115844104444F80C2098F8142009
:10602000032D02FB00F0039A4FEA202000EBE21060
:10603000114A00EB633344F801B0935308F10108AF
:1060400004F104047FF45CAF05B0BDE8F08F00BF3D
:106050007021002008030020CE0A01080000204122
:10606000500300203C0300207C0E0020440300204D
:106070000000E0FF94110020E4030020C60300208C
:106080002DE9F04F87B005938E4B0492B3F90220AF
:10609000B3F90030002AB8BF5242002BB8BF5B42B0
:1060A00000249A42B8BF1A46019003922646A146A0
:1060B00027460294A0462546DFF83CA2BAF80030F5
:1060C00099075AD0022D58D07E4BDDF810C0F25EF1
:1060D0007D4BF35E03EB4202CCF100039A4203DBFB
:1060E00063469A42B8BF1346784ADDF814C036F9C1
:1060F00002B03CF90620CBEB030303EB020BFCF7E9
:10610000B3F890B1724B584615F8038005F008FCBF
:10611000704905F00DFD01464046FFF739FD6D4918
:1061200005F052FC05F016FE834601996423CA79F6
:1061300002FB0BF292FBF3F2CB7E6FF0040101FB4A
:1061400003F8424505DB03EB83039A42B4BF904654
:106150009846614A42F21071A3585B448B42A8BF33
:106160000B465E498B42B8BF0B46A350019A92F88A
:1061700011B00BFB03F31B130293BAF8003003F0CA
:106180000302012A01D1022D3DD101994D4A11F896
:1061900005C05349B75E895F524A81EAE170A0EBBE
:1061A000E170B0F5206F54F802901DDC022D15D07F
:1061B0005020784390FBFCFC042091FBF0F1C1EBF4
:1061C0000C0CE1444848B9F57A5FA8BF4FF47A59FE
:1061D0008145ACBF42F80490105107E087EAE770B0
:1061E000A0EBE7706428E3DD002111513D4AA1587E
:1061F0007D2291FBF2F9019A2A44927A02FB09F975
:10620000402299FBF2F99A0716D5022D14D0039A71
:10621000DDF80CC0C2F5FA730CFB09F07A43DDF827
:1062200008C003FB082203FB0C034FF4FA7192FB36
:10623000F1F293FBF1F308E0DB0701D5022D02D167
:106240004B463A4601E0029B42462549DFF8ACB096
:10625000715A04200FFA81FC15F80BB09CFBF0FA80
:106260000BFB0AFB6FF04F0A9BFBFAFB93441F4AA0
:1062700036F902A0B152CAEB0C0C9CFBF0F002F113
:10628000080102F1140A54F801C054F80A206050C1
:1062900017496244695C02444A43202192FBF1F2AF
:1062A0009A1A144801359344032D44F80AC026F87D
:1062B00000B004F1040406F102067FF4FDAE07B05D
:1062C000BDE8F08FC60300207021002008030020E5
:1062D000CE0A010800002041E80D0020F0D8FFFFA1
:1062E0003C0300207C0E002080C1FFFFB81100207D
:1062F000AC0E0020E403002050030020A60E002076
:106300002DE9F04F89B007937A4B814618880491A4
:10631000059205F001FB784905F056FB0024039037
:106320004F4625462646022EDFF80CA20BD10499D3
:10633000BAF904004B790A33584305F0F1FA6F4972
:1063400005F0F6FB44E06E4B3AF90520EB5E05994B
:106350001A444B429A4203DB0B469A42B8BF13469B
:10636000684AAA5E9B1A079A505F184405F0D8FA4B
:10637000654905F0DDFB8046FBF776FF28B1634BEE
:106380004146985DFFF704FC8046614B1A88D107AF
:1063900005D54046D9F8441005F016FB18E00499DD
:1063A0003AF905000B7901921433584305F0B8FA15
:1063B000524905F0BDFB019A8346930709D5D9F8E8
:1063C0004810404605F000FB0146584605F0F4F938
:1063D0008346504A505F05F0A3FA4F4AD16805F052
:1063E000F3FA82465146584605F0E4F9396A804688
:1063F00005F0EAFADFF844B106900399404605F04B
:10640000E3FAF96A05F0E0FA54F80B1005F0D4F954
:106410004249804605F076FC38B94046404905F0CF
:106420008FFC20B1DFF8F88001E0DFF8F0804BF856
:106430000480DFF80CB1504654F80B1005F0BAF99F
:1064400044F80BA0034603994FF07E50029305F0E9
:106450006FFB029B0146184605F0B6FA0BF10C03E0
:10646000E2580BF1180B54F80B10824610460192BB
:10647000029305F0A1F9514605F09EF9019A029B9D
:1064800044F80B2044F803A0264905F051FBB96BF2
:1064900005F09AFA2449824605F034FC38B9504692
:1064A000224905F04DFC20B1DFF880A001E0DFF8C3
:1064B00078A00698414605F07FF9514605F07AF933
:1064C00008F034FB1A4BB0F57A7FA8BF4FF47A700E
:1064D0009842B8BF18460136164B032EE85204F115
:1064E000040405F1020507F104077FF41CAF09B0AD
:1064F000BDE8F08F44030020BD37863500004842D8
:10650000702100200803002000002041CE0A01086D
:10651000500300203C0300201C02002000007AC32E
:1065200000007A4300004040000096C300009643FC
:1065300018FCFFFFE4030020C6030020880E0020A3
:10654000D811002010B50446204608F0CBF810F012
:10655000FF0F06D10C4B0D481978BDE8104000F034
:10656000EDBC204608F013F902280CD8064B0A228D
:106570001870074B074C02FB0030074B06301860C1
:10658000FBF774FBE0E710BDE40D0020921B01084F
:10659000282100200F1C0108E00300202DE9F0470E
:1065A000704B86B01A789946DFF8C88192B90123FA
:1065B000D8F80000022189F8003003F097F8D8F8E5
:1065C0000030694A6948C2F8A430FBF789FC684882
:1065D000FBF786FCD8F80000FBF7E2FB002800F090
:1065E000BE80644B604C1868FBF7D5FB0928014658
:1065F00001D03F284FD14FF0000AA56B5E4F5646A1
:106600002DB15E4839682A4608F074F810B9BA46C8
:1066100006B93E465A4B0C379F42F1D3CEB137688C
:10662000DAF800E02B46F85C1EF80310814201D036
:10663000A3630EE05A1C41B92D2B06D8A263234454
:10664000202022441872117203E04C49585413461A
:10665000E9E7A36B0BB1564512D04A48FBF740FC63
:10666000564509D856F80C0BFBF73AFCD8F8000051
:106670000921FBF7A7FBF3E73D48FBF731FC0025B9
:10668000A36B9D42A6D23D4BD8F80000595DFBF7A5
:1066900099FB0135F4E7A36B33B904283BD104F12E
:1066A0000800FFF701FC5AE00C2801D136488CE7BE
:1066B0000A2901D00D2949D13448FBF711FCA36BFD
:1066C000E21800231372227A232A17D00493304B46
:1066D0002A4E009303A8284915220C23039608F09C
:1066E0005AF8054638B1006807F0FCFF0130AB6886
:1066F0003044984702E02748FBF7F2FB1F4800218F
:10670000302207F0AEFF0023A36399F80030002B7E
:106710007FF45DAF23E00C28C8D07F2903D159E76F
:106720002F2B3FF657AFA1F12002D2B25E2A3FF6DF
:1067300051AF13B920293FF44DAF5A1CA263D8F8CA
:1067400000001C442172FBF73DFB43E77F29E7D1A2
:10675000013BA363002223441A720F4838E706B0B6
:10676000BDE8F0877B21002058110020A31B010801
:10677000DB1B0108CC080020940B010860110020ED
:10678000900C0108E01B0108E51B01089523010896
:10679000F31A0008F01B01080C1C010800230F4924
:1067A000DAB2595C272903D00133092BF7D11A46F5
:1067B0000B4B83F82C21002283F82D2183F82E2106
:1067C0004FF4E132C3F83021C3F83421C3F8382143
:1067D000C3F83C21522283F8402170474A1B01082C
:1067E000D81900202DE9F04FD74AD84C85B0106851
:1067F000516802AB03C3DFF88C8300214FF4EF62D2
:10680000204607F02EFF04F50573C8F80030D04B82
:106810000025DFF874A31D7004F25673CAF8003027
:1068200054232370032363710223A36040F24C427C
:106830004FF41673A4F8F030A4F81A21FA2340F2AA
:106840006C72A4F8F230A4F81C212A231922A4F8AF
:10685000EE3084F823214FF4FA7340F27E42A4F81C
:10686000F630A4F8D020202340F23A7284F8F430B5
:10687000A4F8D2206E234FF47A7284F80431A4F87D
:10688000D4202B2340F27E5284F80531A4F8D62080
:10689000212340F2EA52012640F2DC514FF01E0B58
:1068A0004FF0320984F80631A4F8D8204FF4C873A9
:1068B00040F2B45284F8EC60A4F80831A4F818113E
:1068C00084F81FB184F8226184F82561A4F8DA20E5
:1068D000A4F8DE300191A4F8DC90A4F8E090FFF772
:1068E0005DFF40F6AC53A381D8F800300B20A573B0
:1068F0001872142017225872187550201A765A767A
:106900009877552264209A71D8772D224FF0080E7F
:1069100078201A7483F813E05A775873DA75DFF821
:106920006CC28C4A8C484FF00E0E282783F80EB0AC
:1069300083F80FB083F80AE04FF00A0B4FF05A0EBD
:106940001F715F7183F80BE01F7383F82160C3F838
:1069500024C01D709D7683F807905D74DD769D746C
:106960001D7783F815B01A63D86318644FF082401E
:10697000D8624FF07C5098637848C3F828C05864B8
:10698000DFF80CC2764801995A639864C3F84CC08A
:1069900084F856E74FF0410EA4F85E1784F857E7E5
:1069A00084F85A5784F85B5784F8589784F85957F5
:1069B00084F85C579A666B4A0421DA666A4A83F85F
:1069C00058101521D86583F8607083F861701A67D4
:1069D00083F87460A3F85450A3F85650A3F85250AB
:1069E00083F864106148FEF7A7FCD8F800304FF434
:1069F0004872A3F86221C82283F8A7214FF4966257
:106A0000A3F8A82140F2D932A3F8AA2140F6430204
:106A100083F85F7183F86061A3F8AC2183F85D515E
:106A200083F85E5183F8645183F8A6B11A4647464D
:106A300056464FF47F71A2F866114FF4FA61A2F83E
:106A4000681102A840F2DC51A2F86A11415D0135DB
:106A500082F86C11082D4FF0FF0182F86D1102F1E0
:106A60000802E6D1012283F8AE2183F8AF2183F832
:106A7000B021C82183F8B6216422A3F8B211A3F88B
:106A8000B82114214FF4967283F8B411A3F8BA21F7
:106A90001E21282283F8B511A3F8BC210023E21897
:106AA00010330021C02B1161F9D13148002140225F
:106AB00007F0D7FD00232F49E2185958043308681E
:106AC000382BC2F8D401F6D12B480021802207F0E0
:106AD000C8FD2A4B284D03F1300E186859682A4624
:106AE00003C2083373451546F7D1254DFBF74AFD20
:106AF000FBF784FDFBF75EFD3F68284639464FF4FF
:106B0000E07207F0A5FD394605F5E0704FF4E0723C
:106B100007F09EFD336805F563725968186803C273
:106B2000198911801A68C5F896235A68C5F89A23FE
:106B30001B89A5F89E33012384F82434022384F8AA
:106B4000E43505B0BDE8F08FD00A0108D81900205F
:106B5000E40D00209A99193F8FC2753DCDCC4C3D74
:106B60000000A040F6287C3F3D0A773F101C01083A
:106B7000AC1B0020F00101082C1B0020D80A0108E2
:106B8000AC1D002018020020E0030020000020407F
:106B90000000404008B50548FBF7A2F9FFF722FEC8
:106BA00002F078FEBDE80840FFF764B9191C01083F
:106BB0000EB40FB5074906AB0190074A01A803932D
:106BC000FEF7F4FA019B00221A7004B05DF804EBA2
:106BD00003B07047B11800082F1C0108F8B5012157
:106BE0000446FEF760FD01283B4F01D0002616E069
:106BF0004FF6FE732382A68D0025B6B22046795D3E
:106C0000FBF7E6FD354B142202FB0030C36813B1DD
:106C1000007C314698470235082DEFD1E6E7BD5D8F
:106C200095B920460221FEF73EFD012850D14FF6CE
:106C3000FD73238229462046FBF7CAFD274B142209
:106C400002FB0030A18E3EE0042D12D120462946E1
:106C5000FEF729FD01283BD14FF6FB73238229461D
:106C60002046FBF7B5FD1D4B142202FB0030218F9F
:106C700029E0082D12D120462946FEF714FD0128EF
:106C800026D14FF6F773238229462046FBF7A0FD55
:106C9000124B142202FB0030A18F14E00C2D17D1EF
:106CA00020461021FEF7FFFC012811D14FF6EF73AB
:106CB000238229462046FBF78BFD084B142202FB5A
:106CC0000030B4F84010836889B20BB1007C98475B
:106CD0000236082EA3D1F8BD080B0108D806002003
:106CE0002DE9F041067B04460F4600683146904688
:106CF0001D46FBF76DFD0F2808D8194B142202FB27
:106D00000030C0F80880C56006710774237B2268D4
:106D10000C2B1CD8DFE803F0071B1B1B0C1B1B1BD9
:106D2000111B1B1B160093899BB243F002030DE05D
:106D300093899BB243F0040308E093899BB243F02C
:106D4000080303E093899BB243F01003938125B1BC
:106D500093899BB243F001039381BDE8F08100BFAA
:106D6000D80600200D4B10B5DC680122E443C4F3C3
:106D70000224C4F1040402FA04F40178A3F5406388
:106D800024011944E4B281F800430178480901F074
:106D90001F018A4043F8202010BD00BF00ED00E035
:106DA000254B10B55343254A254C12680139B2FBD7
:106DB000F3F20388013AA04289B292B29BB212D098
:106DC00004F50064A0420ED0B0F1804F0BD0A4F5C2
:106DD0009834A04207D004F58064A04203D004F5A3
:106DE0008064A04202D123F070039BB2154CA042F4
:106DF00006D004F58064A0421CBF23F440739BB20C
:106E000003800F4B8185984202850FD003F5006304
:106E100098420BD003F54063984207D003F5806396
:106E2000984203D003F58063984201D10023038682
:106E30000123838210BD00BF40420F008400002068
:106E4000002C014000100040284BF0B51D680022C6
:106E50002748165C1418AB19597801F0040101F0A9
:106E6000FF0371B10132102AF2D10020F0BD1BB135
:106E700003EB83035B00DBB210F8012B303A1344C1
:106E8000DBB2221A022AF2DC002184420AD919B1AB
:106E900001EB81014900C9B210F8012B303A1144CD
:106EA000C9B2F2E72E2E14D1601C00220424067809
:106EB00002EB8202AF197F7852007F0792B203D5AE
:106EC000303A3244013092B2013C14F0FF04EED16A
:106ED00000E00022074806244143642000FB021220
:106EE0000548B2FBF4F200FB0320F0BD9000002047
:106EF000FB0E002040420F008096980030B5002223
:106F000013460D495C5C9CB12E2C04D1013378B141
:106F10001C1800250D550A246243C95CA1F13004F8
:106F2000092C9CBF303A52180E2B03D80133E8E7E6
:106F3000104630BD002030BDFB0E00200FB407B559
:106F40000A4904AB08680A4953F8042B09680193FD
:106F5000FEF72CF9074B1868FAF713FF0028F9D051
:106F600003B05DF804EB04B0704700BF8406002056
:106F700080060020FC1100202DE9F0438DB005466D
:106F800007F0B0FBC0B2002858D104467F4B002167
:106F90001E68142207A807F064FBA500002303A9BC
:106FA00005A80393059377190B7183801A46DFF8C0
:106FB000F8E1B7F802C03EF8138018EA0C0F0CD0C5
:106FC0000EF10A0E0DF1300813F80EE002F1010C7B
:106FD000424402F824EC5FFA8CF20133052BE6D12F
:106FE00000231A46DFF8C4E1B7F802C013F80E8098
:106FF00018EA0C0F0CD00EF1060E0DF1300813F844
:107000000EE002F1010C424402F81CEC5FFA8CF233
:107010000133062BE6D1735D8DE803001A0907A83A
:107020005B4903F00F03FFF7C3FD2146594807AA48
:107030000134FFF783FF202CA8D1A4E0284607F0F5
:10704000A6FB1F28044600F3928028462021E4B2C4
:1070500007F03BFB1F2C01D94F4889E04B4B471CE5
:107060001B68002103EB84042046042207F0F9FA90
:1070700000254A4B07AE304600210A2215F803903E
:107080005FFA85F807F0EDFA0023FA5CF91832B1DF
:107090000A2B04D04A4502D0F2540133F5E74A45A1
:1070A00001F1010768D1B8F1020F0DD0B8F1030F5B
:1070B0000CD0B8F1010F0BD0304607F068FB2378F5
:1070C000C0B243EA00100AE0002219E0002226E0E4
:1070D000304607F05CFB237800F00F001843207067
:1070E00039E00133062B0AD02D4800F11D069E5DC4
:1070F0008E42F6D10344D97D63880B43638001320D
:107100000CA9D3B20B4413F8141C21B30023EBE7F2
:10711000412B1ED0542B08BF04230ED00132D3B212
:107120000DF13008434413F8143CA3B1492B01D1AD
:10713000002302E0572B08D10123194901EB430337
:10714000198963880B436380E8E7462BE0D102236B
:10715000F3E70323F1E70135042D8AD10124FBF77E
:1071600011FAFBF74BFAFBF725FA64B974E70D48FF
:107170002021FFF7E3FE06E020460021042207F06D
:1071800070FA0024EBE70DB0BDE8F083DC050020C9
:107190002F1C01083B1C0108471C01082B0B010890
:1071A000080B0108551C0108100B01081F0B0108F2
:1071B00007B5064B06480093064B074A1968074B6C
:1071C000FFF7BCFE03B05DF804FB00BFA81C01087C
:1071D000771C010888000020931C01089F1C0108EF
:1071E00010B50748FAF77CFE0024064B0648E21863
:1071F000E15852680C34FFF7A1FEFC2CF5D110BD0C
:10720000B01C0108940B0108C61C01087FB5044698
:1072100007F068FA082824D100231F49E25C0968B6
:107220001144497801F00301022908BF203AE254D1
:107230000133082BF1D10025665D1848314607F06F
:1072400044FA28B101356019314607F03EFA18B109
:107250001348FAF745FE1CE0082DEDD12046FEF755
:107260006BF81048FAF73CFE00230F4A04A91A44B1
:1072700092F80E210A440949595C0133082B02F89F
:107280000C1CF2D10023094801A98DF80C30FFF73E
:1072900055FE04B070BD00BF90000020902501088D
:1072A000CE1C0108EE1C0108D8190020C91C0108D9
:1072B0002DE9F04389B0044607F014FAC6B2002E57
:1072C0006CD18B48FAF70CFE8A4C2069002104F03F
:1072D0000FFD40BB013688483146FFF72FFE20697D
:1072E00004A9FEF76DF801468448FFF727FE6069A0
:1072F00004A9FEF765F801468048FFF71FFEA06964
:1073000004A9FEF75DF801467C48FFF717FEE06927
:1073100004A9FEF755F801467948FFF70FFE0C2E39
:1073200004F11004D1D10025764C2F462B464FF0A6
:107330000008B04504F1100415DA184654F8101C82
:1073400004F03AFA54F80C1C8146284604F034FA4A
:1073500054F8081C0546384604F02EFA08F10108D6
:107360004B460746E5E76848019302950397FAF70D
:10737000B7FD002401ABE058644920F0004004F060
:10738000DFFC634B634A0434002814BF10461846E0
:10739000FAF7A6FD0C2CEDD15F4891E020465F493D
:1073A000052207F0A7F938B9524B002203441030E8
:1073B000C0281A61F8D197E020465949042207F005
:1073C00099F906462046002E40D1202107F07DF98C
:1073D000002800F08980451C284607F083F93446D0
:1073E0008046504B53F824600EB94F4868E0284659
:1073F00031465FFA88F207F07DF9671C20BB3D4BF0
:107400000021C2181030C02811619C46F7D1474BAB
:10741000002403EBC702D2F804E09846BEF1000F47
:1074200004D143483146FFF789FD55E018F837305D
:107430009C42F6DA23010CEB0305103573440FCBA5
:10744000013485E80F00F1E73C46CAE707F09FF9F1
:10745000461E0B2E074643DC2046202107F035F957
:10746000054640B1451C2846FAF710FF214B3F0165
:10747000D851012400E004462846202107F025F9D0
:10748000054640B1451C2846FAF700FF194B013468
:1074900003EB061358612846202107F016F905462C
:1074A00040B1451C2846FAF7F1FE124B013403EBBC
:1074B000061398612846202107F007F918B91D48DE
:1074C000FAF70EFD10E00130FAF7E0FE094B032C4D
:1074D00003EB0616F061F2D11748FFF7E9FE03E06F
:1074E00016480C21FFF72AFD09B0BDE8F08300BF64
:1074F0000B1D0108D8190020361D01083C1D01088C
:10750000C91C0108EC190020401D01080AD7233CC2
:10751000071D0108031D0108952301084F1D0108DF
:10752000551D0108800D01085A1D01083C02010883
:107530006F1D01087F1D01080F1C0108B91D0108FE
:10754000F8B5074607F0CEF8044638B9194B1A4883
:107550005A791A4B013A53F8221028E03846184954
:10756000224607F0C7F860B91648FAF7B9FC164C7E
:1075700054F8041F19B11548FFF7E0FCF8E7144868
:1075800005E000250D4B53F8256026B91148BDE8EC
:10759000F840FAF7A5BC38463146224607F0AAF86B
:1075A00001350028EED1034B0B485D713146BDE833
:1075B000F840C3E4D8190020E11D0108800D01083E
:1075C00009210108F51D01087C0D0108081E0108AC
:1075D000952301085A1D01080C1E010870B50446C8
:1075E00007F080F808B91E482EE020461D4907F034
:1075F000F3F800242646254678B12CB1012C06D19B
:1076000007F0C5F8064602E007F0C1F8054615493F
:107610000020013407F0E0F8EEE70B2D04D9BDE8B7
:10762000704011480C2189E4012C07DC0F4B2946DE
:1076300033F915200E48BDE870407FE4A6F57A7353
:10764000B3F57A7F03D90B48BDE8704076E40A4869
:1076500029463246FFF772FC044B23F8156070BDD3
:107660001E1E0108DE1B0108581E0108F40400203C
:107670007E1E0108961E0108B81E01082DE9F74379
:10768000044607F02FF8C0B290B9314C054694F883
:10769000D711B4F8D42194F8D6312E480091294658
:1076A0000135FFF74BFC102D04F10404EFD14BE042
:1076B000204607F06CF80F28054636DC20462021CE
:1076C00007F003F8244FEDB2D7F80090441CAD004A
:1076D0000026204607F05BF85FFA86F8B8F1010F44
:1076E00083B208D0B8F1020F0BD0B3F5B47F1ED22D
:1076F0003A6853530AE0FF2B19D83B682B44987023
:1077000004E0FF2B13D83B682B44D87020462C2173
:1077100006F0DBFF044608B1441C02E0B8F1020F9A
:1077200005D10136032ED4D10EE00C4806E009EB5A
:1077300005000021042206F094FF0948102103B03F
:10774000BDE8F043FFF7FABB03B0BDE8F08300BF2C
:10775000D8190020D11E0108480A0020E51E0108A2
:10776000471C01082DE9F0418CB01E469DF84830B9
:107770008846012B1746974B06D198425DD10422CB
:10778000A3F530531A6101E0984256D19248934BC9
:1077900087600360924BB507436103F1C0038361C7
:1077A0004FF0C003C36003618A4B036503F1040318
:1077B0008364C36403F5484303F154030363A3F1F3
:1077C0001403D3F8D42F436342F48042C3F8D42F78
:1077D000D3F8D02F42F00102C3F8D02F4FF00203AC
:1077E0008DF803304FF40073ADF800304FF01803FC
:1077F0008DF8023003D57B486946FBF741F84FF41A
:107800008063ADF80030F4074FF048038DF8023084
:1078100003D574486946FBF733F80E238DF804301E
:107820000022012301A88DF805308DF806208DF87F
:107830000730694CFFF796FA4DE06B4B984240F0E9
:10784000C5806A4C654BA7602360694B2065636106
:10785000C033A361C023E3602361664BB007A36418
:10786000E36403F5E33303F5FE73DA6942F480223F
:10787000DA619A6942F008029A614FF002038DF8CA
:1078800003304FF48063ADF800304FF018038DF8EB
:10789000023003D558486946FAF7F2FF4FF4006307
:1078A000ADF80030F1074FF048038DF8023003D5F2
:1078B00051486946FAF7E4FF27238DF80430002287
:1078C000012301A88DF805308DF806208DF80730CA
:1078D000FFF748FA454C0025012384F8443025621F
:1078E000E561A5626562C4F82C806671A760A57128
:1078F000204601F0BBFAF20731D5206B002826D0D4
:10790000E36C039501934FF480530A93802306930D
:10791000E36805950493202309936369079502930F
:1079200008950B95FDF7EDFD01A9206BFDF7CBFD4B
:10793000236B1A6842F001021A60226D918A89B2A3
:1079400041F0400191825B689BB2236407E0236DA4
:107950004FF6DF721A80DA6842F02002DA60B3076D
:107960002CD5606B28B3A36C002501934FF4805392
:107970000A938023069323690295049310230393AB
:1079800005950795089509950B95FDF7BAFD606B70
:1079900001A9FDF798FD636B1A6842F002021A60B4
:1079A0005D605D60236D9A8A92B242F080029A8295
:1079B00004E0236DDA6842F08002DA60236D20462D
:1079C0009A8992B242F400529A8100E000200CB0F1
:1079D000BDE8F081003801407C190020300B01081F
:1079E0000012002000080140004800402819002033
:1079F0008013002004480040000C01402DE9F047AE
:107A0000054606F06FFE304B0446D3F808809A46D0
:107A100090B92E48FAF764FA2D4B53F8241049B167
:107A20000123A34013EA080F02D02A48FFF786FA81
:107A30000134F1E7284821E028462849224606F08B
:107A400059FE58B92648FAF74BFA264C54F8041F49
:107A50000029EFD01F48FFF771FAF7E72B780026CF
:107A60002D2B03BF013504F1FF344FF001094FF016
:107A70000009174B53F8267027B91B48BDE8F0479B
:107A8000FAF72EBA28463946224606F033FEC8B920
:107A90000120B040830501D51448EFE7B9F1000F8C
:107AA00003D0FAF720FD124804E040EA0800CAF8C3
:107AB00008001048FAF714FA39460F48BDE8F047B5
:107AC000FFF73CBA0136D4E7D81900200E1F010891
:107AD000480B0108081E0108952301080921010827
:107AE000211F0108440B0108361F01084D1F010822
:107AF000611F01086B1F0108C91C01082DE9F04F27
:107B000087B09A468046894616469DF8404000F068
:107B1000ABFA02AF0546034600F1100E186859682B
:107B20003A4603C2083373451746F7D12B7B0BB98E
:107B300003960496404602A901F030FD054640B187
:107B40004368586830B1404602A92A4600F094FDC7
:107B5000F4E72CE0AB6895F800B01F78022F08D14D
:107B600014480094494632465346FFF7FBFD04464D
:107B70000AE0032F17D149462346324601F0CAFDD9
:107B800051460446FAF7F8F85CB10B4B277103EB4A
:107B90008B03C3F800436B6820465C60414601F0EC
:107BA000A5FD204603E017B900940448DAE707B0C2
:107BB000BDE8F08F0048004000120020003801406E
:107BC000874B2DE9F7431B78002B00F00581FAF76E
:107BD000BDFC844E05463378834200F0FD80824C24
:107BE00023681B78002800F0B18063BB0420F9F7FC
:107BF000BFFF7E4F01463860DFF8FC8190B14379CA
:107C00004FF4165188F80C338368C8F81033FAF72C
:107C1000BDF838680221FAF7AFF83868042101F09E
:107C200065FD10E0724B04201B684FF416529B78E0
:107C300000930223FFF762FF4379386088F80C3322
:107C40008368C8F8103323681F78012F33D10420CC
:107C5000F9F78EFFDFF8AC810146C8F80000DFF8C5
:107C60009891A0B143794FF4964189F81433836811
:107C7000C9F81833FAF78AF8D8F800003946FAF745
:107C80007BF8D8F80000042101F030FD13E00090EB
:107C90003B4604204FF49642FFF730FF4379C8F883
:107CA000000089F814338368C9F818330379032B6B
:107CB00004BF504B1F7023681F78022F40F0838051
:107CC0000420F9F755FF4C4C0146C4F81C03A0B141
:107CD00043794FF4964184F820338368C4F8243301
:107CE000FAF754F8D4F81C033946FAF745F8D4F8F3
:107CF0001C03042101F0FAFC0EE000903B46042036
:107D00004FF49642FFF7FAFE4379C4F81C0384F857
:107D100020338368C4F82433D4F81C73374C94F8A8
:107D20004A30022B04D094F89620022A4DD14C34CC
:107D3000334B1C60002C46D0204600214C2206F01C
:107D400090FC0223276084F84A303CE083B9274F37
:107D5000DFF8A480386898F80C13FAF70DF8386843
:107D6000D8F81013FAF712F838680421F9F7EBFE87
:107D700023681B78012B10D1224FDFF87C803868F4
:107D800098F81413F9F7F8FF3868D8F81813F9F7CA
:107D9000FDFF38680421F9F7D6FE23681B78022B13
:107DA00011D1154CD4F81C0394F82013F9F7E4FF13
:107DB000D4F81C03D4F82413F9F7E8FFD4F81C0313
:107DC0000421F9F7C0FE357006E0002BB0D04C342A
:107DD000002A18BF0024ABE703B0BDE8F08300BF62
:107DE00010050020110500201405002018050020B2
:107DF000240500207906002000120020340800200D
:107E0000BC050020A8050020F7B5254B1B78042BE6
:107E10003FD12020F9F7ACFE044670B12046F9F7B7
:107E2000B0FF18B90A20F9F754FFF7E71D4B2046B9
:107E30001B681969F9F7AAFF0AE01A4B21461B686B
:107E400000901A6920200323FFF758FE044600B370
:107E5000154B08221A61154D2868F9F7A1FF50B19A
:107E6000114E082777612868F9F795FF01462046EB
:107E7000F9F7A8FF37612046F9F792FF0028EAD00A
:107E800020462D68F9F787FF01462846F9F79AFF43
:107E9000E1E7074803B0BDE8F040FAF721B800BFBA
:107EA000240A0020200A0020000C0140440A00207F
:107EB000741F010837B5254C254DA369284643F4A6
:107EC0008053A361E36801A943F48053E36018235E
:107ED0008DF80630A023ADF8043003238DF8073069
:107EE000FAF7CEFC4023ADF8043004230DEB030178
:107EF00028468DF80630FAF7C3FC1023284601A95E
:107F0000ADF804308DF80630FAF7BAFCE36843F4B4
:107F10008053E360E36823F48053E3600D4B1A88D9
:107F200002F4415242F4457242F003021A809A8BE5
:107F300022F400621204120C9A8307221A821A8811
:107F400092B242F040021A8003B030BD00100240ED
:107F5000000801400030014008B540F2E9330D4A05
:107F60001189890709D5908140F2E933094A1189BD
:107F7000C9070AD59089C0B208BD013B9BB2002B4E
:107F8000EDD1FAF7B6FCFF2008BD013B9BB2002BF8
:107F9000ECD1F6E700300140224B70B519684FF480
:107FA0007A73B1FBF3F1204B20481A78204B214D16
:107FB0001B78FEF7C3FF204B20481968204B2E6822
:107FC000B1FBF3F1FEF7BAFF00241E4BE2B253F807
:107FD000221049B1012303FA02F2324202D01A48B8
:107FE000FEF7ACFF0134F0E72A6892070DD5174A77
:107FF0001748127803EB8203196AFEF79FFF154BAF
:10800000197A11B11448FEF799FF1448F9F768FF7F
:10801000BDE87040124B1348198800224FF4EF63FB
:10802000FEF78CBFD4190020280500203922010852
:1080300080000020880200208400002077220108B0
:1080400040420F00900C0108081E01087D2100200D
:10805000952201088C0200209F2201089523010827
:1080600044030020A322010830B5002205462E4912
:1080700010014318415CA94204D00132062AF6D10E
:10808000002030BD294C042D0FCB84E80F0023467F
:1080900018D007D8012D0CD0022D43D1244B1B68DA
:1080A0009B680DE0102D37D0202D06D0082D39D13A
:1080B0001CE01F4B1B685B6831E01D4B1B681B6994
:1080C00063602CE01B4A126812783AB1012A08D08A
:1080D000022A0CBF4FF49642002204E04FF41652DD
:1080E00001E04FF496425A609A601BE0124A12680F
:1080F000127A042A16D8DFE802F0080803080800FC
:108100000E4A6260A260032204E04FF4E132626032
:10811000A26001225A7305E0054B1B68DB68A3606F
:10812000204630BD014830BDF4020108281500206A
:10813000180800201405002004010020A08601007A
:108140008A2802D08E2809D07047094B1B689B06ED
:108150000DD5084B1B7853B9074A03E0054B1B7834
:108160002BB9064A064B1A60064B2D221A7070472F
:1081700088020020A4050020740500204805002086
:10818000B0050020B90500202DE9F74F9F4F9B4611
:108190003B7C0C4691465A1C05463A7400682246C0
:1081A00049460C265E43FEF7FBFDAB686868ADF8F8
:1081B000043018238DF8063001A902238DF807300A
:1081C000FAF75EFB2B7B143707EB060A2C680C2BA7
:1081D00000F2F280DFE813F00D00F000F000F00094
:1081E0004D00F000F000F0008200F000F000F00020
:1081F000B600238C864823F001031B041B0C238448
:10820000218CA288238B844223F073034FEA03431B
:108210004FEA134389B292B243F0700314D000F5D1
:108220000060844210D000F5406084420CD000F51C
:108230008060844208D000F58060844204D021F040
:10824000020141F0030107E021F00E0122F4407227
:1082500041F0030142F48072A2802383A4F834B079
:108260002184238B23F008031B041B0C43F0080319
:1082700032E0238C664823F010031B041B0C23847C
:10828000218CA288238B844223F4E6434FEA0343E4
:108290004FEA134389B292B243F4E04308D000F5A9
:1082A0000060844204D021F0200141F0300107E059
:1082B00021F0E00122F4406241F0300142F480629A
:1082C000A2802383A4F838B02184238B23F4006395
:1082D0001B041B0C43F4006323836DE0238C4C4888
:1082E00023F480731B041B0C2384218CA288A38B92
:1082F000844223F073034FEA03434FEA134389B2E6
:1083000092B243F0700308D000F50060844204D0BC
:1083100021F4007141F4407107E021F4606122F41E
:10832000405241F4407142F48052A280A383A4F8E9
:108330003CB02184A38B23F008031B041B0C43F0E7
:10834000080338E0B4F820C0314A2CF4805C4FEACE
:108350000C4C4FEA1C4CA4F820C0B4F820C0A388F1
:10836000B4F81C802CF4005C28F4E6484FEA084876
:108370004FEA0C4C4FEA18484FEA1C4C94429BB20F
:1083800048F4E0484CF4405C03D002F500629442AB
:1083900003D123F4804343F48043A380A4F81C80DA
:1083A000A4F840B0A4F820C0A38B23F400631B04FE
:1083B0001B0C43F40063A383AB7B43B1B4F844309C
:1083C0006FEA43436FEA53439BB2A4F844302388D7
:1083D0009BB243F0010323802B7B0C2B10D8DFE8EA
:1083E00003F0070F0F0F090F0F0F0B0F0F0F0D00EB
:1083F000343404E0383402E03C3400E04034BC5112
:108400005046AAF8049003B0BDE8F08F281500206C
:10841000002C014070B5054C10250E466561FFF734
:108420009BFD3046FFF798FD256170BD00080140B7
:1084300008B5284B80211A886B2022F040021204D4
:10844000120C1A801A8822F038021204120C42F020
:1084500030021A801A8892B242F040021A80FFF766
:10846000D9FF9620F9F735FC03216820FFF7D2FFEA
:108470009620F9F72EFC03216B20FFF7CBFF01209C
:10848000F9F71CFC10216A20FFF7C4FF0120F9F75F
:1084900015FC00216C20FFF7BDFF0120F9F70EFC51
:1084A00000211920FFF7B6FF0120F9F707FC102182
:1084B0001C20FFF7AFFF0120F9F700FC1B2018215B
:1084C000FFF7A8FF0120F9F7F9FB034B01221A700F
:1084D00008BD00BF00300140CA06002070B5184E2C
:1084E0001023736140F080000C461546FFF734FD01
:1084F000144B9B894FF47A737DB1124A1189880716
:1085000006D5FF2191810F4A1189C90711D509E0CC
:108510005A1E92B223B9FAF7ECF91023336170BDF9
:108520001346EAE7928992B20CB122700134013D00
:10853000E2E75A1E92B2002BEDD01346E3E700BFEC
:108540000008014000300140434A2DE9F84F91688E
:1085500040F201130B4040F201118B4293460CD1C3
:108560003E4B93F8A42093F8A59083F8A520B9EB8F
:10857000020918BF4FF0010901E04FF001094FF067
:108580000008374B5FFA88F41B78A34261D9354B5A
:10859000354E1B68354F23B93B685B8926F814308C
:1085A00054E03A68072C94BF12F804A0A2462C4865
:1085B00051469847DBF808300546DB0509D5B9F187
:1085C000000F06D02A4B50461B6829461B68DB6902
:1085D0009847A5F2EE2240F2DC5392B29A4288BF4D
:1085E0003B68DBF8082088BF5D8942F20103134035
:1085F00053B3204B1978194B01F0030202EB8402AC
:1086000093F8060103EB4202A2F8A6501A4620B9DD
:10861000032919D9012183F8061102EBC403B3F829
:10862000A810B3F8A65002EB44020D44B3F8AA1008
:10863000B3F8AC300D441D44ADB2A2F80851042388
:108640002DB295FBF3F5ADB226F8145008F10108F0
:1086500097E7BDE8F88F00BFD81900202815002043
:10866000070A0020100A0020CA040020040100208C
:10867000080200208C0D00202DE9F043214C137CD2
:10868000A468814604F0400C022B38D80C255D43C9
:108690001D4C01332E19377A19EA070F2DD02D5DA5
:1086A0003DB1022D04D0032D14BF0325022500E0A7
:1086B0000125DFF858802F0108EB0704BCF1000FFB
:1086C00004D118F80770033F012F16D94F7B27B14B
:1086D00094F80C8017EA080F0FD048686768B84212
:1086E0000BD38868A768B84207D8157094605660A5
:1086F000D16013741046BDE8F083DBB2C4E70020FC
:10870000BDE8F083D819002048000020DC0C0108E7
:10871000094B30B59D68094B05F480551868084B26
:108720001C6800230DB1828800E0A28805495A52D6
:108730000233182BF6D130BDD8190020F0040020E8
:10874000B4040020F404002070B50E462021154624
:1087500005F0BBFF0446B8B1441C204606F017F8EC
:10876000B0F5617F05DB40F634039842A8BF184698
:1087700001E04FF461701923A0F5617090FBF3F0F4
:1087800030702B7801332B702046202105F09DFF9F
:108790000446B8B1441C204605F0F9FFB0F5617FEE
:1087A00005DB40F634039842A8BF184601E04FF4B9
:1087B00061701923A0F5617090FBF3F070702B7855
:1087C00001332B70204670BD70B586B0054605F0AC
:1087D00089FFC0B208BB044606236343444A03F53D
:1087E0008873126819201344591D4D789A7A4543AD
:1087F00005F561755B7900958D78684300F56170CA
:108800000190C878029009793A48039121460134D1
:10881000FEF794FB0C2CDFD168E0284605F0B7FF8B
:108820000B285FDC06267043314B00F588701E680C
:10883000202106440023681C8DF8173005F045FF01
:10884000741D054658B1451C284605F0A0FF0328B5
:1088500005D89DF81730607101338DF81730284620
:10886000202105F032FF054658B1451C284605F089
:108870008EFF0D2805D870719DF8173001338DF8E3
:1088800017302846611C0DF11702FFF75DFF20210C
:1088900005F01BFF054658B1451C284605F077FF3B
:1088A0000C2805D89DF81730E07001338DF817308B
:1088B0002846202105F009FF50B1013005F067FF7F
:1088C0000D2805D89DF81730207101338DF8173029
:1088D0009DF81730062B09D020460021062205F00E
:1088E000C0FE03E004480C21FEF728FB06B070BD73
:1088F000180200202F230108611C0108F0B585B083
:10890000074605F0EFFEC0B2E0B90446324B04F171
:108910001C021B68192003EB8203591D8D785A79BC
:10892000454305F561759B790095C978484300F585
:1089300061700190214629480134FEF7FFFA282C86
:10894000E4D146E0384605F022FF27283DDC224BE3
:1089500000F11C061B68781C03EB8606202100230F
:108960008DF80F3005F0B1FE751D044658B1441C5A
:10897000204605F00CFF152805D870719DF80F30C2
:1089800001338DF80F302046202105F09EFE04466D
:1089900058B1441C204605F0FAFE0D2805D89DF874
:1089A0000F30687001338DF80F302046A91C0DF18F
:1089B0000F02FFF7C9FE9DF80F30042B09D028469F
:1089C0000021042205F04DFE03E005482821FEF7B2
:1089D000B5FA05B0F0BD00BF180200204F23010812
:1089E000611C010837B582880446836810060D466D
:1089F00006D529494FF4E07091F8541700FB013374
:108A0000D10504D525490A20097800FB013302F07D
:108A10003F02042A12D006D8012A0DD0022A2FD1F3
:108A200093F900102DE0102A0AD0202A0AD0082A33
:108A300026D1B3F9001024E0197822E0198820E04B
:108A400019681EE069461868FCF7BAFC014614482C
:108A5000FEF774FAF5B1E06802F062FF6946FCF7D0
:108A6000AFFC01460F48FEF769FA206902F058FF93
:108A70006946FCF7A5FC01460A48FEF75FFA09E0E3
:108A800000210948FEF75AFA25B10848E168226931
:108A9000FEF754FA03B030BDD8190020E40D0020D1
:108AA0009C2201089B220108682301086423010815
:108AB0002DE9F041002407462546104B3946E6587B
:108AC00004EB0308304605F049FE58B10C48314626
:108AD000FEF734FA40460021FFF784FF0948FEF70D
:108AE0002DFA01351434B4F52F6FE6D125B90648B7
:108AF000BDE8F041F9F7F4B9BDE8F081DC0D0108FB
:108B0000C7230108952301086B2301082DE9F74FBE
:108B1000044605F0E7FD054620B1012818D1237869
:108B20002A2B15D15548F9F7DBF90024544B554849
:108B3000E618E158FEF702FA30462946FFF752FFE1
:108B400014345148F9F7CCF9B4F52F6FEED192E017
:108B500020463D2105F0B9FD002800F0878003463E
:108B600013F8012C202A01D1013BF9E7451C2846C6
:108B7000C4EB030A05F00BFE83462846F9F786FB93
:108B80000026054614237343DFF8F49053F8097068
:108B900003EB0908384605F0A5FD03461A462046B2
:108BA0003946019305F0A6FD019B002855D15FFAD7
:108BB0008AF29A4251D1D8F80C0002F0B1FE014677
:108BC000284603F0B3F8002845D0D8F8100002F08A
:108BD000A7FE0146284603F09FF800283BD0B8F8CE
:108BE00004309B064FF0140303FB0696B28858BF6F
:108BF0005D4614062946B36806D524484FF4E07450
:108C000090F8540704FB0033D00504D520480A240B
:108C1000007804FB003302F03F02042A0BD004D892
:108C2000013A012A0CD819700AE0102A05D0202A2E
:108C300005D0082A04D1198002E0196000E01D6007
:108C400039461448FEF77AF93046002103B0BDE8F2
:108C5000F04FFFF7C7BE104803E001368C2E91D1CC
:108C60000E4803B0BDE8F04FF9F73AB9204603B01B
:108C7000BDE8F04F1CE703B0BDE8F08F8323010887
:108C8000DC0D0108C723010895230108D81900202D
:108C9000E40D002098230108A32301086B23010899
:108CA000104B043033F91030B3F5617F05DB40F62B
:108CB00033029342A8BF134601E04FF46173087872
:108CC0001922504300F28330984208DA4878504322
:108CD00000F283309842B4BF00200120704700208A
:108CE000704700BFCA04002038B5114B114D1A78E7
:108CF000114C29688AB122680244914217D300209E
:108D00001870F8F7F0FF2B6823600C4B1A780AB143
:108D1000013A1A700123237138BD2268C83291428A
:108D200005D301201870F8F7DEFF2B68236038BDEB
:108D3000E30E0020D419002048160020CE020020A7
:108D400037B5214D8DF807306B798DF8062002AAD2
:108D50008DF804008DF805101A4412F8042C443ADA
:108D6000D2B20F2A29D81949022B31F8124003D860
:108D700014B12046FFF7B8FF6B79134A022B09D9CB
:108D8000134B19681368091B8B4203D200235371DC
:108D9000104A13702B79012B00D09CB96B79022BF0
:108DA00002D8094A013353710B4B00202871187007
:108DB00003B0BDE83040F8F796BF022B4FF0C8046F
:108DC000D7D9D9E703B030BD481600200C0D0108F3
:108DD000D4190020CE020020E30E00200449054BE8
:108DE0000968002218701A6159611A76704700BF2D
:108DF000D4190020240A002013B504460068FDF7AA
:108E0000CFFF236801A81A8892B242F001021A80AB
:108E1000637B00228DF8043001238DF805308DF836
:108E200006208DF80730FDF79DFF02B010BD70B52C
:108E3000064600240A4BE518AA8816420AD0E158D3
:108E40000848FEF77BF828460021FFF7CBFD0648CF
:108E5000F9F746F81434B4F52F6FEBD170BD00BFAD
:108E6000DC0D0108C323010895230108F0B5046D4A
:108E70004679A389054623F400531B041B0CA381E8
:108E800006F00403876887B003F0FF0023B14FF4B6
:108E900080604FF4005300E0034616F0010F14BF4A
:108EA00004220022B107218A48BF42F0080289B299
:108EB00021F4405143EA01032382A38948BF92B2BF
:108EC0009BB223F4B05323F00C0318430243A28156
:108ED000A38A01A823F440731B041B0CA382FCF794
:108EE00087FB1949049A039B8C4208BF1346A28949
:108EF0001921594312B2002AB4BF7F00BF00B1FB51
:108F0000F7F16423B1FBF3F21201100903FB101116
:108F1000A08900B2002806DAC9003231B1FBF3F3B0
:108F200003F0070305E009013231B1FBF3F303F06D
:108F30000F031A4392B22B6D22819A8992B242F4A6
:108F400000529A8107B0F0BD0038014041718DE7B1
:108F500081608BE72DE9F04F624CA3686249581C91
:108F60000A78894602F0FF0C0AB10346F6E7277C2F
:108F7000667CA57C6169A360E0461FFA88F213B2A3
:108F80001F2B00F39380594901EB8300C27880784E
:108F900031F82310C0F1FF0080B2002861D0C0F189
:108FA000FF0050433C23B1FBF3FA0012BAF1050F66
:108FB0005AD8DFE80AF0030B1A283846161A4E432F
:108FC000C5B2B6FBF3F62E44F6B248E0B1FBF3F7B8
:108FD00003FB1717BFB2C5B2C7F13C07101A4743CE
:108FE000B7FBF3F72F44164629E0B1FBF3F503FB7B
:108FF0001515C7B2ADB2101A4543B5FBF3F53D44A4
:10900000EDB2164630E0B1FBF3F603FB1616B6B22E
:10901000C7B2C6F13C06101A4643B6FBF3F63E440F
:109020001546F6B220E0B1FBF3F703FB1717C6B203
:10903000BFB2101A4743B7FBF3F737441546FFB2E8
:1090400012E0B1FBF3F503FB1515ADB2C6B2C5F1E5
:109050003C05101A4543B5FBF3F53544EDB2174610
:1090600002E01546164617464FEA072A4AEA064A1C
:109070004AEA050A1723012199400CF1170211EA67
:109080000A0FC3EB02021A490CBF0920112092B249
:1090900013F1FF338854EED20CF1180C08F10108DB
:1090A0001FFA8CFC1FFA88F8124966E7012389F839
:1090B0000030114BE28140F22A3227746674A574A5
:1090C0006161A4F80CC05A600C4A00219184118897
:1090D00089B241F0010111801A6842F001021A6060
:1090E000BDE8F08F481600207A210020E00500201E
:1090F0004C0A0020581600206C000240000400407A
:109100004B8810B5DC0607D52C4B14791B6853F837
:1091100024402B4B43F820404B889B0607D5274B18
:1091200054791B6853F82440254B43F820404B8862
:109130001C070DD5234B0C781B78B3EB141F07DBF2
:109140001E4BD4781B6853F824401D4B43F8204035
:109150004B889B070DD51C4B0C781B78B3EB141F69
:1091600007DC164B54781B6853F82440144B43F823
:1091700020404B88DC070ED5144B0C781B7804F08C
:109180000F049C4207DC0D4B14781B6853F82440F5
:109190000B4B43F820404B885B070ED50C4B0978EE
:1091A0001B7801F00F01994207DB044B92781B6892
:1091B00053F82220024B43F8202010BD480A00201B
:1091C000E0050020730600207106002070060020D4
:1091D00072060020174B13B51A88044622F040028D
:1091E0001204120C1A801A88432022F0380212044A
:1091F000120C1A801A88694692B242F040021A8014
:109200000622FFF76BF99DF800209DF8013043EA34
:10921000022323809DF802209DF8033043EA0223B5
:1092200063809DF804209DF8053043EA0223A38063
:1092300002B010BD00300140174B13B51A88044628
:1092400022F040021204120C1A801A883B2022F0ED
:1092500038021204120C1A801A88694692B242F03F
:1092600040021A800622FFF739F99DF800209DF888
:10927000013043EA022323809DF802209DF8033049
:1092800043EA022363809DF804209DF8053043EAF9
:109290000223A38002B010BD003001401FB501239E
:1092A000ADF80830ADF80410002301A9ADF80A307C
:1092B000ADF80C30ADF80620FCF700FA05B05DF80B
:1092C00004FB464B10B54FF4127404FB003494F8C1
:1092D0003C22C2B9A36A616A994229D0591CA0698B
:1092E000A162C05C2369C0B299424FEA400343F4D3
:1092F0000073A4F83E324FF00A0384F83D3228BFD1
:10930000A262012312E094F93D327BB1B4F83E121F
:1093100020464B08A4F83E3201F00101F9F787FA24
:1093200094F83D32013B84F83D3201E084F83C3250
:1093300094F83832002B4FD194F839320133DBB234
:10934000092B84F8393204D12046BDE81040F9F7E2
:1093500059BA0A2B40D194F83B322BB9B4F84032B9
:1093600043F00103A4F840326379D9071CD5B4F85F
:109370004002820501D4C30705D4B4F84432013356
:10938000A4F8443210E0E36AC0F347000BB19847F9
:109390000AE0E3696269D054E269E3680132B2FB32
:1093A000F3F103FB1123E361012284F8382294F8DE
:1093B0003B220023012A84F839320DD1A27984F8A6
:1093C0003B32236B012A1868197B14BF022200224A
:1093D000BDE81040FFF762BF10BD00BF601600205F
:1093E0002A4B10B54FF4127404FB00346379DB0789
:1093F0004AD594F8383203B3236B0022186882846C
:1094000094F83C2222B1B4F842220132A4F842225C
:10941000A279197B012A0CBF02220022FFF73EFF2E
:10942000012384F83B32002384F8393284F83A323D
:1094300084F83832A4F8403210BD94F83B3220460C
:10944000012B04BF94F8393284F83A32F9F7DAF98B
:1094500094F83B12236BA27949B9012184F83B129D
:109460008A421868197B0CBF0222002208E0002102
:1094700084F83B12012A1868197B14BF02220022CB
:10948000BDE81040FFF70ABF10BD00BF6016002006
:10949000426A10B58469A154416A02690131B1FB85
:1094A000F2F402FB14124262426B32B11368DB0722
:1094B00008D4BDE81040FBF7EDBF036DDA6842F059
:1094C0008002DA6010BDF7B50368174C174D2360B2
:1094D0000B68174E63600068F9F7FAF895E8030027
:1094E000144B0196009394E80C00F9F7AFF8366836
:1094F000114B60681E606B68104FC01A02F010FAC2
:109500000F4B196802F060FA02F024FC22682B6805
:109510007860D31A3B600B4B1E600B4B1B68DA88DC
:109520000A4B1A8003B0F0BD601000203C050020FB
:109530006C10002068100020A8100020701000207F
:1095400030000020A0100020D40300209C10002038
:10955000114B07B51A88752022F040021204120C34
:109560001A801A880DF1070122F038021204120C39
:1095700042F030021A801A8892B242F040021A80F9
:109580000122FEF7ABFF9DF80700B0F168035842D7
:10959000584103B05DF804FB003001402DE9F04371
:1095A000142285B0814688461B48002105F059F8F1
:1095B00002261A4B0027B74224DA13F8042C0021A4
:1095C000C8B2013112B1501E0240F9E71C7AD1B283
:1095D000013214B1611E0C40F9E7421A002A0EDD77
:1095E00001ACA3F10C0595E8070084E8070093E8B7
:1095F000070085E8070094E8070083E807000137C3
:109600000C33D8E7013ED4D1034A4846414605B061
:10961000BDE8F043FFF730B8A81800205400002040
:1096200008B50420FEF720FD01460420FFF7B6FF31
:1096300018B14368187A00F0010008BD70B52548DC
:10964000037813F0010F03F004023AD0002A40D14E
:1096500003F0020101F0FF06002932D143F00403B8
:1096600003701D4B1A881D4B1A801D4B9B685905B2
:109670002FD50420FEF7F8FC01460420FFF78EFFEB
:1096800043681A7AD20724D55C6814B3154D2B6849
:10969000A34208D120460121F8F755FA2846314661
:1096A0004C2204F0DEFFEB6CA34212D120460121D4
:1096B000F8F749FABDE870400B4800214C2204F04D
:1096C000D0BF32B90220FF210122BDE87040F8F777
:1096D00011BB70BD7C21002018030020C80E0020A3
:1096E000D81900203408002080080020084B5A6850
:1096F00082420AD01A69824206D0DA69824208BFE1
:10970000183302D0002300E00C335972704700BFB9
:10971000480000202DE9F7431F464FF412734343DE
:109720009146404A0646D41820B93F48206310307D
:10973000C4F834013D480025D050032363714FF431
:1097400080734FF00108E3602361D4F8343184F86A
:109750003C5284F8388284F8395284F8466258685A
:1097600004F134029B68626104F59C72A261E162BB
:109770002562E561A5626562A4F84252A4F84452EC
:10978000ADF804300225102301A9C4F80890A77190
:109790008DF806308DF80750F9F772F8236B01A9A0
:1097A00058689B688DF80750ADF8043048238DF851
:1097B0000630F9F765F841462046F9F738F83220C7
:1097C000F8F787FA1A4BD4F834811B681D46B5FBAD
:1097D000F9F1B1F5803F03D3012DF8D96D08F6E713
:1097E000144A4046B3FBF2F289B2D2B2FFF704FB4F
:1097F000404631460023104AFDF772FA256B012FCF
:1098000014BF022200222868297BFFF747FD284663
:1098100031460A4A0023FDF763FA204603B0BDE84B
:10982000F08300BF60160020F01801082C0D01081D
:109830008400002040420F00C3920008E19300081A
:1098400003460A4690F84602D96A9B7962E70F4BB5
:109850001A78542A16D15A88B2F5EF6F12D11A79B4
:10986000BE2A0FD193F874270020EF2A0CD113F8E9
:10987000012B5040064A9342F9D1D0F1010038BF84
:109880000020704700207047704700BF00F80108B3
:1098900078FF01084A4B54222DE9F3411A704FF426
:1098A000EF625A80BE221A71EF2283F874270022D9
:1098B00083F8752711461E46B35C0132B2F5EF6F8F
:1098C00081EA0301F8D13E4B3E4A83F875173E4BBF
:1098D00004275A6002F188325A600020013F17F0D5
:1098E000FF075DD0384B3422384CDA60C4F30903EB
:1098F0007BB1331903F17843A3F5FC33D3F800802F
:109900004FF4005000230193FBF7BCFE0428E5D17F
:109910001BE04FF43020FBF7B5FE0428DED12A4DC2
:109920004FF430202B6943F002032B616C612B69EB
:1099300043F040032B61FBF7A5FE2A6941F6FD7356
:10994000134004282B61D4D0C8E71F4D4FF40050BA
:109950002B6943F001032B611FFA88F32380FBF787
:1099600091FE042812D1A31C0193019B4FEA1848D1
:10997000A3F800804FF40050FBF784FE2B6941F6FA
:10998000FE721A4004282A6106D0A7E72B6941F627
:10999000FE721A402A61A1E70D4B04349C42A5D106
:1099A000094B04281A6942F080021A6102D1FFF7BC
:1099B0004EFF10B90A20F8F7C3F902B0BDE8F081F4
:1099C000D8190020230167450020024000F8010853
:1099D00078FF01082DE9F04F692887B0044600F0B0
:1099E000A38200F296802E2800F0378562D82428C2
:1099F00000F007852BD8202800F07E82222800F076
:109A0000B383012840F05A852C20F8F70FFA002084
:109A1000F8F7DDF92046F8F7DAF90020F8F7D7F97A
:109A20004320F8F7D4F94C20F8F7D1F94620F8F79D
:109A3000CEF94C20F8F7CBF92046F8F7C8F900200A
:109A4000F8F7C5F90020F8F7C2F90024F0E028285B
:109A500000F0DF8412D8262840F03085924C032095
:109A6000F8F7E4F9B4F9E600F8F7E3F9B4F9E80037
:109A7000F8F7DFF9B4F9EA0000F029BC2A2800F071
:109A8000D3842C2840F01A85874C0720F8F7CEF9AC
:109A900094F81601F8F79BF9B4F91C01F8F7C9F925
:109AA000B4F91801F8F7C5F9B4F91A01F8F7C1F9D2
:109AB00000F0C0BC642800F0E2801AD8322800F020
:109AC000B9840AD8302840F0F984774C8020F8F720
:109AD000ADF904F1800500F0D6BC342800F06483B1
:109AE000402840F0EB840820F8F7A0F9002400F0AB
:109AF000AABC662800F09881C0F0EE80672800F0CC
:109B0000CC81682840F0DA841020F8F78FF900241F
:109B100002E2732800F0AF8355D86D2800F0178259
:109B200012D86B2800F0D78340F2B0835F4C062038
:109B3000F8F77CF9B4F90000F8F77BF9B4F9020002
:109B4000F8F777F95A4BC0E36F2800F03082C0F085
:109B50000682702800F07682722840F0AF84524C62
:109B60001620F8F763F90020F8F763F9B4F9D0008C
:109B7000F8F75FF94F4DB4F9D200F8F75AF9B4F994
:109B8000D400F8F756F92B68B3F9A801F8F751F9A2
:109B90000020F8F74EF90020F8F76CF92B68B3F9BC
:109BA00052000A2390FBF3F0F8F743F994F804010C
:109BB000F8F70DF994F80601F8F709F994F805019A
:109BC000F8F705F9E3E3782800F0738110D87528D9
:109BD00000F0BE82C0F00983762800F08E837728DB
:109BE00040F06C84344D00242878F8F71FF937E3EF
:109BF000A42800F0CE8310D8A02840F05F840C2069
:109C0000F8F714F92D4B1868F8F734F92C4B18684D
:109C1000F8F730F92B4B1868F8E3F02800F0E483EC
:109C2000FE2840F04B840820F8F700F90024D3E325
:109C3000254B1B68185D0134F8F7C9F8042CF7D1DF
:109C40000020F8F7F6F80024204B185D0134F8F7EF
:109C5000BEF80B2CF8D100241D4B185D0134F8F729
:109C6000B6F8082CF8D10720F8F7B1F80024194B02
:109C7000185D0134F8F7ABF8072CF8D187E307201B
:109C8000094CF8F7D3F8E620F8F7A1F86079F8F76F
:109C90009EF80020F8F79BF894F82431002B0CBFB5
:109CA00004200C20B2E300BFD819002008030020D4
:109CB000180300201802002032080020E8F7FF1FD8
:109CC000ECF7FF1FF0F7FF1F8C000020931C01082A
:109CD0009F1C0108A81C01080B20F8F7A7F8C34B2C
:109CE000B3F90000F8F7A5F80020F8F7A2F8C04B88
:109CF0001B68C3F3C000C3F38002800040EA420047
:109D0000C3F340021043C3F3401240EAC20003F021
:109D100010031843F8F78DF8B64B1A8812F0010FAC
:109D20000CBF0020022012F0020F0CBF0021042102
:109D300012F0040F0CBF0023102312F0400F0CBFD1
:109D400000242024019312F0100FAB4B02940CBF9F
:109D500000244FF4007412F0200F1B6803940CBF12
:109D600000244FF4806412F4807F04940CBF00241C
:109D70004FF4006402F0080B03F4807A059403F4B6
:109D8000805903F4005803F4004C03F4803E03F4BC
:109D9000003703F4802603F4002503F4801403F055
:109DA000C00343EA0B0343EA0A0343EA090343EA15
:109DB000080343EA0C0343EA0E0E904B4EEA0707F2
:109DC0003E431B7835432C43C3F3800323430343B3
:109DD0000B430199029C0B4303992343049C0B43BF
:109DE0000599234312F4007F43EA01030CBF0022CC
:109DF0004FF400121A43824B00201C780346A34202
:109E00000CD280495D5C012101FA05F5154218BFAD
:109E1000994003F1010318BF0843F0E7F8F72AF867
:109E2000794B93F854070BE31220F7F7FFFF774BBA
:109E3000774C1B88B3F5806F22D90025605F08231B
:109E400090FBF3F00235F7F7F4FF062DF6D1714CD5
:109E5000B4F90000F7F7EDFFB4F90200F7F7E9FFF6
:109E6000B4F904006C4CF7F7E4FFB4F90000F7F71D
:109E7000E0FFB4F90200F7F7DCFFB4F9040026E2D2
:109E8000B4F90000F7F7D5FFB4F90200F7F7D1FFF6
:109E9000B4F90400F7F7CDFFD9E71020F7F7C6FFB4
:109EA00000245E4B185D0134F7F791FF102CF8D1B8
:109EB0000FE23820F7F7BAFF0025594E05F12C04C0
:109EC0003368E4002344B3F90600F7F7B2FF3368C0
:109ED00001352344B3F90800F7F7ABFF3368234497
:109EE000B3F90A00F7F7A5FF33681C44207BF7F7A6
:109EF0006EFF082DE1D1ECE10820F7F797FF002471
:109F0000474B1B6803EBC40393F86D010134F7F76B
:109F10005EFF082CF4D1DCE1424B185D0134F7F709
:109F200056FF102CF8D1D4E13F4D00242878400092
:109F300000F0FE00F7F77AFF2B789C4280F0C98191
:109F40003A4B33F91400F7F774FF0134F4E70620B5
:109F5000F7F76CFF0020F7F78DFF0020B7E107202F
:109F6000F7F764FF324B4FF6FF741878F7F72FFFBF
:109F7000304B1868A042A8BF204620EAE07000B22B
:109F8000F7F757FF2C4BB3F90000F7F752FF1E4BC2
:109F900093F80C21294B18680028B8BF40420AB139
:109FA0000A235843A042A8BF204600B28FE1244CA8
:109FB0000720F7F73BFF23681878F7F708FF2368B7
:109FC0005878F7F704FF23681879F7F700FF23683C
:109FD0005879F7F7FCFE23689879F7F7F8FE2368BD
:109FE0009878F7F7F4FE2368D87829E24403002034
:109FF00088020020500300204C0300207C21002018
:10A00000320800201C080020D81900200000002081
:10A01000E80200203C0300207A0600206C000020AB
:10A020001802002052210020070A0020CA04002044
:10A0300028050020300500208E0D00202C05002072
:10A04000E0030020B44D1E20F7F7F0FE2B6800243B
:10A050001B78022B69D12B68B04903EB8403586A43
:10A0600001F0B2FC04F062FDFA28A8BFFA2020EA51
:10A07000E070C0B2F7F7ABFE2B68A94903EB84038D
:10A08000186B01F0A1FC04F051FDFA28A8BFFA20DA
:10A0900020EAE070C0B2F7F79AFE2B68A14903EB03
:10A0A0008403D86B01F090FC04F040FD6428A8BF45
:10A0B000642020EAE070C0B20134F7F788FE032C78
:10A0C000C9D1072C2B681ED1986C944901F07CFCF7
:10A0D00004F02CFDFA28A8BFFA2020EAE070C0B2F4
:10A0E000F7F775FE2B688D49D86C01F06DFC04F014
:10A0F0001DFDFA28A8BFFA2020EAE070C0B2F7F7E9
:10A1000066FE00200BE023441879F7F760FE2B6809
:10A110002344987BF7F75BFE2B682344187E0134B9
:10A12000F7F755FE0A2CCCD1D3E02B6823441879DD
:10A13000F7F74DFE2B682344987BF7F748FE2B6812
:10A140002344187E0134F7F742FE0A2CEDD1C0E01B
:10A150002F20F7F76BFE744C14F8010F002800F065
:10A16000B880F7F734FEF7E7A020F7F75FFE00248A
:10A17000694B04F11C021B680C2103EB82035D1D7B
:10A180006A4A5B79013401FB0323187AF7F71FFE53
:10A190006878F7F71CFEA878F7F719FEE878F7F764
:10A1A00016FE282CE4D194E04820F7F73FFE002566
:10A1B00006266E43584B06F588761B6801351E440B
:10A1C000B07AF7F704FE7079F7F701FEB079F7F788
:10A1D000FEFDF079F7F7FBFD307AF7F7F8FD707ABE
:10A1E000F7F7F5FD0C2DE3D173E0002701240025DE
:10A1F0004F4B1B789D4222DA4E4BE95C00234B4AC1
:10A2000003EB02089A5C8A4204D00C33B3F58A7FD0
:10A21000F5D112E0D8F8040004F064FA81460CB9D4
:10A22000264601E0074408E04E4506DAD8F8043037
:10A23000985DF7F7CCFD0136F6E70135D8E7002C3D
:10A2400047D0F8B2F7F7F2FD0024D0E7374A991863
:10A250009A5C82420BD00C33B3F58A7FF6D101347D
:10A260002B789C4235D2334BE05C0023EEE7087A32
:10A27000F7F7ADFDF3E70820F7F7D8FD0124E0B2CA
:10A280000134F7F7A4FD092CF9D122E01020F7F7EB
:10A29000CDFD294B294C187800F00200F7F797FD07
:10A2A000274B1878F7F793FD2068F7F7E3FD606810
:10A2B000F7F7E0FD234BB3F90000F7F7BAFD224BA7
:10A2C000B3F90000F7F7B5FD204BB3F90000F7F73D
:10A2D000B0FD0120F3E00520F7F7A8FD1C4BB3F912
:10A2E0000000F7F7A6FD1B4BB3F90000F7F7A1FD3F
:10A2F000194B187800F00100A2E0F7F707FC0646BA
:10A300001220F7F793FD0EB9144B02E0102E29D15D
:10A31000134B1D685C6827E01802002000002041F4
:10A320000000C84200007A44430D0108E808010813
:10A33000320800201C080020FE0200203C050020FE
:10A34000380500203605002034050020BC18002008
:10A35000A0050020A2050020EA0E0020F00D00203C
:10A36000FC0D0020002425463046F7F730FD284636
:10A37000F7F780FD2046F7F77DFD524B1868F7F799
:10A3800079FD0020F7F755FD0020F7F752FD00207A
:10A3900056E04D4D0024A8782E4680000130C0B212
:10A3A000F7F744FDA878F7F712FDB3789C4290D2F6
:10A3B000464D285DF7F70BFD05F11003185DF7F723
:10A3C00006FD05F12003185D3035F7F700FD285D27
:10A3D000F7F7FDFC0134E8E73D4B185F0234F7F76F
:10A3E00028FD082CF8D174E73A4C0420F7F71EFD3D
:10A3F0002368B3F95600F7F71CFD2368B3F954003E
:10A4000065E70420F7F712FD334B9868F7F732FD44
:10A410005FE7314C0420F7F709FDB4F90801F7F7BD
:10A4200008FDB4F90A0152E70120F7F7FFFC2A4BB7
:10A43000587905E00120F7F7F9FC274B93F81E0146
:10A44000F7F7C5FC45E7244B234493F80E0101348C
:10A45000F7F7BDFC082CF6D13BE74020F7F7E6FC08
:10A460001D4C04F14005B4F9D401F7F7E2FC94F86F
:10A47000D601F7F7ACFC043494F8D301F7F7A7FC46
:10A48000AC42F0D125E7B4F85601043400F03F00A7
:10A49000F7F7CFFCB4F85201C0F38410F7F7C9FC0A
:10A4A00094F850010009F7F792FC94F8500100F07D
:10A4B0000F00F7F78CFCAC42E5D10AE7002007B0AB
:10A4C000BDE8F08FEC0E0020BC180020BF18002063
:10A4D0000019002018020020D819002000000000F8
:10A4E000044B1A6942F480421A611A6922F48042CC
:10A4F0001A61704700100240254B37B5DA69254CC8
:10A5000042F48042DA611A69204642F480421A61BC
:10A5100018238DF806304FF42043ADF8043001A91C
:10A5200003238DF80730F8F7ABF94FF48043ADF80B
:10A53000043004230DEB030120468DF806304FF460
:10A540008055F8F79DF91023204601A98DF80630B3
:10A55000ADF80450F8F794F92561FFF7C1FF0E4BF1
:10A560001A8802F4415242F4457242F003021A8002
:10A570009A8B22F400621204120C9A8307221A8228
:10A580001A8892B242F040021A8003B030BD00BF78
:10A5900000100240000C0140003800402DE9F0415D
:10A5A000FFF755F910B90A20F7F7CAFB774C4FF4BB
:10A5B000EF622046764904F04BF894F854374FF494
:10A5C000E072022B84BF002384F8543794F8543788
:10A5D000704E02FB034303F5057393F8502033607C
:10A5E000022A84BF002283F8502093F850306A4A30
:10A5F00013700A2202FB0343684A03F25673136086
:10A60000A36842F201021A403AB944F208021A4021
:10A610001AB95E4A43F400539360A368DB0703D57D
:10A620004FF40050F7F75FFFA3685F0409D50820D7
:10A63000F7F759FF4FF40050F7F755FF0120F7F7F0
:10A6400052FFA3681D0706D54FF40050F7F74BFFE4
:10A650000120F7F748FFA36898040ED54FF4004097
:10A66000F7F741FF4FF40060F7F73DFF4FF48030FC
:10A67000F7F739FF4020F7F736FFA368590603D5EF
:10A680004FF48030F7F72FFF454D464BA8461D602D
:10A69000FAF76AFE444B05F11E0201201A60FDF72D
:10A6A000E3FC01460120FEF779FF002840D002209C
:10A6B000FDF7DAFC01460220FEF770FF002837D0D4
:10A6C0001020FDF7D1FC01461020FEF767FFA368BC
:10A6D0001A0600D560B30820FDF7C6FC0146082025
:10A6E000FEF75CFFA3681B0700D508B30420FDF745
:10A6F000BBFC01460420FEF751FFA3685F0503D4AD
:10A7000000231A46194609E00028F9D110E079B96A
:10A710000121C00708D40C33242B0BD02348184444
:10A72000007A8507F5D5F2E70132D2B2022AF2D9D2
:10A73000FCF734F8F7F79AFA1D4F1E4B32681F608A
:10A740001D4B101D186002F175010023CD5C55B939
:10A7500001EB030E9EF802C09EF803E0F44502D21E
:10A76000164B1D7002E00433A02BEFD1144B15499A
:10A770000B60154950330B601178144B012903D03D
:10A78000022929D0124928E0124926E0D8190020D0
:10A7900000F8010818020020E40D0020E00300206A
:10A7A000E61A0020040100201808002048000020BC
:10A7B000A81A0020DC0D0020E00D00202C00002055
:10A7C000CC1A002034020020140500207C00002058
:10A7D00081600008ED5E00083F4919603F4B02F5BB
:10A7E000D9721A60F7F792FF35683D4B05F5D372C1
:10A7F0001A603C4B00229A803B4B3C4A05F5B371F2
:10A8000013603B4AB4F8F00011603A4AA3F1220108
:10A810001160394A05F5D7711760384A2C33116039
:10A82000374A384E1360384B05F5D872C3F80080AC
:10A83000364B1A6001F070F87060B4F8F20001F065
:10A840006BF895F8583005F16002337095F8743064
:10A85000B060737094F82331F76133732C4BB5F803
:10A8600062011E602B1D33612A4B1A6005F16403DF
:10A87000736105F25D13B36101F052F80146264899
:10A8800001F056F900F094FC0FA3D3E9002300F087
:10A89000E3FC00F03BFF214B1860E86D00F088FC02
:10A8A0000BA3D3E9002300F0D7FC0B4602461C495A
:10A8B000002000F0FBFD00F029FF1A4B1860BDE8F6
:10A8C000F08100BFAFF300803B597E90A9E7814043
:10A8D000182D4454FB21094001630008D4030020D3
:10A8E000D0190020F0090020D01A0020A402002076
:10A8F000B0040020F0040020B4040020EC03002089
:10A90000B804002008190020BC040020C404002062
:10A91000D80200203403002000006144D00300204E
:10A920000000E03F2403002008B5FEF7B3FFFFF767
:10A9300035FEBDE808400F2014210122F7F7DAB9EF
:10A9400010B50446204603F0CDFE10F0FF0F07D1EE
:10A950000B4B0C4893F85417BDE81040FCF7EEBAC7
:10A96000204603F014FF022808D8054B064C83F854
:10A970005407FEF78FFFFFF711FEE3E710BD00BF9E
:10A98000D8190020961B01080F1C01082DE9F04F73
:10A99000844985B0054603F06DFE834900282846AA
:10A9A0000CBF0124072403F065FE804900282846D7
:10A9B00008BF022403F05EFE002808BF0424E1075C
:10A9C00040F1BE807A48FCF7B9FA0020FCF7F0FBB2
:10A9D000784F7948FCF7B2FA7848FCF7AFFA7A7901
:10A9E000774B013A774853F82210FCF7A7FA3869F9
:10A9F000002101F07DF900285CD13D460646D5F8DE
:10AA000010800021404601F073F900284ED1013634
:10AA10006D483146D5F814B0D5F818A0D5F81C907B
:10AA2000FCF78CFA4046002101F06CF910B1674840
:10AA3000FCF784FA69464046FAF7C2FC01466448CE
:10AA4000FCF77CFA5846002101F05CF910B15F4830
:10AA5000FCF774FA69465846FAF7B2FC01465C48BE
:10AA6000FCF76CFA5046002101F04CF910B1574840
:10AA7000FCF764FA69465046FAF7A2FC01465448CE
:10AA8000FCF75CFA4846002101F03CF910B14F4850
:10AA9000FCF754FA69464846FAF792FC01464D48DD
:10AAA000FCF74CFA0C2E05F11005A8D14A48711C90
:10AAB000FCF744FA4948FCF741FA494DD7F80880B9
:10AAC00055F8041F19B14748FCF738FAF8E70D4666
:10AAD000454B53F8256056B10123AB4013EA080FEC
:10AAE00003D042483146FCF729FA0135F0E74048E7
:10AAF000FCF724FA31467B1893F80E3104AA13446C
:10AB00003C4A8A5C0131082903F8102CF3D1002358
:10AB1000694639488DF80830FCF710FA3748FCF7D9
:10AB20000DFA3748FCF728FA3648FCF707FA34489C
:10AB3000FCF7A4FD3448FCF701FA4020FEF777F952
:10AB4000A2071AD53148FCF7F9F93148FCF7F6F9B4
:10AB50002B48FFF7F5FE2F48FCF7F0F92848FDF7E2
:10AB6000CDFE2D48FCF7EAF92548FDF72DFE2648D5
:10AB7000FCF7E4F98020FEF75AF963070FD5274860
:10AB8000FCF7DCF92648FCF7D9F91D48FBF7DAFC9D
:10AB90001D48FCF7D3F94FF48070FEF748F905B073
:10ABA000BDE8F08FCD230108B02A0108D4230108A5
:10ABB000DA230108D8190020E8230108FA23010844
:10ABC000800D01080624010811240108DE1B01087C
:10ABD0009C220108C91C0108192401082B24010822
:10ABE000440B01083B240108480B010849240108D3
:10ABF0005624010890250108622401086B240108ED
:10AC00000F1C0108772401089523010885240108F9
:10AC100098240108A6240108B0240108BF240108D3
:10AC2000D0240108AFF300800148FBF7D7BF00BF75
:10AC3000000800400148FBF7D1BF00BF00040040FE
:10AC40004FF08040FBF7CABF0148FBF7C7BF00BF0A
:10AC5000002C014038B5194C236D1D88ADB2AA06F1
:10AC600012D5E26A1AB1988880B290470CE09B88AE
:10AC7000E2696169DBB28B54E269E3680132B2FBDD
:10AC8000F3F103FB1123E3612B0616D5A26A616A77
:10AC90000A4B8A420CD09869196D805C0132C0B2AF
:10ACA00088801969B2FBF1F001FB10229A6238BD6D
:10ACB0001B6DDA6822F08002DA6038BD28190020A6
:10ACC0000D4BD3F8A4201188090613D5D96F986FBE
:10ACD00081420BD0D86E405C0131C0B290805A6E78
:10ACE000B1FBF2F002FB1011D9677047D36823F073
:10ACF0008003D360704700BF281900200B480C4B1D
:10AD00004FF400525A60D0F888204FF6FE73116855
:10AD10000B401360826FC36F9A4202D05430FAF72F
:10AD2000B9BB012380F89830704700BF2819002074
:10AD300000000240084A13689B020BD5074B002114
:10AD4000197007494FF6FE73086803400B604FF413
:10AD500000135360704700BF000002407A210020BA
:10AD60006C0002402DE9F743124C814604F198082B
:10AD700094F84A60C6B9D9F804200025009501204E
:10AD800029460323FCF7BAFE074620B97EB94FF4E3
:10AD900096420126F1E7204629464C2203F061FC49
:10ADA0000123276084F84A304C344445E0D103B095
:10ADB000BDE8F0833408002010B50B4B1A7851071A
:10ADC00010D50A4C22F004021A70A3685B0509D55D
:10ADD000FCF7F6FEFEF724FC20B104F59670BDE802
:10ADE0001040BFE710BD00BF7C210020D819002013
:10ADF00070B5F6F723FD38B3144C237A0BB9A38052
:10AE000070BD134D2E78C6F38000F6F729FD90B182
:10AE1000104B46F002061A680F4B51892E701980AC
:10AE20005189598052899A800C4A12685288DA8076
:10AE3000E3880133E380F6F7EDFC10B92B785B076C
:10AE400002D4BDE87040B7E770BD00BFF009002034
:10AE50007C210020EC090020CA040020D019002029
:10AE60000F4B1A6842F001021A6059680D4A0A40F5
:10AE70005A601A6822F0847222F480321A601A68CA
:10AE800022F480221A605A6822F4FE025A604FF4BB
:10AE90001F029A60044B4FF000629A60704700BF37
:10AEA000001002400000FFF800ED00E0024B1A68BD
:10AEB00001321A60704700BFD419002008B5084B52
:10AEC000B3F8D80093F87C270023D9B2914204D27A
:10AED000044921F813000133F7E7F7F74CF8FEE7D0
:10AEE000D41900205221002081F0004102E000BF6F
:10AEF00083F0004330B54FEA41044FEA430594EA3A
:10AF0000050F08BF90EA020F1FBF54EA000C55EA74
:10AF1000020C7FEA645C7FEA655C00F0E2804FEA45
:10AF20005454D4EB5555B8BF6D420CDD2C4480EA27
:10AF3000020281EA030382EA000083EA010180EA57
:10AF4000020281EA0303362D88BF30BD11F0004FA5
:10AF50004FEA01314FF4801C4CEA113102D04042DB
:10AF600061EB410113F0004F4FEA03334CEA133316
:10AF700002D0524263EB430394EA050F00F0A7802E
:10AF8000A4F10104D5F1200E0DDB02FA0EFC22FA29
:10AF900005F2801841F1000103FA0EF2801843FA1D
:10AFA00005F359410EE0A5F120050EF1200E012A0E
:10AFB00003FA0EFC28BF4CF0020C43FA05F3C0184C
:10AFC00051EBE37101F0004507D54FF0000EDCF1C5
:10AFD000000C7EEB00006EEB0101B1F5801F1BD36E
:10AFE000B1F5001F0CD349085FEA30004FEA3C0C72
:10AFF00004F101044FEA445212F5800F80F09A8068
:10B00000BCF1004F08BF5FEA500C50F1000041EB6B
:10B01000045141EA050130BD5FEA4C0C404141EB6F
:10B02000010111F4801FA4F10104E9D191F0000F96
:10B0300004BF01460020B1FA81F308BF2033A3F119
:10B040000B03B3F120020CDA0C3208DD02F1140C10
:10B05000C2F10C0201FA0CF021FA02F10CE002F14B
:10B060001402D8BFC2F1200C01FA02F120FA0CFC44
:10B07000DCBF41EA0C019040E41AA2BF01EB04518D
:10B08000294330BD6FEA04041F3C1CDA0C340EDC8B
:10B0900004F11404C4F1200220FA04F001FA02F3CE
:10B0A00040EA030021FA04F345EA030130BDC4F18C
:10B0B0000C04C4F1200220FA02F001FA04F340EA81
:10B0C0000300294630BD21FA04F0294630BD94F032
:10B0D000000F83F4801306BF81F480110134013D19
:10B0E0004EE77FEA645C18BF7FEA655C29D094EA8A
:10B0F000050F08BF90EA020F05D054EA000C04BF08
:10B100001946104630BD91EA030F1EBF00210020F2
:10B1100030BD5FEA545C05D14000494128BF41F091
:10B12000004130BD14F580043CBF01F5801130BDF5
:10B1300001F0004545F0FE4141F470014FF0000080
:10B1400030BD7FEA645C1ABF194610467FEA655C31
:10B150001CBF0B46024650EA013406BF52EA0335D3
:10B1600091EA030F41F4002130BD00BF90F0000FC1
:10B1700004BF0021704730B54FF4806404F13204FD
:10B180004FF000054FF0000150E700BF90F0000FB6
:10B1900004BF0021704730B54FF4806404F13204DD
:10B1A00010F0004548BF40424FF000013EE700BFAD
:10B1B00042004FEAE2014FEA31014FEA02701FBF3D
:10B1C00012F07F4393F07F4F81F06051704792F00F
:10B1D000000F14BF93F07F4F704730B54FF4607489
:10B1E00001F0004521F0004120E700BF50EA0102D4
:10B1F00008BF704730B54FF000050AE050EA010281
:10B2000008BF704730B511F0004502D5404261EBF0
:10B2100041014FF4806404F132045FEA915C3FF431
:10B22000DCAE4FF003025FEADC0C18BF03325FEACA
:10B23000DC0C18BF033202EBDC02C2F1200300FA7F
:10B2400003FC20FA02F001FA03FE40EA0E0021FAA4
:10B2500002F11444C1E600BF70B54FF0FF0C4CF48E
:10B26000E06C1CEA11541DBF1CEA135594EA0C0F44
:10B2700095EA0C0F00F0DEF82C4481EA030621EA7F
:10B280004C5123EA4C5350EA013518BF52EA0335BA
:10B2900041F4801143F4801338D0A0FB02CE4FF06C
:10B2A0000005E1FB02E506F00042E0FB03E54FF09C
:10B2B0000006E1FB03569CF0000F18BF4EF0010E94
:10B2C000A4F1FF04B6F5007F64F5407404D25FEA90
:10B2D0004E0E6D4146EB060642EAC62141EA555143
:10B2E0004FEAC52040EA5E504FEACE2EB4F1FD0C85
:10B2F00088BFBCF5E06F1ED8BEF1004F08BF5FEA03
:10B30000500E50F1000041EB045170BD06F00046B4
:10B3100046EA010140EA020081EA0301B4EB5C0461
:10B32000C2BFD4EB0C0541EA045170BD41F4801159
:10B330004FF0000E013C00F3AB8014F1360FDEBF7E
:10B34000002001F0004170BDC4F10004203C35DA5A
:10B350000C341BDC04F11404C4F1200500FA05F3DD
:10B3600020FA04F001FA05F240EA020001F000427E
:10B3700021F0004110EBD37021FA04F642EB0601F4
:10B380005EEA430E08BF20EAD37070BDC4F10C041E
:10B39000C4F1200500FA04F320FA05F001FA04F2E2
:10B3A00040EA020001F0004110EBD37041F10001CE
:10B3B0005EEA430E08BF20EAD37070BDC4F12005D9
:10B3C00000FA05F24EEA020E20FA04F301FA05F241
:10B3D00043EA020321FA04F001F0004121FA04F2E9
:10B3E00020EA020000EBD3705EEA430E08BF20EAB9
:10B3F000D37070BD94F0000F0FD101F000464000F3
:10B4000041EB010111F4801F08BF013CF7D041EA74
:10B41000060195F0000F18BF704703F00046520078
:10B4200043EB030313F4801F08BF013DF7D043EA49
:10B430000603704794EA0C0F0CEA135518BF95EAFF
:10B440000C0F0CD050EA410618BF52EA4306D1D186
:10B4500081EA030101F000414FF0000070BD50EAA5
:10B46000410606BF1046194652EA430619D094EA2F
:10B470000C0F02D150EA013613D195EA0C0F05D119
:10B4800052EA03361CBF104619460AD181EA03016D
:10B4900001F0004141F0FE4141F470014FF0000025
:10B4A00070BD41F0FE4141F4780170BD70B54FF0C0
:10B4B000FF0C4CF4E06C1CEA11541DBF1CEA135540
:10B4C00094EA0C0F95EA0C0F00F0A7F8A4EB050422
:10B4D00081EA030E52EA03354FEA013100F0888019
:10B4E0004FEA03334FF0805545EA131343EA1263E2
:10B4F0004FEA022245EA111545EA10654FEA002697
:10B500000EF000419D4208BF964244F1FD0404F54F
:10B51000407402D25B084FEA3202B61A65EB0305AB
:10B520005B084FEA32024FF480104FF4002CB6EB68
:10B53000020E75EB030E22BFB61A754640EA0C00E8
:10B540005B084FEA3202B6EB020E75EB030E22BF28
:10B55000B61A754640EA5C005B084FEA3202B6EB69
:10B56000020E75EB030E22BFB61A754640EA9C0028
:10B570005B084FEA3202B6EB020E75EB030E22BFF8
:10B58000B61A754640EADC0055EA060E18D04FEAB6
:10B59000051545EA16754FEA06164FEAC30343EA56
:10B5A00052734FEAC2025FEA1C1CC0D111F4801F23
:10B5B0000BD141EA00014FF000004FF0004CB6E71C
:10B5C00011F4801F04BF01430020B4F1FD0C88BFBB
:10B5D000BCF5E06F3FF6AFAEB5EB030C04BFB6EBC6
:10B5E000020C5FEA500C50F1000041EB045170BDB9
:10B5F0000EF0004E4EEA113114EB5C04C2BFD4EBE6
:10B600000C0541EA045170BD41F480114FF0000E69
:10B61000013C90E645EA060E8DE60CEA135594EAE5
:10B620000C0F08BF95EA0C0F3FF43BAF94EA0C0FE8
:10B630000AD150EA01347FF434AF95EA0C0F7FF45D
:10B6400025AF104619462CE795EA0C0F06D152EAB1
:10B6500003353FF4FDAE1046194622E750EA410695
:10B6600018BF52EA43067FF4C5AE50EA41047FF4A6
:10B670000DAF52EA43057FF4EBAE12E74FEA410209
:10B6800012F5001215D211D56FF47873B3EB625234
:10B6900012D94FEAC12343F0004343EA505311F05B
:10B6A000004F23FA02F018BF404270474FF00000ED
:10B6B000704750EA013005D111F0004008BF6FF02B
:10B6C000004070474FF00000704700BF4A0011D2A1
:10B6D00012F5001211D20DD56FF47873B3EB6252EC
:10B6E0000ED44FEAC12343F0004343EA505323FAF8
:10B6F00002F070474FF00000704750EA013002D16D
:10B700004FF0FF3070474FF0000070474FEA4102A2
:10B71000B2F1E04324BFB3F5001CDCF1FE5C0DD9AF
:10B7200001F0004C4FEAC0024CEA5070B2F1004FF9
:10B7300040EB830008BF20F00100704711F0804FFC
:10B7400021D113F13872BCBF01F00040704741F4C1
:10B7500080114FEA5252C2F11802C2F1200C10FAC5
:10B760000CF320FA02F018BF40F001004FEAC123A9
:10B770004FEAD32303FA0CFC40EA0C0023FA02F34D
:10B780004FEA4303CCE77FEA625307D150EA013323
:10B790001EBF4FF0FE4040F44000704701F00040F3
:10B7A00040F0FE4040F40000704700BF80F00040D1
:10B7B00002E000BF81F0004142001FBF5FEA410389
:10B7C00092EA030F7FEA226C7FEA236C6AD04FEA89
:10B7D0001262D2EB1363C1BFD218414048404140CE
:10B7E000B8BF5B42192B88BF704710F0004F40F480
:10B7F000000020F07F4018BF404211F0004F41F49C
:10B80000000121F07F4118BF494292EA030F3FD067
:10B81000A2F1010241FA03FC10EB0C00C3F120037A
:10B8200001FA03F100F0004302D5494260EB400009
:10B83000B0F5000F13D3B0F1807F06D340084FEA74
:10B84000310102F10102FE2A51D2B1F1004F40EB69
:10B85000C25008BF20F0010040EA030070474900D1
:10B8600040EB000010F4000FA2F10102EDD1B0FA9C
:10B8700080FCACF1080CB2EB0C0200FA0CF0AABF91
:10B8800000EBC25052421843BCBFD040184370472F
:10B8900092F0000F81F4000106BF80F40000013235
:10B8A000013BB5E74FEA41037FEA226C18BF7FEA0C
:10B8B000236C21D092EA030F04D092F0000F08BF4E
:10B8C0000846704790EA010F1CBF0020704712F035
:10B8D0007F4F04D1400028BF40F00040704712F174
:10B8E00000723CBF00F50000704700F0004343F0D9
:10B8F000FE4040F4000070477FEA226216BF08460F
:10B900007FEA23630146420206BF5FEA412390EAD1
:10B91000010F40F4800070474FF0000304E000BFC7
:10B9200010F0004348BF40425FEA000C08BF704778
:10B9300043F0964301464FF000001CE050EA01023C
:10B9400008BF70474FF000030AE000BF50EA010251
:10B9500008BF704711F0004302D5404261EB41013E
:10B960005FEA010C02BF84460146002043F0B64363
:10B9700008BFA3F18053A3F50003BCFA8CF2083A88
:10B98000A3EBC25310DB01FA02FC634400FA02FC91
:10B99000C2F12002BCF1004F20FA02F243EB020098
:10B9A00008BF20F00100704702F1200201FA02FCFA
:10B9B000C2F1200250EA4C0021FA02F243EB0200ED
:10B9C00008BF20EADC7070474FF0FF0C1CEAD05231
:10B9D0001EBF1CEAD15392EA0C0F93EA0C0F6FD0F2
:10B9E0001A4480EA010C400218BF5FEA41211ED0D0
:10B9F0004FF0006343EA501043EA5111A0FB0131BC
:10BA00000CF00040B1F5000F3EBF490041EAD37190
:10BA10005B0040EA010062F17F02FD2A1DD8B3F10C
:10BA2000004F40EBC25008BF20F00100704790F07B
:10BA3000000F0CF0004C08BF49024CEA502040EACD
:10BA400051207F3AC2BFD2F1FF0340EAC250704793
:10BA500040F400004FF00003013A5DDC12F1190FD1
:10BA6000DCBF00F000407047C2F10002410021FA43
:10BA700002F1C2F1200200FA02FC5FEA310040F15B
:10BA8000000053EA4C0308BF20EADC70704792F0D4
:10BA9000000F00F0004C02BF400010F4000F013A0C
:10BAA000F9D040EA0C0093F0000F01F0004C02BF07
:10BAB000490011F4000F013BF9D041EA0C018FE776
:10BAC0000CEAD15392EA0C0F18BF93EA0C0F0AD07C
:10BAD00030F0004C18BF31F0004CD8D180EA0100A2
:10BAE00000F00040704790F0000F17BF90F0004F3B
:10BAF000084691F0000F91F0004F14D092EA0C0F1D
:10BB000001D142020FD193EA0C0F03D14B0218BFAF
:10BB1000084608D180EA010000F0004040F0FE40F5
:10BB200040F40000704740F0FE4040F44000704791
:10BB30004FF0FF0C1CEAD0521EBF1CEAD15392EA10
:10BB40000C0F93EA0C0F69D0A2EB030280EA010C00
:10BB500049024FEA402037D04FF0805343EA111199
:10BB600043EA10130CF000408B4238BF5B0042F1F7
:10BB70007D024FF4000C8B4224BF5B1A40EA0C009C
:10BB8000B3EB510F24BFA3EB510340EA5C00B3EBCE
:10BB9000910F24BFA3EB910340EA9C00B3EBD10FBC
:10BBA00024BFA3EBD10340EADC001B0118BF5FEA0E
:10BBB0001C1CE0D1FD2A3FF650AF8B4240EBC25037
:10BBC00008BF20F0010070470CF0004C4CEA5020F8
:10BBD0007F32C2BFD2F1FF0340EAC250704740F447
:10BBE00000004FF00003013A37E792F0000F00F039
:10BBF000004C02BF400010F4000F013AF9D040EAB7
:10BC00000C0093F0000F01F0004C02BF490011F44A
:10BC1000000F013BF9D041EA0C0195E70CEAD15342
:10BC200092EA0C0F08D142027FF47DAF93EA0C0F29
:10BC30007FF470AF084676E793EA0C0F04D14B020D
:10BC40003FF44CAF08466EE730F0004C18BF31F0BF
:10BC5000004CCAD130F000427FF45CAF31F00043B9
:10BC60007FF43CAF5FE700BF4FF0FF3C06E000BF52
:10BC70004FF0010C02E000BF4FF0010C4DF804CD75
:10BC80004FEA40024FEA41037FEA226C18BF7FEA85
:10BC9000236C11D001B052EA530C18BF90EA010F87
:10BCA00058BFB2EB030088BFC81738BF6FEAE17016
:10BCB00018BF40F0010070477FEA226C02D15FEAB2
:10BCC000402C05D17FEA236CE4D15FEA412CE1D01E
:10BCD0005DF8040B704700BF844608466146FFE7E5
:10BCE0000FB5FFF7C9FF002848BF10F1000F0FBDC7
:10BCF0004DF808EDFFF7F4FF0CBF012000205DF8C0
:10BD000008FB00BF4DF808EDFFF7EAFF34BF012044
:10BD100000205DF808FB00BF4DF808EDFFF7E0FFDD
:10BD200094BF012000205DF808FB00BF4DF808ED2E
:10BD3000FFF7D2FF94BF012000205DF808FB00BF91
:10BD40004DF808EDFFF7C8FF34BF012000205DF873
:10BD500008FB00BF4FEA4002B2F1FE4F0FD34FF095
:10BD60009E03B3EB12620DD94FEA002343F0004368
:10BD700010F0004F23FA02F018BF404270474FF016
:10BD80000000704712F1610F01D1420205D110F09D
:10BD9000004008BF6FF0004070474FF00000704750
:10BDA00042000ED2B2F1FE4F0BD34FF09E03B3EB25
:10BDB000126209D44FEA002343F0004323FA02F051
:10BDC00070474FF00000704712F1610F01D142023D
:10BDD00002D14FF0FF3070474FF00000704700BFB6
:10BDE00073B96AB9002908BF0028BCBF00204FF012
:10BDF0000041C4BF6FF000414FF0FF3000F03CB88D
:10BE000082B0EC462DE9005000F006F8DDF804E0C1
:10BE100002B00CBC704700BF2DE9704F089E14465D
:10BE20001D468046894600F029F804FB01F3A4FB77
:10BE300000AB00FB05329344B8EB0A0869EB0B0931
:10BE4000C6E90089BDE8708F2DE9704F089E144641
:10BE50001D468046894600F061F900FB05F5A0FB10
:10BE600004AB04FB0154A344B8EB0A0869EB0B09CB
:10BE7000C6E90089BDE8708F704700BF00292DE931
:10BE8000F00FC0F2A1800024002BC0F2988015466C
:10BE900006460F46002B3FD18A4258D9B2FA82F3A8
:10BEA0004BB1C3F1200201FA03F720FA02F29D40E0
:10BEB00000FA03F61743290CB7FBF1F201FB1277E6
:10BEC000A8B200FB02F34FEA164C4CEA0747BB420C
:10BED00009D97F1902F1FF3C80F00581BB4240F295
:10BEE0000281023A2F44FF1AB7FBF1F301FB1371F1
:10BEF00000FB03F0B6B246EA0141884208D949196D
:10BF000003F1FF3780F0F180884240F2EE80023B7F
:10BF100043EA0242002303E08B420AD900231A4677
:10BF20001046194614B1404261EB4101BDE8F00FE3
:10BF30007047B3FA83F8B8F1000F40F088808B4265
:10BF400002D3824200F2E28000230122E8E712B924
:10BF50000123B3FBF2F5B5FA85F2002A3AD17F1B33
:10BF6000280C1FFA85FC0123B7FBF0F100FB1177C9
:10BF70000CFB01F24FEA164848EA0747BA4207D9D4
:10BF80007F1901F1FF3802D2BA4200F2C480414663
:10BF9000BF1AB7FBF0F200FB12700CFB02FCB6B24A
:10BFA00046EA0040844507D9401902F1FF3702D222
:10BFB000844500F2AE803A4642EA0142B0E7E443EB
:10BFC000524263EB430362E7404261EB41014FF0B1
:10BFD000FF3459E79540C2F1200927FA09F126FA02
:10BFE00009F99740280CB1FBF0F800FB18111FFA73
:10BFF00085FC0CFB08F349EA07094FEA194747EAB1
:10C0000001418B4206FA02F608D9491908F1FF32BC
:10C010007AD28B4278D9A8F102082944C91AB1FB17
:10C02000F0F300FB13170CFB03F21FFA89F949EA3E
:10C030000747BA4207D97F1903F1FF3160D2BA42EC
:10C040005ED9023B2F44BF1A43EA08438CE7C8F18C
:10C05000200225FA02F103FA08FC27FA02F320FA7B
:10C0600002F207FA08F741EA0C0C4FEA1C49B3FB4D
:10C07000F9F109FB11331FFA8CFA0AFB01FB174394
:10C080003A0C42EA03439B4505FA08F008D913EB42
:10C090000C0301F1FF3235D29B4533D90239634499
:10C0A000CBEB0303B3FBF9F209FB12330AFB02FAF1
:10C0B000BFB247EA0347BA4508D917EB0C0702F1AC
:10C0C000FF331BD2BA4519D9023A674442EA014507
:10C0D000A5FB0001CAEB07078F424FF000030AD30C
:10C0E00005D02A461CE76246FDE63B4610E706FA05
:10C0F00008F68642F5D26A1E002311E71A46E5E7E4
:10C100000B46A0E71146CBE7904687E743464246F9
:10C1100006E7023A50E702392F4439E72DE9F00FDC
:10C12000144605460E46002B43D18A4253D9B2FA33
:10C1300082F757B1C7F1200620FA06F601FA07F395
:10C1400002FA07F400FA07F51E43210CB6FBF1F2E0
:10C1500001FB1266A0B200FB02F32F0C47EA064671
:10C16000B34209D9361902F1FF3780F0FD80B3429E
:10C1700040F2FA80023A2644F61AB6FBF1F301FBCC
:10C18000136100FB03F0ADB245EA0141884208D9D2
:10C19000091903F1FF3680F0E980884240F2E68019
:10C1A000023B43EA0242002310461946BDE8F00F65
:10C1B00070478B424CD8B3FA83F6002E4FD18B4296
:10C1C00002D3824200F2DD80BDE8F00F002301229D
:10C1D00010461946704712B90124B4FBF2F4B4FAC0
:10C1E00084F2002A40F08280091B260CA7B20123AA
:10C1F000B1FBF6F006FB101107FB00F24FEA154CFD
:10C200004CEA01418A4207D9091900F1FF3C02D2E8
:10C210008A4200F2C8806046891AB1FBF6F206FB3A
:10C22000121107FB02F7ADB245EA0145AF4208D94A
:10C230002C1902F1FF3180F09B80A74240F29880D8
:10C24000023A42EA004210461946BDE8F00F704734
:10C2500000231A4610461946BDE8F00F7047C6F194
:10C26000200522FA05F703FA06F421FA05F301FA8C
:10C2700006FB20FA05F53C434FEA1448B3FBF8FCF3
:10C2800008FB1C331FFA84F909FB0CFA45EA0B0B77
:10C290004FEA1B4545EA03439A4502FA06F204D9E0
:10C2A0001B190CF1FF356FD3AC46CAEB0303B3FB8C
:10C2B000F8F508FB153309FB05F91FFA8BFB4BEA70
:10C2C0000347B94504D93F1905F1FF3362D31D4631
:10C2D00045EA0C4CACFB0223C9EB07079F424FF029
:10C2E00000054AD346D062462B465DE79440C2F132
:10C2F000200921FA09FC914020FA09F9260CBCFB1F
:10C30000F6F806FB18CCA7B207FB08F349EA0109C7
:10C310004FEA194141EA0C4C634500FA02F509D98C
:10C320001CEB040C08F1FF323BD2634539D9A8F16C
:10C330000208A444C3EB0C0CBCFBF6F306FB13C1D0
:10C3400007FB03F21FFA89F949EA01418A4207D93A
:10C35000091903F1FF3022D28A4220D9023B21443D
:10C36000891A43EA084343E73A4605E7334618E7A4
:10C370000A4666E7B0409042B5D20CF1FF32002386
:10C3800012E7334632460FE79A458DD9ACF1020CDD
:10C3900023448AE7B9459AD9023D274498E70346E2
:10C3A000DEE79046C6E70238214435E71C481D49C0
:10C3B000026800608A4200F01D80002100F004B88D
:10C3C000194B5B58435004311848194B42189A4294
:10C3D000FFF4F6AF174A00F003B8002342F8043B1D
:10C3E000154B9A42FFF4F9AFFEF73AFD00F038F82A
:10C3F000FFF7FEBF114E124830601248016821F06D
:10C4000070610160410201600F4C182020600F49EB
:10C410000F4808600F48D0F800D04068004700007F
:10C42000F04F0020EFBEADDE183201080000002002
:10C43000FC0000200001002098210020181002407C
:10C440000900000004000140140C0140000C0140F0
:10C450004434434400F0FF1FFFF7FEBF000000001C
:10C460002DE9804893B0F3F753FEDFF850928E4CDD
:10C47000D9F8086000232370330740F1E780636830
:10C480001B7A042B00F2E080DFE803F00303058A47
:10C49000B100237AD9E0627A834B002A00F0D4807D
:10C4A00000225A7293F82020170700F1CD80D97A24
:10C4B0009A7A01F0070042EA00225A621A7B02F0DF
:10C4C0003F00400140EAD1019962597B890041EA6D
:10C4D00092119A7B02F0010041EA8021D962D97B56
:10C4E00001F00F00C00140EA52021A631A7C02F008
:10C4F0007F00000140EA11115963597C490041EA6B
:10C50000D212997C01F0030042EA40229A63DA7C5D
:10C5100002F01F00800140EA9101D963197DC90032
:10C5200041EA5212997D1A645A7D01F0070042EAED
:10C5300000225A64DA7D02F03F00400140EAD10156
:10C540009964197E890041EA92115A7E02F0010035
:10C5500041EA8021D964997E01F00F00C00140EAD0
:10C5600052021A65DA7E02F07F00000140EA1111E2
:10C570005965197F490041EAD212597F01F0030041
:10C5800042EA40229A659A7F02F01F00800140EA49
:10C590009101D965D97FC90041EA52121A6651E06A
:10C5A00094F86420404B002A4ED0002283F8642087
:10C5B00093F86620012A47D193F88A20102A84BF75
:10C5C000102283F88A2094F88A10384A0023D8B2BF
:10C5D000884202F1020235D212F8010C12F8025C14
:10C5E00040EA0525324840F823500133EFE794F83C
:10C5F000CC202D4B42B3002283F8CC2093F8CD20E1
:10C60000A82A21D193F8E050F5B9274901EB450359
:10C6100093F8D00093F8D13003EB0020FEF7A6FD8D
:10C620001DA3D3E90023FEF741FF1DA3D3E9002397
:10C63000FEF75EFCFFF74AF81E4B43F82500013574
:10C64000082DE2D1012300E000232370750408D5F2
:10C6500094F8043123B1144B002283F80421012300
:10C66000237023783BB1F00505D50F4BD3F8083183
:10C670001B681B689847104D23782A6833B90A4B0A
:10C68000D3F80C31D31ADB43DB0F00E00123BBB13D
:10C69000F6F73AF928E000BF9A99999999991940C3
:10C6A00000000000007077400001002068010020B9
:10C6B0008C010020E40100206C210020D81900200A
:10C6C000D4F810315A1CC4F810212BB9D9F808300D
:10C6D000190601D5F7F70CFDD4F81031012B03DD55
:10C6E000A44B0022C3F81021F5F7CEFAB9F80C30AC
:10C6F00028602BB1D4F81421821A002AC1F2798162
:10C700009C4D184499F80570D4F82031C4F81401F0
:10C7100005F59670D4F818610597984705F5967059
:10C72000014694F83221F9F721F9934B1B88002B2D
:10C7300000F09880D5F834314FF000081B7805F5EB
:10C740009C75049347468C4BB3F800A08B4BBAF50D
:10C750007A7F03D1002243F808202A61884AD05FFB
:10C7600053F80820024443F80820FFF7D9F82A6953
:10C770000132012A2A6104D1002368602860AB607D
:10C780002AE0D5F800C001926146CDF808C00390B8
:10C79000FFF710F8019A83461046FFF7C1F80146EB
:10C7A0005846FFF7C5F9DDF808C001466046FFF7B7
:10C7B00003F8039B02461146686018460192FEF793
:10C7C000F9FF01465846FFF7FFF8A968FEF7F4FFA6
:10C7D000019AE8602A60A860694A002302F1540BBC
:10C7E000BAF1010FBB5227F80B30DFF88CA12CD126
:10C7F0002869012807DD0138FFF792F80146E8684B
:10C80000FFF796F900E0002002F05EFA0346049874
:10C8100058B10393FFF784F8039B01461846FFF7CE
:10C820008FFA10B14FF47A731AE0544B4FF47A72C6
:10C8300058F803300A2003F5FA7393FBF2F32BF850
:10C8400007300F210122F5F755FA0237062F08F1BC
:10C85000040805F114057FF476AFBAF80030013B07
:10C86000AAF800300023434D05F5967205F5C07116
:10C87000985A595A411A99520233062BF3D1D5F8D6
:10C88000883113F0020300F0FF82D5F8903105F5EE
:10C89000CC70984705F5CC70014695F89E21F9F7C4
:10C8A00065F8B5F8A03105F5CC77002B44D000220F
:10C8B000D5F8A40113462F4D37F902C0B5F8A011E1
:10C8C00005F5D47EB1F5C87F04BF00214EF80310F2
:10C8D0005EF80310274D61444EF803100433002125
:10C8E0000C2BB952815202F10202E4D1B5F8A03109
:10C8F000012B1CD1D5F8A8314FF4C872C83393FB73
:10C90000F2F30380D5F8AC31C83393FBF2F34380E4
:10C91000D5F8B031C83393FBF2F21A4B1B88D21A08
:10C920008280A6F85410A6F85610FDF7FDFFB4F863
:10C93000A031013BA4F8A031D9F808305A0740F1E2
:10C940008680B4F8B4210B4B322A1DD1D3F8A42130
:10C950001188A3F8B61151889288A3F8B811A3F8EA
:10C96000BA21B6F85420A3F8BC21B6F85620A3F893
:10C97000BE210BE00001002078210020740200207D
:10C980002C02002000000020002A3ED00021D4F814
:10C99000A4510A46904837F901C0B0F8B43100F507
:10C9A000E07E322B04BF00234EF802305EF8020016
:10C9B000894B60444EF80200043200200C2A785261
:10C9C000685201F10201E5D1B3F8B421012A17D16F
:10C9D00083F8CD21052283F8CE21B3F8B62183F860
:10C9E000CC012A80B3F8B8216A80B3F8BA21AA80B2
:10C9F000B3F8BC21B3F8BE31A6F85420A6F85630DF
:10CA0000B4F8B431013BA4F8B43194F8CF21724B9F
:10CA1000EAB1D3F8C001D3F8A4113225002290FB6B
:10CA2000F5F083F8CF210880D3F8C40190FBF5F02E
:10CA30004880D3F8C83193FBF5F5684B1B88ED1A95
:10CA40008D80A6F85420A6F85620FDF76DFFD4F887
:10CA5000A431B4F898111A8800268A1AA4F89821EB
:10CA6000B4F89A115A88B3468A1AA4F89A219B8876
:10CA7000B4F89C21D31AA4F89C31F5F705F9D4F841
:10CA8000D0310546C31A18460493FEF745FFD4F883
:10CA9000D4110690FEF798FFD4F8D881C4F8D0518D
:10CAA00098F80090079035464D4F785FFEF738FFB5
:10CAB0000799FEF789FF09A98851B9F1000F2BD01A
:10CAC0004846FEF72DFF01464FF07E50FFF730F845
:10CAD0000346194607F1B00A4FF07E500393FEF764
:10CAE00069FE56F80A10FEF76FFF07F16C01024667
:10CAF000485F0192FEF714FF039BBC371946FEF70F
:10CB000063FF019A01461046FEF756FE4AF80600FA
:10CB1000FFF720F9785304E007F1BC036C37EA5BB8
:10CB2000EA52304F0436EB5F0235062D03FB03BBA0
:10CB3000BAD12A4D642303FB0BFB2B8807F10800B5
:10CB40005B439BFBF3FBABF1490B09A91FFA8BFB82
:10CB5000F5F756FABBF13B0FD8F8046011D9B4F9D8
:10CB6000FC01FEF7DDFED4F8F86101463046FFF720
:10CB7000E7F8194F94F8FE31002837D043F0080346
:10CB800036E04FF07E513046FEF716FE01464FF07C
:10CB90007E50FEF7CDFF4FF0000A8146DFF848B027
:10CBA00030465BF81A10FEF70FFF034637F90A000C
:10CBB0000393FEF7B5FE039B01461846FEF7FCFD06
:10CBC0004946FEF701FF4BF81A000AF1020ABAF1D2
:10CBD000060FE3D1C3E700BF0001002000000020E2
:10CBE0002C020020E8020020F002002023F00803BD
:10CBF0003146D4F8F40187F8FE3102F063F80746B5
:10CC0000C4F80002D4F8F001D4F8F8A100F100460D
:10CC1000D4F8F4010146FEF7D7FE5146814650464E
:10CC2000FEF7D2FE01464846FEF7C6FD02F04CF87C
:10CC30000146304602F046F80646C4F8040238467B
:10CC4000FEF7B6FAC4A3D3E90023FEF705FBFEF70F
:10CC50005DFD01F06BFFA4F808023046FEF7A8FA6C
:10CC6000BDA3D3E90023FEF7F7FAFEF74FFD01F06D
:10CC70005DFFD4F88831A4F80A021B0725D5BA480D
:10CC800009A9F5F7BDF9D8F808504FF07E512846AC
:10CC9000FEF792FD01464FF07E50FEF749FFDFF8A8
:10CCA000E8A281460AF10C0BDAF804102846FEF7D8
:10CCB0008BFE0021FEF780FD4946FEF785FE4AF80F
:10CCC000040FDA45F0D1A8483CE0DFF8B09209A99A
:10CCD00009F10400F5F794F96868D5F808A0014651
:10CCE000FEF772FE514683465046FEF76DFE014642
:10CCF0005846FEF761FDED68824629462846FEF754
:10CD000063FE01465046FEF757FD01F0DDFF0021AE
:10CD10000546FEF7EDFFA0B9D9F804002946FEF755
:10CD200007FF2946C9F80400D9F80800FEF700FFFC
:10CD30002946C9F80800D9F80C00FEF7F9FEC9F831
:10CD40000C008A48F5F714FA8949A4F818020698E5
:10CD5000FEF73AFE06F10046054607F10047B4F932
:10CD600018020D960C97FEF7DBFD00F10040FEF770
:10CD70001FFA7BA3D3E90023FEF76EFAFEF7C6FC89
:10CD80000E90B4F9E801FEF7CBFD0F90B4F9EA017B
:10CD9000FEF7C6FD1090B4F9EC01FEF7C1FD0CA939
:10CDA00011900FA8F5F72CF998F80130714E012B6E
:10CDB00018D1714B1B785F070ED4D6F81C32402077
:10CDC00093FBF0F0181AFEF7ABFD1199FEF7F4FC97
:10CDD000FEF7C0FFC6F81C02D4F81C32402093FBBB
:10CDE000F0F001E0654B1888FEF79AFD01461198B6
:10CDF000FEF7E0FCD4F8241211902846FEF7DCFC84
:10CE000001462846FEF794FED4F8206205463146D6
:10CE10001198FEF7CFFC01462846FEF7D5FD0146E6
:10CE20003046FEF7C9FC0646C4F820020F98D4F835
:10CE3000287201F07BFED4F834522978F5F744FBD0
:10CE40003844C4F828021098D4F82C7201F06EFE11
:10CE50002978F5F739FB3844C4F82C023046D4F869
:10CE6000307201F063FE6978F5F72EFB444B049DA8
:10CE70001A6838442A441A60D4F83832C4F83002A8
:10CE80000133C4F8383205E0A5F89831A5F89A3195
:10CE9000A5F89C31B4F82C21059EA4F83C22B4F8E6
:10CEA0002E21012E334BA4F83E220ED1B3F94212AB
:10CEB000B3F9302102EB4102032192FBF1F292B26D
:10CEC000A3F84022A3F8422203E0B3F83021A3F8EC
:10CED0004022F4F7D9FE2B4B264D1860D4F8483287
:10CEE000C4F84802C31AA4F84432F6F709FAD4F891
:10CEF0004C3213F4801300F0AA80B5F850321806B3
:10CF000000F1ED801C4B1B78590740F18D8095F89E
:10CF100052221A4B12B195F853223AB10022C4F8AA
:10CF2000542201221A74002284F853221B7CD4F864
:10CF30001851032B95F800800E4E05F1040784F874
:10CF4000523223D1384606F516714C2201F080FB8F
:10CF500060E000BFAFF300803B597E90A9E78140BD
:10CF6000399D52A246DF913F0C03002004000020AF
:10CF7000BD378635000100207C2100200000002004
:10CF8000742100206C21002008030020012B07D110
:10CF900006F5167039464C2201F05AFB002302E0D8
:10CFA000022B02D1012386F8A432012384F8A53292
:10CFB00084F8A6320023C4F8A832C4F8AC32A64ADA
:10CFC00094F8A432C4F8B072D35CA44A1D4484F827
:10CFD000B532C4F85422287984F8B482FEF7A0FC54
:10CFE0009F49FEF7A5FDC4F8B802A87BFEF798FCA0
:10CFF0009C49FEF79DFDC4F8BC02287EFEF790FC1C
:10D000009949FEF7E1FCC4F8C002FEF7C9FE00230F
:10D010002876AB73B4F8503243F08003A4F8503252
:10D02000012384F8C4325AE00026D5F85402314670
:10D03000FEF75EFE0746002851D1FDF775FC8B4BCD
:10D040000122C5F8546285F852721A7447E0B5F8A7
:10D05000509219F0800F37D095F85222834F511E0D
:10D06000012924D87F49D5F8BC02FEF7ADFCFEF7B4
:10D0700097FED5F8B06295F8B5827D49B04488F83E
:10D080000A00D5F8C002FEF79FFCFEF789FE88F87B
:10D0900014003078FEF744FC0146FEF78DFBFEF7E6
:10D0A0007FFEB37AB0703373337DB37505E0032A26
:10D0B00003D185F85232012301E03B7C013329F092
:10D0C00080093B74A4F850926A4B1B785A0706D427
:10D0D00094F8C4321BB1684B012283F85322D4F870
:10D0E0001881654D98F86471002F53D0B5F850320F
:10D0F0009B074FD0D5F8F001D5F8F4B10146FEF703
:10D1000063FC594682465846FEF75EFC014650468F
:10D11000FEF752FBD5F8F861824631463046FEF7FD
:10D1200053FC01465046FEF747FBB5F8CC9201F0A0
:10D13000CBFD01463046FEF7FBFC50490646FEF7A4
:10D14000EBFD18BB304601F06DFDD5F8D012FEF7AF
:10D150003BFC01F0EBFCB0F5617FA8BF4FF46170C0
:10D16000FEF714F83AA3D3E90023FEF79FF9FEF780
:10D17000CDFA01F019FD05463846FEF7D1FB2946E8
:10D18000FEF722FC01F0D2FC80B200E0002048440F
:10D19000A4F8CC02D4F88831374D9F0640F1A28024
:10D1A000B5F8503203F03003002B00F09B8095F867
:10D1B000FE31DE0740F19680B5F91802FEF7B0FBAC
:10D1C0002F49FEF701FC064601F0EEFC8146304691
:10D1D00001F076FCD5F8D432074693F803A0B5F9F0
:10D1E000DE02284EBAF1000F4ED0B5F8DA32CAF19D
:10D1F00000051FFA83FB1BB2C01AF5F7D7FAA84245
:10D2000003DB5045A8BF504600E02846B4F8D832AA
:10D210008344B4F9DC029AB21BB21FFA8BFBC01A2A
:10D22000A4F8DAB20192F5F7C1FAA842019A03DB39
:10D230005045B4BF054655461544ADB2A4F8D85282
:10D240000FFA8BF0FEF76CFB824628B221E000BF9C
:10D25000A2EB0FE5DD169640980101080000A04101
:10D260000000204100007A445555553F0000002041
:10D270009A99993F7C210020000100208FC2753CC3
:10D2800035FA8E3C70210020FEF74AFB8246B5F944
:10D29000DC02FEF745FB394605465046FEF794FB97
:10D2A000494683462846FEF78FFB01465846FEF75F
:10D2B00081FABD49FEF73CFCFEF74CFD4946308043
:10D2C0005046FEF781FB394681462846FEF77CFB37
:10D2D00001464846FEF770FAB349FEF729FCFEF70F
:10D2E00039FD7080B14BB24F1E6808F1040008F19F
:10D2F0005403D4F8E012B7F8F620B047AD4BAE4D6A
:10D3000093F800A0BAF1030F13D9B5F9CA02B5F921
:10D31000E8120028B8BF40426FF06302121A91422F
:10D3200004DB00F164028A42A8BF0A46A4F8E8229E
:10D3300020E0BAF1010F1DD894F8EA329F4D013B6D
:10D34000142B00F2FE81DFE813F09B00FC01FC01CE
:10D350006D00A900FC01FC015A01FC01FC01FC016B
:10D36000FC01FC01C600FC01FC01FC01FC01FC010C
:10D37000B901D101D4F8EC32B4F8CC22B4F8E68289
:10D38000B4F8E492B4F9E8B28D4D04930026564502
:10D3900005F11005D0D210B20192FEF7C1FA55F88E
:10D3A000101CFEF711FB84460FFA88F0CDF808C078
:10D3B000FEF7B6FA55F8081CFEF706FBDDF808C0C4
:10D3C00001466046FEF7F8F984460FFA89F0CDF879
:10D3D00008C0FEF7A5FA55F80C1CFEF7F5FADDF8C3
:10D3E00008C001466046FEF7E7F9049B844693F9BE
:10D3F0000000CDF808C040420BFB00F0FEF790FAA9
:10D4000055F8041CFEF7E0FADDF808C00146604656
:10D41000FEF7D2F9FEF79EFC6A49019A21F8160040
:10D420000136B4E702210420F4F7C0FDB4F8E88225
:10D43000012100FB08F01FFA80F90420F4F7B6FD83
:10D44000B4F8E66200FB06901FFA80F90420F4F7B6
:10D45000BBFD4844288102210520F4F7A7FD00FB0D
:10D4600008F001211FFA80F80520F4F79FFD00FB6A
:10D4700006801FFA80F80520F4F7A6FD40440BE073
:10D4800005200121F4F792FDB4F8E862704386B2FA
:10D490000520F4F799FD3044688152E10020F4F74B
:10D4A00093FDD4F8B063B4F90A2296F906304FF030
:10D4B0003208534393FBF8F3184428800120F4F713
:10D4C00083FD96F90E30B4F90822534393FBF8F824
:10D4D0004044688035E13C4B1B78580703D4D4F8AE
:10D4E000B4339B880BE0D4F8B413B4F9CC220B8886
:10D4F00049889A4203DB9142B4BF0B461346EB8145
:10D50000EA89304B1A80D4F8B8331E7866B302200B
:10D51000F4F75AFD284BD3F8B033B3F91020598AE9
:10D52000904203DB0AB29042B8BF0246D4F8BC1363
:10D5300021484989C2EB010EB4F8C0230FFA8EFED0
:10D540000FFA82FCF44501DA164401E002DD961B75
:10D55000A0F8C063B4F9C02393F916305343642292
:10D5600093FBF2F31944A980B4F85022124BD10571
:10D570000FD5B3F8C622EA802A81B3F8CA22B3F8DD
:10D58000C8326A81AB81D4F8B0A3DFF830800326BB
:10D590001CE0B3F8E422EA802A81B3F8E822B3F869
:10D5A000E6326A81EEE700BF000020417C000020E7
:10D5B000D819002050210020000100206C0000201C
:10D5C000F0030020522100207C2100200AEBC6033A
:10D5D00093F90630B8F90690304609FB03F9642345
:10D5E00099FBF3F9A8F80690F4F7EEFC01364844ED
:10D5F000072EA8F8060008F10208E7D1A1E0BD4B0C
:10D600001B785A0703D4D4F8B4339B880BE0D4F8C2
:10D61000B413B4F9CC220B8849889A4203DB9142B7
:10D62000B4BF0B461346EB81EA89B34BB34E1A8065
:10D63000B4F85032DFF8C882DB054FF003004FF03A
:10D6400001010ED5F4F7B2FCB8F8C892022100FB34
:10D6500009F01FFA80FA0320F4F7A8FCB8F8C68294
:10D660000DE0F4F7A3FCB8F8E692022100FB09F004
:10D670001FFA80FA0320F4F799FCB8F8E48200FB63
:10D6800008A00121F0800420F4F790FC00FB09F0D1
:10D6900002211FFA80F90420F4F788FC00FB0890AF
:10D6A00030810320F4F790FCEB881844E8800420D4
:10D6B000F4F78AFC2B891844288142E001210420D8
:10D6C000F4F774FCB4F8E662704386B204202E814D
:10D6D000F4F77AFC3044288101210520F4F766FC38
:10D6E000B4F8E462704386B26E81D1E6B4F8E89291
:10D6F000032630460221F4F759FC00FB09F0012112
:10D700001FFA80F83046F4F751FCC6F106037C4955
:10D7100023F001030B44B3F8E43200FB03801FFA4B
:10D7200080F825F816803046F4F74EFC404425F882
:10D7300016000136072EDCD1714BB3F8CC226E4BAC
:10D740001A80BB68990633D50020F4F73DFC288089
:10D7500080460120F4F738FCD4F84C22674E1206BC
:10D760006880674B24D5D3F8C423B3F90AE2127852
:10D7700012F0020FB3F908221ED0D3F8B03393F998
:10D780000E1093F906304A435B420EFB03FE322132
:10D7900092FBF1F26FF0310392B29EFBF3F313446C
:10D7A0009EFBF1FE98447244A6F8008010447080FD
:10D7B000D4F8B013002316E0D3F8B01391F9063073
:10D7C0000EFB03FE32239EFBF3FEF044A6F800801E
:10D7D00091F90E104A4392FBF3F31844E7E7EA523B
:10D7E0000233102B0CD0E85E31F9232001EB8306C5
:10D7F00090427688F3DB32B28242A8BF0246EEE75F
:10D80000D4F8C4331B785E0705D43E4B3A4A1878E7
:10D810001188012321E03A4B002693F8C8830423A2
:10D82000A8F104085FFA88F85FFA88F94FFA89F2DC
:10D83000D6420ED4324A03F1010A08EB060002EB8D
:10D840004303B3F8CA135FFA8AFAC0B2F4F7FFFFD2
:10D8500053460136042EE9D1D7E7834208D232F984
:10D86000136009B28E42A8BF314689B20133F4E792
:10D87000BB68D4F8B42303F4805B03F01003059372
:10D880001C4BB4F9D0631B78D4F8BC7303F00403C9
:10D89000DBB2D4F8F0E304934FEA400900234B4590
:10D8A00057D0B2F8028008B24045134806DD30F880
:10D8B00003C0C1EB0808C44420F803C0BBF1000F4B
:10D8C00022D0B7F80AC030F903806645CBBFBEF856
:10D8D00002009088B2F802A0BEF800A08045DFF8F0
:10D8E00018C003DBD045B4BF404650462CF80300B7
:10D8F00025E000BF7C210020522100206C00002088
:10D90000000100205021002030F903C01088B2F837
:10D910000280844503DBC445B4BF60464046DFF85F
:10D92000248223F80800B88903EB080C864206DA43
:10D93000059808B9108800E09088ACF800000498B9
:10D9400028B97F4833F800C07E4823F800C002336E
:10D95000A5E7D4F80C34002B49D07B4B93F8EA327E
:10D96000013B142B3DD8DFE803F00B3C3C26403C48
:10D970003C1F3C3C3C3C3C2D3C3C3C3C3C262D0074
:10D98000D4F8EC325B782BB1704B00205989F4F756
:10D990005EFF2CE06E4B1B7803F0040303F0FF00E6
:10D9A000002BF1D10146F2E70020E988F4F74FFFA0
:10D9B00001202989EBE700202989F4F748FF01209D
:10D9C0006989E4E70020E988F4F741FF012029890B
:10D9D000F4F73DFF02206989F4F739FF0320A98994
:10D9E000D5E75C4B9B68980601D5F4F73BFFF4F74D
:10D9F000C2FA594B1B78002B40F0B283DFF85481F8
:10DA0000D8F80830590540F1AB8394F810344E4EE5
:10DA1000002B00F0A583F4F799FD002800F0A08307
:10DA200096F81134002B00F09B83D6F814341B7841
:10DA3000002B40F04E82D6F81804F4F7B1F9002814
:10DA400040F04782454DD6F81C242B689A1A7C2A50
:10DA500040F23F82C6F81C3496F82034013386F831
:10DA60002034064606F12400374FC0B2F4F74CFAD2
:10DA700007F5F47333F91600FDF752FF384B814672
:10DA80001888FDF74DFF01464846FEF751F8354925
:10DA9000FDF79AFFFEF75EF9013600B2F4F760FA7F
:10DAA000032EDFD13020F4F72FFA0020F4F758FAD4
:10DAB000F4F738FA97F8206416F0030620D1D7F867
:10DAC0001C2441F288339A420BD91020F4F71CFA37
:10DAD0003046F4F745FA2120F4F716FA3046F4F709
:10DAE0003FFA1420F4F710FAB4F91802F4F738FAF0
:10DAF0001C20F4F709FA0020F4F732FAF4F712FACE
:10DB000094F82034104E5A0740F0BE810220F4F7FA
:10DB1000FBF9B6F922040A2390FBF3F0F4F720FA9C
:10DB20000320F4F7F1F90A4B1B7813F0040F4FF0C0
:10DB3000050319D0B6F9CC0290FBF3F01AE000BF50
:10DB4000F404002052210020000100206C0000207D
:10DB50007C210020D81900207B210020D41900202E
:10DB60000000002000007A44D6F82424D289B2FBB9
:10DB7000F3F000B2F4F7F4F9D8F808309B0740F15D
:10DB80008A80974E94F82824337840F63401B2FB0B
:10DB9000F3F24A432A21B2FBF1F2B4F82A14062028
:10DBA00091FBF3F803FB18184FEA08181FFA88F8DE
:10DBB00048EA02281FFA88F8C2F3032248EA02085A
:10DBC000F4F7A2F90FFA88F0F4F7CAF9B4F82A24A6
:10DBD0003378013292B292FBF3F103FB1123A4F8E4
:10DBE0002A3494F828346E265E43152396FBF3F608
:10DBF0003A204FF06409F4F787F9B6FBF9F840468C
:10DC0000F4F7AEF93B20F4F77FF909FB186080B216
:10DC10004FF00A08053090FBF8F000B2F4F7A0F9D5
:10DC20002820F4F771F9D4F82C046E4F90FBF8F02B
:10DC300000B2F4F795F9D4F824340420B3F80E8038
:10DC4000F4F762F9D7F830044FF6FF739842A8BF93
:10DC5000184620EAE070B8F1000F19D0C0EB0800B8
:10DC6000FDF794FA0022604BFDF7F6FA06464046AF
:10DC70000F46FDF78BFA02460B4630463946FDF754
:10DC800015FCFDF7FBFC4845A8BF484620EAE070BC
:10DC900000B2F4F765F9D4F88831524E9F0672D578
:10DCA00096F8FE3198071AD51120F4F72DF9B6F839
:10DCB0003404FDF76BFA46A3D3E90023FDF7CCFA51
:10DCC00000224A4BFDF716F9FDF7D8FC00B2F4F735
:10DCD00047F91920F4F718F90020F4F741F994F8FE
:10DCE000FE31B4F8366413F0020F08BF002601209D
:10DCF000F4F70AF930B2F4F733F90920F4F704F92C
:10DD00000020F4F72DF93A4B94F838641B88B3F5EA
:10DD1000967F0BD9334A92F8202402F00F02072A8B
:10DD200004D842F20F76B342B8BF1E460520F4F77E
:10DD3000EBF8D4F824345B7B0BB930B221E0A6F1C8
:10DD40002000FDF723FA24A3D3E90023FDF7AEFB5F
:10DD5000FDF7DCFC8046FDF72BFA06460F464046F1
:10DD60000021FDF7CFFF002208B1224B00E01F4B3E
:10DD700030463946FDF7BEF8FDF7C8FCFDF7EAFF6F
:10DD800000B2F4F7EDF8D4F8883199060ED4154BAB
:10DD90000021D3F824647068FDF7AAFF002871D130
:10DDA000B0680021FDF7A4FF00286BD194F8FE2194
:10DDB0000C4B920703D493F83924012A1CD1012378
:10DDC000D4F83C74D4F8406484F8393424E000BFBB
:10DDD0007B14AE47E17A843FCDCCCCCCCCCCFC3F9D
:10DDE0008000002000010020000059400000E03FBA
:10DDF000820000200000E0BFD3F82464B8497068B6
:10DE0000FDF7E2FDFDF7A6FFB5490746B068FDF74F
:10DE1000DBFDFDF79FFF06460FA93846F4F76CFBC4
:10DE20001320F4F771F8BDF93C00F4F799F81B20C2
:10DE3000F4F76AF8BDF93E00F4F792F82320F4F7FE
:10DE400063F8002FACBF4E205320F4F789F80FA9D8
:10DE50003046F4F751FB1220F4F756F8BDF93C00B8
:10DE6000F4F77EF81A20F4F74FF8BDF93E00F4F706
:10DE700077F82220F4F748F8002EACBF4520572051
:10DE8000F4F76EF8F4F74EF894F82034282B20D1EC
:10DE9000944B00222F6883F820244FF47A73B7FB49
:10DEA000F3F73C251720F4F72FF8B7FBF5F6B6FB90
:10DEB000F5F005FB1060000200B2F4F751F81820ED
:10DEC000F4F722F805FB167000B2F4F749F8F4F7FE
:10DED00029F8D4F81434834D1B78012B40F01E81AF
:10DEE000F3F7D2FED5F844347F4AC31A934206466C
:10DEF00040F2AA8095F82824002385F8662485F846
:10DF00005C24D5F82C2485F84A3485F84C3485F8FF
:10DF1000673485F85D340A2392FBF3F285F86424B4
:10DF2000121285F86524D5F8302492FBF3F385F8B6
:10DF3000683495F8FE211B1285F8693495F8383459
:10DF4000970785F88E3403D42D2385F88F3479E034
:10DF5000042B8CBF3323322385F88F346348D4F8E5
:10DF60003C54DFF890C195FBF0F70CFB07584FF0DD
:10DF7000060E0EFB08F85E4B07EB870798FBF3F9DC
:10DF800003FB198807EB87074FFA89F9D4F8401487
:10DF900009EB8707BFB291FBF0F084F87E743F0A6B
:10DFA00084F87F740CFB00170EFB07F7ED0F84F865
:10DFB0007D5497FBF3F503FB1573642293FBF2F397
:10DFC00084F885341B1284F88634B4F8343498FB12
:10DFD000F2F8B3FBF2F202EBC202920092B2B4F892
:10DFE000A03484F87B24120A84F87C2484F88734D3
:10DFF000B4F836241B0A84F888340A23B2FBF3F3FE
:10E0000000EB800003F5FA739BB26DB200EB800069
:10E0100005EB800084F889341B0A80B284F88A34C6
:10E02000B4F8A23484F88084C90F4FEA282884F811
:10E030008304000A84F8818484F8821484F88404B8
:10E0400084F89034C4F8446494F8A434254D5BB942
:10E05000D5F8A804F3F7A4FE95F87935002B40F025
:10E06000C082012800F2C582D4F8B0241D4D002AD8
:10E0700054D095F8A4743FB1D5F8B43440F6B73114
:10E08000F31A8B420BD849E00123D5F8A8040221EA
:10E0900085F8A434F3F770FE85F8B8743CE095F881
:10E0A000B9345BB9D5F8A8040121C5F8B03485F8B6
:10E0B000A434F3F761FEF3F778FE2DE0013BDBB209
:10E0C00085F8B93495F8B81495F8BA04A3B90130B5
:10E0D0004B1C85F8BA0485F8B834D5F8A80419E0C3
:10E0E0008096184B000100203F0D03008096980099
:10E0F00040420F00806967FF134613F8012B01307F
:10E10000114485F8BA04D5F8A80485F8B814C5F800
:10E11000B0341146F3F756FEC4F8B464D4F814349E
:10E12000AE4D1B78022B1BD1D5F8BC34C3B1C5F85A
:10E13000C0341B68AA4AC5F8C434D5F8C83413449F
:10E140009878FBF747FCD5F8C0349879F3F73FFE91
:10E15000D5F8C8340133092B88BF0023C5F8C8346B
:10E16000DFF8B8A2DAF80830DD037EF57EA994F86E
:10E17000CC349A4E002B3EF478A99A4B1B78002B96
:10E180007EF473A9F3F780FDD6F8D0340546C31AA0
:10E190006FEA0308D6F8D4344FEAD878C31A6FEA86
:10E1A0000309D6F8D8344FEAD979C3EB000B6FEAEC
:10E1B0000B0B4FEADB7BBBF1000F06D1B9F1000F6F
:10E1C00003D1B8F1000F3EF450A90027DFF80CC2CC
:10E1D000FEB2624692F860359E423AD28249DCF83D
:10E1E000DC34B200096813446244C2F8E014598870
:10E1F000C8050BD48B052AD57C4B1B785E0754BF12
:10E200007B4B7C4B1B68C2F8E03420E019467A4A0D
:10E2100030460393CDF808C0FAF772FFDDF808C066
:10E22000039BBCF8502212F0400F03D03046194631
:10E23000724A0AE0900703D530461946704A04E056
:10E24000D10704D56F4A30461946FAF759FF01370E
:10E25000BCE79E000023B3421FD06049D1F8DC2404
:10E260001A445288520516D501F59C62D058089080
:10E27000B1F9D0037821A0F57A7048434FF47A7150
:10E2800090FBF1F000F22B1040F2671190FBF1F7D8
:10E2900001FB170199520433DDE7BBF1000F32D0C7
:10E2A00005F5C333A033C4F8D83494F861354B4E28
:10E2B00033BB86F86235DAF8083001279B0786F809
:10E2C000617504D5F7F70AFC08B186F86275D4F8D1
:10E2D0006435424E1B689B68984728B196F86235B2
:10E2E00043F0020386F86235404B1B7813F0050FAC
:10E2F00009D194F8623543F0040384F8623502E0F2
:10E30000002386F8613594F86225344B1AB9B9F1C7
:10E31000000F42D187E093F8617537B193F8681523
:10E32000013101F0030183F8681500262B4BF1B28F
:10E3300093F860058842EAD9D3F8DC0489000844E0
:10E340004088000627D593F868058FB920B9500793
:10E3500021D50B442C491BE0012804D1D0071AD544
:10E360000B442A4914E0900715D50B4428490FE0C7
:10E3700010B912F0040F03E0012805D112F0010FCB
:10E3800009D00B44184903E0900704D50B442149F8
:10E390000968C3F8E0140136C8E7B4F9C832B4F923
:10E3A000C6223221002AB8BF5242002BB8BF5B42BE
:10E3B00093FBF1F392FBF1F1DBB2C9B28B4238BFB0
:10E3C0000B46154A0BB192FBF3F22A44C4F8D4244D
:10E3D00094F86925014B1ABB012222E000010020BC
:10E3E000980101087A210020CC1801087C21002026
:10E3F000A4010108A8010108AC010108B20101084B
:10E40000B8010108BE010108C4010108C8010108E2
:10E41000CC010108D0010108400D0300D8190020EB
:10E42000002283F8692594F86925844B22B9844A2F
:10E43000C3F86C25002009E0824AF9E7D3F8DC1420
:10E4400094000E197688760607D401307B4BC2B251
:10E4500093F860159142F1D89FE0B3F9C662192E86
:10E4600021DD11F8227093F870E507F00F0CF445E8
:10E47000D3F86C6508DC93F871E5BEEB171F03DC7D
:10E4800023443468C3F8E0446C4B11F8224093F8FD
:10E4900072C504F00F0EE6452DDB93F87175B7EBEE
:10E4A000141F28DC22E0193625DA11F8227093F8BF
:10E4B00070E507F00F0CF445D3F86C6508DC93F8B1
:10E4C00073E5BEEB171F03DB23443468C3F8E04455
:10E4D0005A4B11F8224093F872C504F00F0EE6452E
:10E4E00009DB93F87375B7EB141F04DB346803EB97
:10E4F0008203C3F8E044514BB3F9C842192C21DD23
:10E5000011F8227093F8706507F00F0EB645D3F836
:10E510006C4509DC93F871E5BEEB171F04DC276836
:10E5200003EB8203C3F8E07411F8223003F00F010B
:10E53000B1428ADC414E96F87315B1EB131F84DBB0
:10E54000334624E0193480DA11F8227093F87265AA
:10E5500007F00F0EB645D3F86C4509DB93F871E56B
:10E56000BEEB171F04DC276803EB8203C3F8E074DB
:10E5700011F8223003F00F01B142FFF666AF2F4FC2
:10E5800097F87315B1EB131FFFF65FAF3B4603EB34
:10E5900082022368C2F8E03457E7B8F1000F1CD0BC
:10E5A00093F8752593F8741505F5434588180138D7
:10E5B00090FBF2F402FB140083F87715013183F825
:10E5C000760591FBF2F002FB10125035D2B2C3F87F
:10E5D000D05483F8782583F87425FAF7BBFCFDF74F
:10E5E00044BF00283FF440ADD5F8A804F3F7D3FBAF
:10E5F00021E00228144F03D0F3F7D7FB012303E0F7
:10E600007A7C1AB1C5F8AC647B742DE5D5F8AC34CE
:10E61000F31AB3F57A6FFFF427AD0123D5F8A804F8
:10E620007B74F3F7B8FB0746D5F8A804F3F7B3FB00
:10E63000802F7FF419ADF9F783FD15E50001002067
:10E64000D4010108CC18010800000020AFF30080BD
:10E6500010B50023934203D0CC5CC4540133F9E7D6
:10E6600010BD02440346934202D003F8011BFAE7AF
:10E67000704700000D4B70B51D680022845C2B199B
:10E680005B7803F00303012B8B5C08BF2034EE188A
:10E69000767806F00306012E08BF2033E41A02D173
:10E6A0000132002BEAD1204670BD00BF900000204F
:10E6B00010B50446224613780134002BFAD1CC5C05
:10E6C000D4540133002CFAD110BDC9B2024610F85F
:10E6D000013B1BB18B42F9D1104670470029FBD09A
:10E6E00018467047034613F8012B002AFBD1181A6D
:10E6F000013870470F4BF0B51E680023934215D0C8
:10E70000C55C7419647804F00304012CCC5C08BF68
:10E71000203537197F7807F00307012F08BF203411
:10E720002D1B04D10133002CE8D100E00025284640
:10E73000F0BD00BF9000002010B5034632B111F8C3
:10E74000014B013A03F8014B002CF7D11A449342D4
:10E7500003D0002103F8011BF9E710BD30B50378A1
:10E760000BB1044604E00B78002B18BF002030BD2D
:10E7700022461078013438B10023C85C28B1D55C3A
:10E780008542F5D10133F8E730BD104630BD002198
:10E790000A2200F001B92DE9F04E82468B461F4651
:10E7A000144612B90020BDE8F08E002BFAD00026E6
:10E7B000A642F7D2A5196D0807FB05B95046494690
:10E7C000089B9847002802DB03D06E1C25462C4688
:10E7D000EEE74846BDE8F08E174B2DE9F0411D6885
:10E7E0000646AC6D0F46FCB9502000F0E3F8A86572
:10E7F0008460AB6D046044601C61DC60AB6D9C6147
:10E800005C61AB6DDC629C62AB6D5C631C63AB6D89
:10E81000DC639C63AB6D5C641C64AB6DDC649C640A
:10E82000AB6D1C77AB6D5C6230463946AA6D012337
:10E83000BDE8F04100F002B8F4000020F0B508B9DE
:10E84000106828B3044614F8015B0F4617F8016BF3
:10E850003EB1B542FAD10BB12046F3E71460037024
:10E86000F0BD4DB915602846F0BD17F8016BAE42FA
:10E8700007D0002EF9D11C46234613F8015B0F4642
:10E88000F3E715B10021217000E02B461360F0BDC5
:10E89000F0BD000084463F482DE9F04FD0F80080DD
:10E8A0000E46344614F8015B08EB0500407800F092
:10E8B000080000F0FF0708B12646F2E72D2D03D12E
:10E8C000B41C7578012703E02B2D04BF7578B41CA8
:10E8D00033F010000DD1302D08D1207800F0DF008A
:10E8E000582851D165781023023402E0002B08BF6C
:10E8F0000A23002F0CBF6FF0004A4FF0004ABAFB0A
:10E90000F3F903FB19AA0026304608EB050B9BF828
:10E9100001B01BF0040F01D0303D0BE01BF0030BE6
:10E920001BD0BBF1010F14BF4FF0570B4FF0370B4B
:10E93000CBEB05059D4210DAB6F1FF3F0AD0484502
:10E9400006D801D1554503DC03FB0050012601E048
:10E950004FF0FF3614F8015BD7E7731C0CD1002F82
:10E960004FF022030CBF6FF000404FF00040CCF896
:10E9700000302AB9BDE8F08F07B1404242B106B17C
:10E98000611E1160BDE8F08F002B08BF0823B0E7BF
:10E99000BDE8F08F9000002030B51346044A0546CC
:10E9A0000C46106829462246BDE83040FFF772BF8A
:10E9B000F4000020024B0146186800F003B800BFC5
:10E9C000F400002070B5CD1C25F0030508350C2D92
:10E9D00038BF0C25002D06463FDB8D423DD3214B31
:10E9E0001C6818462146A1B10B685B1B0ED40B2B8B
:10E9F00003D90B60CC18CD501FE08C4202D1626865
:10EA000002601AE04B6863600C4616E00C464968E9
:10EA1000E9E7154C23681BB9304600F027F8206061
:10EA20002946304600F022F8431C014615D0C41C8C
:10EA300024F0030484420AD1256004F10B00231D55
:10EA400020F00700C31A0BD05A42E25070BD304686
:10EA5000611A00F00BF80130EED10C233360002076
:10EA600070BD00BF8C2100208821002038B5064CE5
:10EA7000002305460846236000F008F8431C02D135
:10EA8000236803B12B6038BD94210020094A136824
:10EA900063B118446946884202D81060184670472E
:10EAA000054B0C221A604FF0FF307047034B136088
:10EAB000EFE700BF90210020942100209821002042
:10EAC00000B5194A20F00043934283B0014617DD98
:10EAD000B3F1FF4F04DBFCF76DFE03B05DF804FB00
:10EAE000694600F037FB00F00302012A0098019903
:10EAF00011D0022A0AD09AB1012201F0EFF8ECE716
:10EB0000002100F0EFFC03B05DF804FB00F0EAFC2C
:10EB100000F10040E1E701F0E1F800F10040DCE73E
:10EB200000F0E0FCD9E700BFD80F493F30B5C0F393
:10EB3000C754A4F17F031E2B83B0014620DC581C70
:10EB40001BDB162B4FEAD17509DDC1F3160040F42B
:10EB50000000963CA04005B1404203B030BD114BCF
:10EB600053F825402046FCF727FE019001982146E6
:10EB7000FCF720FE20F0004333B9002003B030BD85
:10EB8000FDF7E8F803B030BDC0F31604C0F3C7507A
:10EB900044F40004C0F1960024FA00F0002DDCD00B
:10EBA000DAE700BF042E010800B51D4A20F000433B
:10EBB000934283B0014618DDB3F1FF4F04DBFCF74D
:10EBC000F9FD03B05DF804FB694600F0C3FA00F0FC
:10EBD0000300012818D002280ED0D0B10098019966
:10EBE00000F080FC00F10040EBE70021002201F082
:10EBF00075F803B05DF804FB00980199012201F05B
:10EC00006DF800F10040DCE70098019900F06AFC23
:10EC1000D7E700980199012201F060F8D1E700BF21
:10EC2000D80F493F70B58AB0054600F09BF8224CDA
:10EC3000064694F90030013303D0284601F02CFA3F
:10EC400010B930460AB070BD284601F0DBF94FF02C
:10EC50007E51FDF775F80028F3D0184901220023F2
:10EC60002846009208930191FCF7A2FA02460B464F
:10EC70001348CDE90423CDE9022301F0A7F894F964
:10EC80000030CDE90601022B0BD0684601F09CF85C
:10EC900038B1089B53B9DDE90601FCF737FD0AB02E
:10ECA00070BD01F073FA21230360F2E701F06EFA00
:10ECB000089B0360EFE700BFF80000200C2E01085E
:10ECC000142E010800F0B6B970B58AB0054600F000
:10ECD000B5FB224C064694F90030013308D0284693
:10ECE00001F0DAF920B128460021FDF70BF810B940
:10ECF00030460AB070BD1A4901220023284601910E
:10ED000000920893FCF754FA2478CDE90401CDE988
:10ED100002017CB900220023CDE90623684601F0F8
:10ED200053F888B1089BA3B9DDE90601FCF7EEFCB6
:10ED30000AB070BD0020002102460B46FCF7B6FB6E
:10ED4000022CCDE90601E9D101F020FA212303606C
:10ED5000E8E701F01BFA089B0360E5E7F8000020F4
:10ED6000182E0108F8B520F00043B3F17E5F044689
:10ED700010D008DCB3F17C5F11DAB3F10C5F00F363
:10ED800084809D48F8BD0146FCF714FD0146FCF760
:10ED9000CFFEF8BD002840F3CD800020F8BD00284C
:10EDA000C0F2CA8001464FF07E50FCF703FD4FF0E1
:10EDB0007C51FCF709FE044600F040FB8F490646F3
:10EDC0002046FCF701FE8E49FCF7F6FC2146FCF7D5
:10EDD000FBFD8C49FCF7EEFC2146FCF7F5FD8A496A
:10EDE000FCF7EAFC2146FCF7EFFD8849FCF7E2FC62
:10EDF0002146FCF7E9FD8649FCF7DEFC2146FCF7DD
:10EE0000E3FD844905462046FCF7DEFD8249FCF718
:10EE1000D1FC2146FCF7D8FD8049FCF7CDFC21460A
:10EE2000FCF7D2FD7E49FCF7C5FC2146FCF7CCFD82
:10EE30004FF07E51FCF7C0FC01462846FCF778FEF7
:10EE40003146FCF7C1FD26F47F6525F00F05074626
:10EE500029462846FCF7B8FD01462046FCF7AAFCE7
:10EE6000294604463046FCF7A7FC01462046FCF73D
:10EE70005FFE01463846FCF79FFC01462846FCF73A
:10EE80009BFC0146FCF798FCF8BD0146FCF79CFD95
:10EE90005A490546FCF798FD5949FCF78DFC29466F
:10EEA000FCF792FD5749FCF785FC2946FCF78CFDE1
:10EEB0005549FCF781FC2946FCF786FD5349FCF7D0
:10EEC00079FC2946FCF780FD5149FCF775FC294681
:10EED000FCF77AFD4F4906462846FCF775FD4E497A
:10EEE000FCF768FC2946FCF76FFD4C49FCF764FC15
:10EEF0002946FCF769FD4A49FCF75CFC2946FCF70A
:10EF000063FD4FF07E51FCF757FC01463046FCF79D
:10EF10000FFE01462046FCF757FD01464148FCF72D
:10EF200049FC01462046FCF745FC01463E48FCF7FB
:10EF300041FCF8BD3D48F8BD4FF07E51FCF73CFC6C
:10EF40004FF07C51FCF740FD2C490446FCF73CFD9A
:10EF50002B49FCF731FC2146FCF736FD2949FCF72B
:10EF600029FC2146FCF730FD2749FCF725FC21460A
:10EF7000FCF72AFD2549FCF71DFC2146FCF724FD82
:10EF80002349FCF719FC2146FCF71EFD06462046E6
:10EF900000F054FA1F4905462046FCF715FD1E49AE
:10EFA000FCF708FC2146FCF70FFD1C49FCF704FCAC
:10EFB0002146FCF709FD1A49FCF7FCFB2146FCF74A
:10EFC00003FD4FF07E51FCF7F7FB01463046FCF79E
:10EFD000AFFD2946FCF7F8FC1249FCF7EBFB0146B4
:10EFE0002846FCF7E9FB0146FCF7E6FB0146104822
:10EFF000FCF7E0FBF8BD00BFDB0FC93F08EF11389D
:10F00000047F4F3A4611243DA80A4E3E90B0A63EDA
:10F01000ABAA2A3E2EC69D3D6133303F2D5701409D
:10F0200039D119406821A233DA0FC93FDB0F4940BB
:10F03000DA0F494021F00042B2F1FF4FF8B5044623
:10F0400014DC20F00045B5F1FF4F06460EDCB1F1AF
:10F050007E5F3AD08F1707F0020747EAD07755B99D
:10F06000022F2FD0032F2FD13148F8BD084621465B
:10F07000FCF7A2FBF8BDFAB1B2F1FF4F29D0B5F110
:10F08000FF4F19D0AA1AD2153C2A19DC002938DB07
:10F090002046FCF74DFD00F0B5FF00F09DFE012F6E
:10F0A0002CD0022F22D0002F2FD02249FCF784FB36
:10F0B0002149FCF77FFBF8BD002E15DB1F48F8BD8A
:10F0C0001E48ECE71C48F8BDF8BDBDE8F84000F06C
:10F0D00083BEB5F1FF4F19D0022FF3D0032FC3D059
:10F0E000012F1BD00020F8BD1548F8BD1149FCF7D1
:10F0F00063FB01461048FCF75DFBF8BD00F10040E2
:10F10000F8BD3C32C4DA0020C9E7F8BD022F0CD0AC
:10F11000032F08D0012F04D00A48F8BD4FF000405B
:10F12000F8BD0948F8BD0948F8BD0948F8BD00BF59
:10F13000DB0F49C02EBDBB33DB0F4940DB0FC93F9E
:10F14000DB0FC9BFDB0F493FDB0F49BFE4CB16C064
:10F15000E4CB16402DE9F04FAB4A20F00044944236
:10F1600089B006460D4664DDA84A94421CDC00289E
:10F17000A74940F3EC80FCF71DFBA64B24F00F04DD
:10F180009C42064664D0A449FCF714FB0146286063
:10F190003046FCF70FFBA049FCF70CFB012368602D
:10F1A000184609B0BDE8F08F9C4A944262DDB4F184
:10F1B000FF4F46DAE715863FA4EBC7542046FCF71D
:10F1C000C9FDFCF7ADFB0346014620460593FCF75D
:10F1D000F1FA4FF08741FCF7F7FB8046FCF7BAFDE8
:10F1E000FCF79EFB0146044640460694FCF7E2FA13
:10F1F0004FF08741FCF7E8FB00210790FCF778FD12
:10F20000002800F0C58020460021FCF771FD002891
:10F2100014BF0123022382480221019000913A4643
:10F2200005A8294600F022FA002EC0F2A780034666
:10F2300003E00022286000234A60184609B0BDE8B8
:10F24000F08F0146FCF7B6FA002368602860F4E707
:10F250007449FCF7AFFA74490446FCF7ABFA01466F
:10F2600028602046FCF7A6FA6F49FCF7A3FA0123B1
:10F270006860E2E700F0C6FE6C490746FCF7A4FBB5
:10F280004FF07C51FCF798FAFCF764FD8246FCF7DE
:10F2900047FB5F498346FCF797FB01463846FCF77E
:10F2A00089FA5D4980465846FCF78EFBBAF11F0F7C
:10F2B00081464946404618DC5D4B0AF1FF3253F85F
:10F2C000223024F0FF029A420FD0FCF773FA07466F
:10F2D0002F6039464046FCF76DFA4946FCF76AFA5A
:10F2E000002E686056DB5346A7E7FCF763FAE31588
:10F2F000C0F3C7529A1A082A0746E9DD4949584619
:10F300000393FCF761FB074639464046FCF752FA87
:10F31000044621464046FCF74DFA3946FCF74AFAC6
:10F32000414907465846FCF74FFB3946FCF742FA7D
:10F33000814649462046FCF73DFA039BC0F3C7527D
:10F340009B1A192B074641DC2860A046C1E7FCF751
:10F3500033FA304B24F00F049C42064623D02E494A
:10F36000FCF72AFA014628603046FCF723FA2A49BE
:10F37000FCF722FA4FF0FF3368605EE795E80C0077
:10F3800003F1004102F1004243422A60696054E700
:10F39000032340E707F1004700F100402F60686059
:10F3A000CAF1000349E71F49FCF706FA1E49044663
:10F3B000FCF702FA014628602046FCF7FBF91A49DF
:10F3C000FCF7FAF94FF0FF33686036E71949584601
:10F3D000FCF7FAFA074639462046FCF7EBF9804677
:10F3E00041462046FCF7E6F93946FCF7E3F91249B5
:10F3F00004465846FCF7E8FA2146FCF7DBF981465B
:10F400004946404661E700BFD80F493FE3CB16406D
:10F41000800FC93FD00FC93F43443537800F494360
:10F42000A02E01080044353708A3852E84F9223F19
:10F43000202E010800A3852E32318D2420F00042B9
:10F44000B2F1FF4FF8B5044603462DD25AB3002857
:10F450003DDBB2F5000F4FEAE0502CD37F38C3F309
:10F460001603C20743F4000348BF5B0000274010A7
:10F470005B003E4619244FF08072B5189D4202DCB5
:10F480005B1BAE181744013C4FEA43034FEA52029C
:10F49000F3D113B107F001031F447F1007F17C572C
:10F4A00007EBC050F8BDF8BD0146FCF78DFA2146C8
:10F4B000FCF782F9F8BD14F400020FD15B001902C9
:10F4C00002F10102FAD5C2F101021044C6E7014679
:10F4D000FCF770F90146FCF72BFBF8BD0122104444
:10F4E000BCE700BF2DE9F84320F00046B6F1485FC5
:10F4F00005460F4649DAFCF72DFC002800F09D80F8
:10F5000029462846FCF760FA4E490446FCF75CFAA7
:10F510004D49FCF751F92146FCF756FA4B49FCF7E7
:10F5200049F92146FCF750FA4949FCF745F92146CB
:10F53000FCF74AFA4749FCF73DF92146FCF744FA43
:10F540004549FCF739F92146FCF73EFA804620464A
:10F550004FF07C51FCF738FA414606462046FCF74E
:10F5600033FA394604462846FCF72EFA014620466F
:10F57000FCF720F901463046FCF71CF901464FF034
:10F580007E50FCF717F9BDE8F8830146FCF71CFA3A
:10F590002C490446FCF718FA2B49FCF70DF92146D3
:10F5A000FCF712FA2949FCF705F92146FCF70CFA99
:10F5B0002749FCF701F92146FCF706FA2549FCF733
:10F5C000F9F82146FCF700FA2349FCF7F5F8214643
:10F5D000FCF7FAF9214B80469E42B8DD204B9E4253
:10F5E00027DC06F17F4631464FF07E50FCF7E2F80B
:10F5F000814620464FF07C51FCF7E6F93146FCF796
:10F60000D9F8414606462046FCF7DEF9394604465D
:10F610002846FCF7D9F901462046FCF7CBF801460D
:10F620003046FCF7C7F801464846FCF7C3F8BDE88A
:10F63000F883DFF834900B4EDBE74FF07E50BDE8E7
:10F64000F88300BF4ED747ADF6740F317CF2933488
:10F65000010DD037610BB63AABAA2A3D9999993E74
:10F660000000483F0000903E0000383F2DE9F04F79
:10F67000DFB00B93013B0293D31E48BF131DB84C60
:10F6800006466898DB1054F8204023EAE3730C9395
:10F69000DB4302EBC30308940693089C029B0C9A7D
:10F6A0001D190991C3EB02071DD4699C3D4404EB6D
:10F6B000870901354FF0000822AC0AE059F808002C
:10F6C000FCF72EF90137AF4244F8080008F10408AE
:10F6D00009D0002FF2DA01370020AF4244F80800C9
:10F6E00008F10408F5D1089A002AC0F2DF82089ACE
:10F6F0000B9B02F101089C0022AF4FEA88082744C7
:10F700000025029A002AC0F2F28105EB070B4FF0A8
:10F7100000094FF0000A56F809005BF8041DFCF7D9
:10F7200053F901465046FCF747F809F10409A14591
:10F730008246F0D14AA840F805A004354545E0D1FD
:10F74000089A0EAB03EB82030D9391464FEA8903AF
:10F750000793079A5EAB1344B9F1000F53F850AC0E
:10F7600023DD0DF134084AAF174490440DAD4FF03E
:10F770006E515046FCF728F9FCF7ECFAFCF7D0F88C
:10F780004FF087418346FCF71FF901465046FCF7CE
:10F7900011F8FCF7DFFA594645F8040F57F8040D45
:10F7A000FCF70AF845458246E1D15046069900F03B
:10F7B0008DFC4FF078510546FCF706F900F026FC69
:10F7C0004FF08241FCF700F901462846FBF7F2FFB3
:10F7D0000546FCF7BFFA8246FCF7A2F80146284628
:10F7E000FBF7E8FF069A8046002A40F3678109F19B
:10F7F000FF310EA850F82130C2F1080043FA00F2A0
:10F8000002FA00F01B1A06989244C0F1070743FA67
:10F8100007F70EA840F82130002F32DDB9F1000FB4
:10F820000AF1010A40F375810EAB079A194611449B
:10F83000002507E0C2F5807012B143F8040C0125E1
:10F840008B420BD053F8042B002DF3D0C2F1FF02F2
:10F850008B4243F8042C4FF00105F3D1069B002B9B
:10F860000DDD012B00F03281022B08D109F1FF33AD
:10F870000EA951F8232002F03F0241F82320022F65
:10F8800070D040460021FCF733FA002800F0838056
:10F89000089A09F1FF35AA420DDC079A0EAB0D98C4
:10F8A0001344002253F8041D834242EA0102F9D1B5
:10F8B000002A40F0E481089B0EA85A1E50F822301E
:10F8C000002B40F0F18100EB8202012352F8041D6D
:10F8D00001330029FAD04B4499450A933DDADDF80B
:10F8E0002CA022AACA44DDF8308002EB8A02C84468
:10F8F000C9EB0309131D03920593699A079B4FEA0D
:10F9000089094AAF02EB8808CDF810901F44002502
:10F9100058F8040FFCF704F8029B039A002B50518F
:10F920004FF0000B13DBDDF814A04FF00009AA44E0
:10F9300056F809005AF8041DFCF746F801465846E7
:10F94000FBF73AFF09F10409A1458346F0D1049A77
:10F950000435954247F804BFDAD1DDF82890F5E682
:10F96000B831010841464FF07E50FBF723FF804637
:10F97000002D86D006994FF07E5000F0A7FB01467F
:10F980004046FBF717FF804640460021FCF7B0F9E0
:10F9900000287FF47DAF069B40465942CDF808A071
:10F9A00000F094FB4FF087410446FCF7BFF90028B4
:10F9B00000F07F814FF06E512046FCF705F8FCF710
:10F9C000C9F9FBF7ADFF4FF087410546FBF7FCFF98
:10F9D00001462046FBF7EEFEFCF7BCF90EAB43F800
:10F9E00029002846FCF7B6F9069C09F10105083400
:10F9F0000EA9069441F8250006994FF07E5000F0BC
:10FA000065FB002D04464FDB6E1C4FEA8508C6EBF4
:10FA1000867A0DF138094AABC1444FEA8A0A984404
:10FA20004FF0000B59F80B00FBF77AFF2146FBF76C
:10FA3000CBFF4FF06E5148F80B002046FBF7C4FF98
:10FA4000ABF1040BD3450446ECD1DFF88C92DDF822
:10FA500020A00024B34603950497BAF1000FB8BF65
:10FA6000002515DB00263746002501E0A7420FDC04
:10FA700058F8061059F80600FBF7A6FF014628467D
:10FA8000FBF79AFE0137BA45054606F10406EDDAA2
:10FA90005EA800EB84030134A345A8F1040843F8F1
:10FAA000A05CDAD1039D049F689C032C00F298802F
:10FAB000DFE814F0CB009C009C00310010D109F16C
:10FAC000FF330EA951F823703F12A5E609F1FF3369
:10FAD0000EA850F8232002F07F0240F82320CEE643
:10FAE0004FF07C51FCF722F958B90746C9E64FF0B0
:10FAF000000A4AA840F805A0043545457FF401AE48
:10FB00001EE6B9F1000F4FF002070AF1010A3FF7B4
:10FB10008BAE0025A2E6002D40F3DC804FEA850B7A
:10FB20005EAB36AE05F1FF3A5B4406EB8A0A53F84A
:10FB3000A08C54465B4635AABB462F4600E0C8461B
:10FB400054F804594146284601920093FBF734FECD
:10FB5000814649462846FBF72DFE4146FBF72CFE21
:10FB6000019AC4F804909442A060009BE7D13D46FE
:10FB7000012D5F469B4640F3AD805EAB9B445BF836
:10FB8000A04C00E044465AF8049921464846FBF749
:10FB900013FE804641464846FBF70CFE2146FBF724
:10FBA0000BFE5645CAF80480CAF80800EAD16C1C5E
:10FBB00006EB84040020083654F8041DFBF7FCFD16
:10FBC000B442F9D1002F7ED0369A379B099C00F1C0
:10FBD000004002F1004203F10043A0602260636034
:10FBE000029A02F007005FB0BDE8F08F002DB8BFA9
:10FBF00000200ADB36AE6C1C002006EB840454F8AF
:10FC0000041DFBF7D9FDB442F9D1002F35D000F126
:10FC10000043099C014623603698FBF7CBFD002D7D
:10FC200008DD36AC04EB850554F8041FFBF7C4FD72
:10FC3000AC42F9D10FB100F10040099A5060029A2C
:10FC400002F007005FB0BDE8F08F002D39DB6C1CBF
:10FC500036AE002006EB840454F8041DFBF7ACFD1F
:10FC6000B442F9D10FB100F10040099A1060029A34
:10FC700002F007005FB0BDE8F08F0346C9E7069ABF
:10FC80000EAC54F82530083ACDF808A00692002BA7
:10FC90007FF4B2AE04EB850353F8041D013D083A2E
:10FCA0000029F9D00692A7E6012314E60B9B9C00DD
:10FCB00046E52046FCF74EF80EAA4D4642F82900CC
:10FCC0009AE60020CEE7099C369A379BA060226016
:10FCD000636085E7002075E7C43101082DE9F8432A
:10FCE00020F00043B3F1485F04460F46904603DA24
:10FCF000FCF730F8002857D021462046FBF764FE79
:10FD000021460546FBF760FE294906462846FBF7D3
:10FD10005BFE2849FBF74EFD2946FBF755FE2649B9
:10FD2000FBF74AFD2946FBF74FFE2449FBF742FD4E
:10FD30002946FBF749FE2249FBF73EFD8146B8F113
:10FD4000000F22D038464FF07C51FBF73DFE49466C
:10FD500080463046FBF738FE01464046FBF72AFD59
:10FD60002946FBF731FE3946FBF724FD15490546C8
:10FD70003046FBF729FE01462846FBF71DFD0146EC
:10FD80002046FBF717FDBDE8F88349462846FBF7F8
:10FD90001BFE0C49FBF70EFD3146FBF715FE214615
:10FDA000FBF70AFDBDE8F8832046BDE8F88300BFF5
:10FDB000D3C92E2F342FD7321BEF3836010D5039CF
:10FDC0008988083CABAA2A3E0020704700200149E0
:10FDD000704700BF0000F87F2DE9F04120F000459A
:10FDE000B5F1A14F0446064608DBB5F1FF4F6FDCC5
:10FDF000002840F3A0806F48BDE8F0816E4B9D4223
:10FE000077DCB5F1445F68DB4FF0FF3721462046D1
:10FE1000FBF7DAFD01468046FBF7D6FD674905464C
:10FE2000FBF7D2FD6649FBF7C7FC2946FBF7CCFD83
:10FE30006449FBF7C1FC2946FBF7C6FD6249FBF7A5
:10FE4000BBFC2946FBF7C0FD6049FBF7B5FC294622
:10FE5000FBF7BAFD5E49FBF7AFFC4146FBF7B4FD8B
:10FE60005C4980462846FBF7AFFD5B49FBF7A2FCE7
:10FE70002946FBF7A9FD5949FBF79CFC2946FBF7EE
:10FE8000A3FD5749FBF796FC2946FBF79DFD554915
:10FE9000FBF790FC2946FBF797FD7B1C014640468B
:10FEA0004CD0FBF789FC2146FBF78EFD4E4B4F4DA6
:10FEB00053F82710FBF77EFC2146FBF77BFC01463D
:10FEC00055F82700FBF776FC002E30DBBDE8F0810B
:10FED0000146FBF771FCBDE8F0814549FBF76CFC7E
:10FEE0004FF07E51FBF72CFF00288DD02046BDE857
:10FEF000F08100F087F83F4B04469D4229DCA3F5D2
:10FF0000D0039D4244DC0146FBF756FC4FF07E5186
:10FF1000FBF750FC4FF0804105462046FBF74CFCB8
:10FF200001462846FBF704FE002704466EE700F171
:10FF30000040BDE8F0813048BDE8F081FBF73CFCB3
:10FF40002146FBF741FD01462046FBF733FCBDE8A7
:10FF5000F0812A4B9D4214DC4FF07F51FBF72AFCC5
:10FF60004FF07F5105462046FBF72EFD4FF07E51A6
:10FF7000FBF722FC01462846FBF7DAFD0227044680
:10FF800044E701461E48FBF7D3FD032704463DE73F
:10FF90004FF07E51FBF70EFC4FF07E510546204698
:10FFA000FBF70AFC01462846FBF7C2FD0127044681
:10FFB0002CE700BFDB0FC93FFFFFDF3ED769853C61
:10FFC00059DA4B3D356B883D6E2EBA3D2549123EC0
:10FFD000ABAAAA3E21A215BD6BF16E3D95879D3D52
:10FFE000388EE33DCDCC4C3EF031010800320108A3
:10FFF000CAF24971FFFF973FDB0FC9BFFFFF1B40EC
:020000040801F1
:10000000000080BF20F00040704700BF2DE9F041A4
:1000100020F00047FD0D7F3D162D064613DC002D18
:1000200080461BDB194F2F41074214D01849FBF7BC
:10003000C3FB0021FBF784FE68B1002E1BDB28EA1E
:100040000700BDE8F081B7F1FF4F04D30146FBF78D
:10005000B3FBBDE8F0813046BDE8F0810C49FBF709
:10006000ABFB0021FBF76CFE0028F4D0002E08DB70
:100070000020BDE8F0814FF4000343FA05F5A844E1
:10008000DDE7002FE7D00348BDE8F081FFFF7F00E8
:10009000CAF24971000080BF30F0004001D1022057
:1000A0007047A0F50003B3F1FE4F01D20420704762
:1000B000054B421E9A4201D803207047B0F1FF431E
:1000C00058425841704700BFFEFF7F0038B530F0FE
:1000D0000044024603460D4614D0B4F1FF4F0DD242
:1000E000B4F5000F0FD3E40D2C44FE2C2EDC002CB5
:1000F0001DDD23F0FF4343EAC45038BD0146FBF742
:100100005BFB38BD38BD4FF09841FBF75DFC194BE8
:1001100002469D4207DBC0F3C7540346193CE3E7A0
:10012000154800F02DF81449FBF74EFC38BD14F1CA
:10013000160F13DA4CF250339D421146F0DD0F4892
:1001400000F01EF80D49FBF73FFC38BD11460B4887
:1001500000F016F80949FBF737FC38BD04F1190027
:1001600023F0FF4343EAC0504FF04C51FBF72CFC07
:1001700038BD00BFB03CFFFF6042A20DCAF249711A
:1001800001F0004120F0004008437047014B18681F
:10019000704700BFF40000200001746564666D6A5A
:1001A00069736C67780000FFF00000FF010B020D1F
:1001B0000A03050B030D0A030A0B040D0A03080BBF
:1001C000040D0A033C0000FF000000FFD20000FF06
:1001D0005A0000FF1E0000FF4A0100FF2C0100FF33
:1001E0000E0100FFB40000FF960000FF0000FFFFBB
:1001F000CC180108EC010108C8010108D40101086C
:10020000C4010108D0010108A4010108E8010108A6
:10021000E4010108CC010108A8010108E00101087E
:10022000DC010108D801010800000000000C0140B9
:1002300008001002000C014004001402000000003D
:100240000000000003010000840801080400000011
:10025000440801080400000004080108020100002D
:10026000E407010800010000000000000600000093
:1002700084070108060000002407010801010000AE
:100280000000000004000000E40601080600000071
:1002900084060108080000000406010808000000A8
:1002A00084050108080000000405010801010000A0
:1002B000000000000001000000000000000100003C
:1002C0000000000004000000C40401080600000053
:1002D00064040108000100000000000002010000A9
:1002E00044040108010100000000000000000000BB
:1002F00000000000020000008025000000C2010094
:1003000000000000100000008025000000C2010075
:1003100001000000200000008025000000C2010054
:1003200000000000010000008025000000C2010064
:1003300000000000080000008025000000C201004D
:10034000000300000400000080250000004B0000B6
:10035000000000002A04010810040108F603010847
:10036000DC030108A5180008611800083D18000802
:100370001518000805180008F1AD000891180008CC
:10038000B51700088518000877180008000000005D
:1003900000C2010090190108B31901080100000012
:1003A00000E10000C8190108EA1901080200000074
:1003B00000960000FE190108201A01080300000041
:1003C000004B0000341A0108561A0108040000000E
:1003D000802500000F1C01080F1C01080001060306
:1003E0000703080409040A040B04010402040304BB
:1003F00004040504FFFF00020102020203020402DA
:10040000050206030703080409040A040B04FFFF9E
:10041000000106030703080309030A030B03010392
:100420000203030304030503FFFF000201020202AB
:1004300003020402050206030703080309030A0373
:100440000B03FFFF0000803F0000000000000000E1
:10045000000080BF0000803F00000000000000009E
:100460000000803F0000803F000080BF0000803F10
:10047000000080BF0000803F000080BF000080BF00
:100480000000803F0000803F0000803F0000803F70
:100490000000803F0000803F0000803F000080BFE0
:1004A000000080BF0000803F00000000000000004E
:1004B000000000000000803F00000000000000007D
:1004C000000000000000803F000000000000803FAE
:1004D0000000803F0000803F000080BF000080BF20
:1004E000000000000000803F000000000000803F8E
:1004F000000080BF0000803F0000803F000080BF00
:10050000000000800000803F0000803F000000BF2E
:100510000000803F0000803F000000BF000080BF5F
:100520000000803F0000803F000080BF0000003FCF
:100530000000803F0000803F0000003F0000803F3F
:100540000000803F0000803F0000003F000080BFAF
:10055000000080BF0000803F000080BF000000BF9F
:10056000000080BF0000803F000000BF0000803F0F
:10057000000080BF0000803F0000803F0000003F7F
:10058000000080BF0000803FF704353FF70435BF0F
:100590000000803F0000803FF70435BFF70435BFFF
:1005A0000000803F0000803FF70435BFF704353F6F
:1005B0000000803F0000803FF704353FF704353FDF
:1005C0000000803F0000803F00000000000080BF6E
:1005D000000080BF0000803F000080BF00000000DE
:1005E000000080BF0000803F000000000000803F4E
:1005F000000080BF0000803F0000803F000000003E
:10060000000080BF0000803F000080BF0000803FEE
:10061000000080BF0000803F000080BF000080BF5E
:100620000000803F0000803F0000803F0000803FCE
:100630000000803F0000803F0000803F000080BF3E
:10064000000080BF0000803F000080BF0000803FAE
:100650000000803F0000803F000080BF000080BF9E
:10066000000080BF0000803F0000803F0000803F0E
:10067000000080BF0000803F0000803F000080BF7E
:100680000000803F0000803F000000BFD0B35D3F0E
:100690000000803F0000803F000000BFD0B35DBF7E
:1006A0000000803F0000803F0000003FD0B35D3F6E
:1006B000000080BF0000803F0000003FD0B35DBF5E
:1006C000000080BF0000803F000080BF00000000ED
:1006D000000080BF0000803F0000803F000000005D
:1006E0000000803F0000803F000000000000803FCD
:1006F000000080BF0000803F000080BF000080BF7E
:10070000000000000000803F000000000000803F6B
:100710000000803F0000803F0000803F000080BF5D
:10072000000000000000803FD0B35DBF0000003F2C
:100730000000803F0000803FD0B35DBF000000BFDD
:10074000000080BF0000803FD0B35D3F0000003F4D
:100750000000803F0000803FD0B35D3F000000BF3D
:10076000000080BF0000803F00000000000080BF4C
:100770000000803F0000803F000000000000803F3C
:10078000000080BF0000803F00000000A8AAAA3F30
:100790000000803F0000803F000080BFB0AA2ABF59
:1007A000000080BF0000803F0000803FB0AA2ABF49
:1007B000000080BF0000803F00000000A8AAAA3F00
:1007C000000080BF0000803F000080BFB0AA2ABFA9
:1007D0000000803F0000803F0000803FB0AA2ABF99
:1007E0000000803F0000803F0000803F00000000CC
:1007F000000000000000803F000080BF00000000FB
:10080000000000000000803F000080BF0000803F2B
:10081000000080BF0000803F000080BF000080BF5C
:100820000000803F0000803F0000803F0000803FCC
:100830000000803F0000803F0000803F000080BF3C
:10084000000080BF0000803F000000000000803FEB
:10085000000080BF0000803F000080BF000000005B
:100860000000803F0000803F0000803F000000004B
:100870000000803F0000803F00000000000080BFBB
:10088000000080BF0000803F00000000A8AAAA3F2F
:10089000000000000000803F000080BFB0AA2ABF17
:1008A000000000000000803F0000803FB0AA2ABF87
:1008B00000000000002C0140000000400004004047
:1008C00000080040010001020001030001040001D2
:1008D0000500010600010700010800010900010AE6
:1008E00000010B00010C0103000000008F1A010839
:1008F0000000000001000000941A0108010000003F
:10090000020000009B1A0108020000000300000022
:10091000A41A01080300000004000000AA1A01083C
:100920000500000005000000AF1A010806000000E5
:1009300006000000B91A01080700000007000000C7
:10094000C21A01080800000008000000CB1A0108C4
:100950000900000009000000D41A01080A00000084
:100960000A000000DE1A01080B0000000B00000066
:10097000E81A01080C0000000C000000F21A01083F
:100980000D0000000D000000FA1A01080E00000022
:100990000E000000021B01080F0000000F00000005
:1009A0000A1B01081000000010000000131B0108C2
:1009B00011000000110000001A1B010812000000C5
:1009C00012000000241B01081300000013000000A7
:1009D0002C1B01081400000014000000371B010844
:1009E0001500000015000000411B01081600000062
:1009F0001600000000000000FF000000B5620601C4
:100A00000300F00500FF19B56206010300F00300C2
:100A1000FD15B56206010300F00100FB11B5620689
:100A2000010300F00000FA0FB56206010300F002B6
:100A300000FC13B56206010300F00400FE17B56266
:100A4000060103000102010E47B562060103000121
:100A500003010F49B56206010300010601124FB5FB
:100A600062060103000112011E67B5620608060056
:100A7000C80001000100DE6A00B562061608000326
:100A80000703000000000031E501B562061608000A
:100A900003070300510800008A4102B562061608E8
:100AA000000307030004E00400199D03B562061665
:100AB0000800030703000002020035EF04B56206D8
:100AC0001608000307030080010000B2E8000001DF
:100AD0001E1E646464646464220046022100820174
:100AE00020004302100001010000490201008801BA
:100AF00002004C02120084011100900111009001CB
:100B00001100A0011100A0010000040008000C0069
:100B10004000800000010002000449574641540192
:100B200002040810204E45535755442C3A3A000011
:100B300091940008ED180008BB180008518F0008B8
:100B4000091900084D8F0008942101089B21010814
:100B5000A0210108B1210108BB210108C62101081B
:100B6000D1210108DC210108E0210108E921010867
:100B7000EF210108F92101080B1F010807220108D4
:100B8000172201081E22010827220108312201082C
:100B9000000000009A1F0108A31F0108C987000870
:100BA000C71F0108CB1F0108FD880008E11F0108CD
:100BB000E61F0108B1720008FA1F010800200108B1
:100BC0007D760008261C010811200108956B00089D
:100BD0002E200108332001088DA900086220010899
:100BE0000F1C0108A95E0008672001086F2001089A
:100BF000FD7900088320010887200108B18A0008D8
:100C00009A200108A9200108097E0008C3200108D4
:100C10000F1C0108E1710008C8200108CC20010860
:100C2000796F0008DB200108DF2001080D72000841
:100C3000F41F0108FB200108417500080E2101087E
:100C400014210108DD750008B02A01082F210108D0
:100C500041A900083E2101082F210108456500082F
:100C60004A2101084F210108D55E0008511D0108E5
:100C70005F2101080D8B00088D21010881210108E9
:100C8000997F0008742801080F1C0108B171000841
:100C9000192301081E230108222301082B23010820
:100CA000E9210108DC2101082723010800000000D8
:100CB0000F1C0108D5220108DD220108E5220108E8
:100CC000ED220108F4220108FF2201080723010890
:100CD0000F23010814230108000000000000000099
:100CE0008025000000C20100020000000200000098
:100CF0008025000000C20100030000000300000086
:100D000080250000004B0000050000009001C80095
:100D1000C800C800C800C800C800C800C8006400F7
:100D20000000C800C800C800C80032001F19000831
:100D30003D19000859190008419800088519000854
:100D400091190008524F4C4C3B50495443483B5971
:100D500041573B414C543B506F733B506F73523B78
:100D60004E6176523B4C4556454C3B4D41473B56B8
:100D7000454C3B00A81C01089F1C0108931C01085E
:100D8000E2240108E6240108EC240108F224010809
:100D9000F5240108FC240108FF24010804250108AA
:100DA000102501081325010819250108202501082F
:100DB0002A250108342501083D2501084B25010895
:100DC000572501085E2501086425010871250108E1
:100DD0007C250108892501080000000099250108EB
:100DE00044000000E4190020000000002823000057
:100DF000A225010841000000E619002000000000C3
:100E000001000000B025010844000000F01A002095
:100E1000B0040000A4060000B7250108440000004B
:100E2000F21A002000000000D0070000C1250108D0
:100E300044000000F41A002000000000D007000069
:100E4000CB25010842000000F61A00200000000037
:100E500012000000D825010842000000F71A002007
:100E600001000000FF000000E3250108420000002F
:100E7000F81A00200000000001000000F825010819
:100E800044000000A81A002000000000D007000065
:100E90000526010844000000AA1A002000000000F6
:100EA000D00700001226010844000000AC1A002000
:100EB00000000000D00700001E26010844000000CA
:100EC000AE1A002000000000D00700002E26010806
:100ED00044000000B01A002000000000D00700000D
:100EE0003F26010844000000B21A00200000000064
:100EF000D00700004A26010844000000B41A002070
:100F000000000000D00700005F2601084400000038
:100F1000B61A002032000000007D00006E26010895
:100F200044000000B81A002032000000F201000066
:100F30007D26010841000000F91A00200000000091
:100F4000010000008A26010841000000FA1A002072
:100F500000000000010000009D2601084100000083
:100F6000FB1A002000000000B4000000A9260108C0
:100F700041000000FC1A0020000000006400000096
:100F8000B526010842000000FD1A0020FFFFFFFF08
:100F900001000000CB26010841000000041B0020D6
:100FA0000000000008000000E226010841000000E7
:100FB000051B00200000000008000000F9260108C1
:100FC00041000000061B0020000000000800000097
:100FD0001027010841000000181B0020300000000D
:100FE0007E0000002127010850000000081B00209F
:100FF000B004000000C201002E27010850000000CC
:101000000C1B0020B004000000C201003B270108B7
:1010100050000000101B00200000000000C2010072
:101020004827010850000000141B0020B0040000F5
:1010300000C201006127010841000000FE1A0020E3
:1010400000000000010000006E27010841000000C0
:10105000FF1A002000000000040000007C270108A7
:1010600041000000001B0020000000000100000003
:101070008C27010881000000F41B00200000000004
:10108000C80000009627010881000000FE1B002018
:1010900000000000C8000000A02701088100000037
:1010A000081C002000000000C8000000AA2701085A
:1010B00081000000F51B002000000000C8000000B7
:1010C000B527010881000000FF1B00200000000080
:1010D000C8000000C027010881000000091C002092
:1010E00000000000C8000000CB27010881000000BC
:1010F000F61B002000000000C8000000D5270108F2
:1011000081000000001C002000000000C80000005A
:10111000DF270108810000000A1C002000000000F9
:10112000C8000000E9270108840000009E1D00207F
:1011300000000000D0070000F72701088100000030
:10114000A21D002000000000010000000C28010882
:1011500084000000A41D00200A000000D007000049
:101160001A28010884000000A61D00200A000000C3
:10117000D00700002828010881000000A11D0020E0
:101180000000000064000000362801084100000053
:10119000EE1A0020000000000300000048280108AB
:1011A000410000001C1B00200000000002000000A5
:1011B0005B280108410000001D1B0020000000000A
:1011C000010000006C280108410000001E1B0020E7
:1011D00000000000010000007C2801086000000001
:1011E000201B0020A6FFFFFF5A00000094280108E2
:1011F00060000000241B00204CFFFFFFB400000033
:10120000AC28010841000000281B0020000000005D
:1012100001000000C528010841000000291B002032
:101220000000000001000000D02801084400000078
:101230002A1B002000000000204E0000E3280108C7
:1012400041000000DC1A002000000000FF00000048
:10125000EE28010841000000DD1A00200A0000000D
:10126000320000000429010841000000DE1A0020BD
:101270000A000000320000001A29010844000000A2
:10128000E01A002001000000102700002E290108AC
:1012900044000000E21A0020000000007206000076
:1012A0004329010841000000E41A0020000000006A
:1012B000010000006129010841000000BA1A002065
:1012C00000000000080000006C2901084100000037
:1012D000BB1A002000000000080000007629010869
:1012E00041000000BC1A00200000000008000000BF
:1012F0008029010848000000BE1A00204CFFFFFFB3
:10130000680100009129010848000000C01A00206F
:101310004CFFFFFF68010000A329010848000000FE
:10132000C21A00204CFFFFFF68010000B32901082A
:1013300044000000CE1A0020640000008403000076
:10134000C929010844000000C61A0020000000005E
:1013500000010000D229010841000000CC1A002041
:101360000000000080000000E229010844000000A5
:10137000C81A002064000000E8030000F3290108F7
:1013800044000000CA1A002064000000E8030000C6
:10139000052A0108810000004B1D0020010000000B
:1013A000FA000000172A0108810000004C1D0020EF
:1013B00000000000010000000E2A0108810000006A
:1013C000491D002000000000200000002C2A010818
:1013D000810000004A1D00200000000064000000A1
:1013E000392A010881000000501D00200000000083
:1013F00096000000532A0108840000004E1D0020C2
:1014000001000000840300006D2A01084200000072
:10141000C41A0020FFFFFFFF01000000832A01081B
:10142000820000009A1D0020FFFFFFFF0100000066
:10143000912A0108820000009B1D0020000000008E
:1014400001000000A32A0108810000003C1C0020CC
:101450000000000002000000B82A0108010100009D
:101460002E21002000000000FA000000C02A010820
:10147000010100002F210020000000006400000096
:10148000C82A0108010100003021002000000000EE
:1014900064000000D02A0108010100003121002071
:1014A0000000000064000000D92A010801010000CA
:1014B000322100200000000064000000E92A010839
:1014C0000101000033210020000000006400000042
:1014D000F22A010801010000342100200000000070
:1014E00064000000FB2A01080401000036210020EE
:1014F000E8030000D00700000A2B0108810000006B
:10150000921D002000000000C8000000192B0108F7
:1015100081000000931D002000000000C8000000B2
:101520002C2B010884000000941D0020E80300001B
:10153000D00700003E2B010884000000961D00200B
:1015400064000000D0070000502B01088400000058
:10155000981D002064000000B80B0000622B0108F9
:10156000810000009C1D002000000000FF00000022
:101570006F2B010841000000C51A00200000000088
:10158000090000007C2B010881000000441C0020A1
:1015900000000000FA0000008B2B01088100000011
:1015A0004C1C002000000000640000009A2B010881
:1015B000810000004D1C00200000000064000000BD
:1015C000A82B0108A0000000481C0020010000001A
:1015D00014000000B82B010881000000601C0020EE
:1015E0000000000001000000C72B01088800000077
:1015F000421C0020D4FEFFFF2C010000D62B010866
:1016000088000000401C0020D4FEFFFF2C010000D9
:10161000E42B010881000000501C002000000000A5
:1016200030000000F22B0108A0000000541C002034
:101630000000000001000000012C0108A0000000D3
:10164000581C002000000000010000000D2C0108C3
:10165000A00000005C1C0020000000000100000051
:10166000192C0108880000003E1C0020B0B9FFFFC3
:1016700050460000292C010881000000EC1B0020CE
:101680000000000002000000382C0108810000006A
:10169000F11B002000000000C8000000402C0108E1
:1016A00081000000FB1B002000000000C8000000BB
:1016B0009B29010881000000051C0020000000009B
:1016C000C8000000482C010881000000F01B002029
:1016D00000000000C80000004F2C0108810000003D
:1016E000FA1B002000000000C80000008A29010841
:1016F00081000000041C002000000000C800000061
:10170000562C010881000000F21B002000000000A0
:10171000C80000005C2C010881000000FC1B0020B8
:1017200000000000C8000000AD2901088100000091
:10173000061C002000000000C8000000622C010808
:10174000A0000000141C0020000000006400000045
:101750006B2C0108A0000000201C002000000000ED
:1017600064000000742C0108A00000002C1C002064
:1017700000000000640000007D2C0108A0000000B3
:10178000101C00200000000064000000852C0108EF
:10179000A00000001C1C00200000000064000000ED
:1017A0008D2C0108A0000000281C00200000000073
:1017B00064000000952C0108A0000000181C002007
:1017C00000000000640000009C2C0108A000000044
:1017D000241C00200000000064000000A32C01086D
:1017E000A0000000301C0020000000006400000089
:1017F000AA2C0108A0000000381C002000000000F6
:101800000A000000B82C0108A0000000341C0020D1
:10181000000000000A000000C42C01088100000044
:10182000F31B002000000000C8000000CA2C0108C3
:1018300081000000FD1B002000000000C800000027
:10184000D02C010881000000071C002000000000CF
:10185000C8000000D62C010881000000F71B002002
:1018600000000000C8000000DE2C0108810000001C
:10187000011C002000000000C8000000E62C010848
:10188000810000000B1C002000000000C8000000C8
:10189000EE2C010881000000F91B00200000000070
:1018A000C8000000F42C010881000000031C002087
:1018B00000000000C8000000FA2C010881000000B0
:1018C0000D1C002000000000C80000000000000007
:1018D00000080040000C014040000000001E0028ED
:1018E00000040040000C014020000000041D0028FE
:1018F00000040040000C014001000000081D002809
:1019000000040040000C0140020000000C1D0028F3
:10191000000000400008014001000000001C0028F9
:10192000000000400008014002000000041C0028E4
:1019300000080040000C0140000200000C1E0118CD
:1019400000080040000C014000010000081E0118C2
:1019500000080040000C014080000000041E011837
:10196000002C01400008014000010000001B01188C
:1019700000040040000C014010000000001D011890
:10198000000000400008014004000000081C01188D
:1019900024505542582C34312C312C303030332CDB
:1019A000303030312C3131353230302C302A314525
:1019B0000D0A0024504D544B3235312C3131353223
:1019C00030302A31460D0A0024505542582C34310B
:1019D0002C312C303030332C303030312C35373600
:1019E00030302C302A32440D0A0024504D544B32F2
:1019F00035312C35373630302A32430D0A00245029
:101A00005542582C34312C312C303030332C30307E
:101A100030312C33383430302C302A32360D0A0035
:101A200024504D544B3235312C33383430302A3237
:101A3000370D0A0024505542582C34312C312C30AB
:101A40003030332C303030312C31393230302C3092
:101A50002A32330D0A0024504D544B3235312C318B
:101A6000393230302A32320D0A00303132333435D7
:101A7000363738394142434445464748494A4B4C3A
:101A80004D4E4F505152535455565758595A004184
:101A9000524D3B00414E474C453B00484F52495A3E
:101AA0004F4E3B004241524F3B004D41473B0048A7
:101AB000454144465245453B004845414441444A1E
:101AC0003B0043414D535441423B0043414D54522E
:101AD00049473B0047505320484F4D453B00475036
:101AE0005320484F4C443B005041535354485255A7
:101AF0003B004245455045523B004C45444D415802
:101B00003B004C45444C4F573B004C4C49474854D4
:101B1000533B0043414C49423B00474F5645524ED0
:101B20004F523B004F53442053573B0054454C45C4
:101B30004D455452593B004155544F54554E453B29
:101B400000534F4E41523B002E0000271008042343
:101B50000220010D0A5265626F6F74696E67000D95
:101B60000A4C656176696E6720434C49206D6F644D
:101B7000652C20756E7361766564206368616E679D
:101B80006573206C6F73742E0D0A00536176696E55
:101B900067007261746570726F66696C6520256498
:101BA0000D0A000D0A456E746572696E6720434C1C
:101BB00049204D6F64652C20747970652027657805
:101BC00069742720746F2072657475726E2C206F93
:101BD00072202768656C70270D0A000D0A2320000B
:101BE0000D1B5B4B001B5B324A1B5B313B314800DA
:101BF000556E6B6E6F776E20636F6D6D616E642CCA
